******************************************************************************
                  TI ARM Linker PC v5.2.5                      
******************************************************************************
>> Linked Wed Sep 09 11:49:39 2015

OUTPUT FILE NAME:   <CIO_test_ARM_CPP.out>
ENTRY POINT SYMBOL: "_c_int00"  address: 80021380


MEMORY CONFIGURATION

         name            origin    length      used     unused   attr    fill
----------------------  --------  ---------  --------  --------  ----  --------
  SRAM                  402f0400   0000fc00  00000000  0000fc00  RWIX
  L3OCMC0               40300000   00010000  000034b2  0000cb4e  RWIX
  M3SHUMEM              44d00000   00004000  00000000  00004000  RWIX
  M3SHDMEM              44d80000   00002000  00000000  00002000  RWIX
  DDR0                  80000000   40000000  00023e3c  3ffdc1c4  RWIX


SEGMENT ALLOCATION MAP

run origin  load origin   length   init length attrs members
----------  ----------- ---------- ----------- ----- -------
40300000    40300000    000018e6   000018e6    r--
  40300000    40300000    000018e6   000018e6    r-- .const
403018e8    403018e8    00001a88   00000000    rw-
  403018e8    403018e8    00000800   00000000    rw- .stack
  403020e8    403020e8    00000800   00000000    rw- .sysmem
  403028e8    403028e8    000007cc   00000000    rw- .data
  403030b4    403030b4    000002bc   00000000    rw- .bss
40303370    40303370    00000148   00000148    r--
  40303370    40303370    0000001c   0000001c    r-- .init_array
  40303390    40303390    00000128   00000128    r-- .cinit
80000000    80000000    00023e3c   00023e3c    r-x
  80000000    80000000    00023e3c   00023e3c    r-x .text


SECTION ALLOCATION MAP

 output                                  attributes/
section   page    origin      length       input sections
--------  ----  ----------  ----------   ----------------
.const     0    40300000    000018e6     
                  40300000    00000202     rtsv7A8_A_le_eabi.lib : xlocinfo.obj (.const:_ZSt8_Ctyptab)
                  40300202    00000101                           : ctype.obj (.const:.string:_ctypes_)
                  40300303    00000001                           : xlocale.obj (.const:.string:_ZZNSt7_MpunctIcE5_InitERKSt8_LocinfoEs)
                  40300304    000000b0                           : strftime.obj (.const:.string)
                  403003b4    00000087                           : wlocale.obj (.const:.string:_ZZNKSt8_Locinfo10_GetmonthsEvEs)
                  4030043b    00000079                           : xlocale.obj (.const:.string:_ZZNSt7_MpunctIcE7_MakpatERNSt10money_base7patternEjjjEs_0)
                  403004b4    00000079                           : wlocale.obj (.const:.string:_ZZNSt7_MpunctIwE7_MakpatERNSt10money_base7patternEjjjEs_0)
                  4030052d    00000056                           : wlocale.obj (.const:.string:_ZZNKSt8_Locinfo8_GetdaysEvEs)
                  40300583    00000005     SimpleClass.obj (.const:.string:_ZZNKSt8_Locinfo8_GettrueEvEs)
                  40300588    00000050     rtsv7A8_A_le_eabi.lib : strtod.obj (.const:digits)
                  403005d8    00000048                           : iostream.obj (.const:_ZTVSt13basic_filebufIcSt11char_traitsIcEE)
                  40300620    00000048                           : wiostrea.obj (.const:_ZTVSt13basic_filebufIwSt11char_traitsIwEE)
                  40300668    00000048                           : iostream.obj (.const:_ZTVSt15basic_streambufIcSt11char_traitsIcEE)
                  403006b0    00000048                           : wiostrea.obj (.const:_ZTVSt15basic_streambufIwSt11char_traitsIwEE)
                  403006f8    00000048                           : strtod.obj (.const:powerof10)
                  40300740    00000040                           : wiostrea.obj (.const:_ZTVSt5ctypeIwE)
                  40300780    0000003c                           : xlocale.obj (.const:.typeinfo:_ZTSSt9money_getIcSt19istreambuf_iteratorIcSt11char_traitsIcEEE)
                  403007bc    0000003c                           : wlocale.obj (.const:.typeinfo:_ZTSSt9money_getIwSt19istreambuf_iteratorIwSt11char_traitsIwEEE)
                  403007f8    0000003c                           : xlocale.obj (.const:.typeinfo:_ZTSSt9money_putIcSt19ostreambuf_iteratorIcSt11char_traitsIcEEE)
                  40300834    0000003c                           : wlocale.obj (.const:.typeinfo:_ZTSSt9money_putIwSt19ostreambuf_iteratorIwSt11char_traitsIwEEE)
                  40300870    0000003c                           : locale.obj (.const:_ZTVSt7num_getIcSt19istreambuf_iteratorIcSt11char_traitsIcEEE)
                  403008ac    0000003c                           : wlocale.obj (.const:_ZTVSt7num_getIwSt19istreambuf_iteratorIwSt11char_traitsIwEEE)
                  403008e8    0000003b                           : xlocale.obj (.const:.typeinfo:_ZTSSt8time_getIcSt19istreambuf_iteratorIcSt11char_traitsIcEEE)
                  40300923    0000003b                           : wlocale.obj (.const:.typeinfo:_ZTSSt8time_getIwSt19istreambuf_iteratorIwSt11char_traitsIwEEE)
                  4030095e    0000003b                           : xlocale.obj (.const:.typeinfo:_ZTSSt8time_putIcSt19ostreambuf_iteratorIcSt11char_traitsIcEEE)
                  40300999    0000003b                           : wlocale.obj (.const:.typeinfo:_ZTSSt8time_putIwSt19ostreambuf_iteratorIwSt11char_traitsIwEEE)
                  403009d4    0000003a                           : locale.obj (.const:.typeinfo:_ZTSSt7num_getIcSt19istreambuf_iteratorIcSt11char_traitsIcEEE)
                  40300a0e    0000003a                           : wlocale.obj (.const:.typeinfo:_ZTSSt7num_getIwSt19istreambuf_iteratorIwSt11char_traitsIwEEE)
                  40300a48    0000003a     SimpleClass.obj (.const:.typeinfo:_ZTSSt7num_putIcSt19ostreambuf_iteratorIcSt11char_traitsIcEEE)
                  40300a82    0000003a     rtsv7A8_A_le_eabi.lib : wlocale.obj (.const:.typeinfo:_ZTSSt7num_putIwSt19ostreambuf_iteratorIwSt11char_traitsIwEEE)
                  40300abc    00000034                           : xlocale.obj (.const:_ZTVSt10moneypunctIcLb0EE)
                  40300af0    00000034                           : xlocale.obj (.const:_ZTVSt10moneypunctIcLb1EE)
                  40300b24    00000034                           : wlocale.obj (.const:_ZTVSt10moneypunctIwLb0EE)
                  40300b58    00000034                           : wlocale.obj (.const:_ZTVSt10moneypunctIwLb1EE)
                  40300b8c    00000034                           : xlocale.obj (.const:_ZTVSt7_MpunctIcE)
                  40300bc0    00000034                           : wlocale.obj (.const:_ZTVSt7_MpunctIwE)
                  40300bf4    00000030                           : iostream.obj (.const:_ZTVSi)
                  40300c24    00000030                           : iostream.obj (.const:_ZTVSo)
                  40300c54    00000030                           : wiostrea.obj (.const:_ZTVSt13basic_istreamIwSt11char_traitsIwEE)
                  40300c84    00000030                           : wiostrea.obj (.const:_ZTVSt13basic_ostreamIwSt11char_traitsIwEE)
                  40300cb4    00000030     SimpleClass.obj (.const:_ZTVSt5ctypeIcE)
                  40300ce4    00000030     SimpleClass.obj (.const:_ZTVSt7num_putIcSt19ostreambuf_iteratorIcSt11char_traitsIcEEE)
                  40300d14    00000030     rtsv7A8_A_le_eabi.lib : wlocale.obj (.const:_ZTVSt7num_putIwSt19ostreambuf_iteratorIwSt11char_traitsIwEEE)
                  40300d44    00000030                           : strftime.obj (.const:fmon)
                  40300d74    0000002c                           : iostream.obj (.const:_ZTVSt7codecvtIcciE)
                  40300da0    0000002c                           : wiostrea.obj (.const:_ZTVSt7codecvtIwciE)
                  40300dcc    00000029                           : iostream.obj (.const:.typeinfo:_ZTSSt15basic_streambufIcSt11char_traitsIcEE)
                  40300df5    00000029                           : wiostrea.obj (.const:.typeinfo:_ZTSSt15basic_streambufIwSt11char_traitsIwEE)
                  40300e1e    00000028                           : typeinfo_.obj (.const:.typeinfo:_ZTSN10__cxxabiv123__fundamental_type_infoE)
                  40300e46    00000002     SimpleClass.obj (.const:.string:_ZZNKSt7num_putIcSt19ostreambuf_iteratorIcSt11char_traitsIcEEE5_FputES3_RSt8ios_basecPKcjjjjEs)
                  40300e48    00000028     rtsv7A8_A_le_eabi.lib : xlocale.obj (.const:_ZTVSt8time_getIcSt19istreambuf_iteratorIcSt11char_traitsIcEEE)
                  40300e70    00000028                           : wlocale.obj (.const:_ZTVSt8time_getIwSt19istreambuf_iteratorIwSt11char_traitsIwEEE)
                  40300e98    00000027                           : iostream.obj (.const:.typeinfo:_ZTSSt13basic_filebufIcSt11char_traitsIcEE)
                  40300ebf    00000027                           : wiostrea.obj (.const:.typeinfo:_ZTSSt13basic_filebufIwSt11char_traitsIwEE)
                  40300ee6    00000027                           : wiostrea.obj (.const:.typeinfo:_ZTSSt13basic_istreamIwSt11char_traitsIwEE)
                  40300f0d    00000027                           : wiostrea.obj (.const:.typeinfo:_ZTSSt13basic_ostreamIwSt11char_traitsIwEE)
                  40300f34    00000026                           : typeinfo_.obj (.const:.typeinfo:_ZTSN10__cxxabiv121__vmi_class_type_infoE)
                  40300f5a    00000025                           : typeinfo_.obj (.const:.typeinfo:_ZTSN10__cxxabiv120__si_class_type_infoE)
                  40300f7f    00000024                           : typeinfo_.obj (.const:.typeinfo:_ZTSN10__cxxabiv119__pointer_type_infoE)
                  40300fa3    00000001                           : wlocale.obj (.const:.string:_ZZNSt7_MpunctIwE5_InitERKSt8_LocinfoEs)
                  40300fa4    00000024     SimpleClass.obj (.const:_ZTVSt8numpunctIcE)
                  40300fc8    00000024     rtsv7A8_A_le_eabi.lib : wlocale.obj (.const:_ZTVSt8numpunctIwE)
                  40300fec    00000022                           : typeinfo_.obj (.const:.typeinfo:_ZTSN10__cxxabiv117__class_type_infoE)
                  4030100e    00000022                           : typeinfo_.obj (.const:.typeinfo:_ZTSN10__cxxabiv117__pbase_type_infoE)
                  40301030    00000022                           : iostream.obj (.const:.typeinfo:_ZTSSt9basic_iosIcSt11char_traitsIcEE)
                  40301052    00000022                           : wiostrea.obj (.const:.typeinfo:_ZTSSt9basic_iosIwSt11char_traitsIwEE)
                  40301074    0000001c                           : iostream.obj (.const:_ZTVSt12codecvt_base)
                  40301090    0000001c                           : xlocale.obj (.const:_ZTVSt7collateIcE)
                  403010ac    0000001c                           : wlocale.obj (.const:_ZTVSt7collateIwE)
                  403010c8    0000001c                           : xlocale.obj (.const:_ZTVSt8messagesIcE)
                  403010e4    0000001c                           : wlocale.obj (.const:_ZTVSt8messagesIwE)
                  40301100    0000001c                           : strftime.obj (.const)
                  4030111c    00000018                           : iostream.obj (.const:.typeinfo:_ZTISi)
                  40301134    00000018                           : iostream.obj (.const:.typeinfo:_ZTISo)
                  4030114c    00000018                           : wiostrea.obj (.const:.typeinfo:_ZTISt13basic_istreamIwSt11char_traitsIwEE)
                  40301164    00000018                           : wiostrea.obj (.const:.typeinfo:_ZTISt13basic_ostreamIwSt11char_traitsIwEE)
                  4030117c    00000018                           : ios.obj (.const:_ZTVNSt8ios_base7failureE)
                  40301194    00000018                           : string.obj (.const:_ZTVSt11logic_error)
                  403011ac    00000018                           : string.obj (.const:_ZTVSt12length_error)
                  403011c4    00000018                           : string.obj (.const:_ZTVSt12out_of_range)
                  403011dc    00000018                           : ios.obj (.const:_ZTVSt13runtime_error)
                  403011f4    00000018                           : locale.obj (.const:_ZTVSt9bad_alloc)
                  4030120c    00000018                           : ios.obj (.const:_ZTVSt9exception)
                  40301224    00000018                           : xlocale.obj (.const:_ZTVSt9money_getIcSt19istreambuf_iteratorIcSt11char_traitsIcEEE)
                  4030123c    00000018                           : wlocale.obj (.const:_ZTVSt9money_getIwSt19istreambuf_iteratorIwSt11char_traitsIwEEE)
                  40301254    00000018                           : xlocale.obj (.const:_ZTVSt9money_putIcSt19ostreambuf_iteratorIcSt11char_traitsIcEEE)
                  4030126c    00000018                           : wlocale.obj (.const:_ZTVSt9money_putIwSt19ostreambuf_iteratorIwSt11char_traitsIwEEE)
                  40301284    00000017                           : locale.obj (.const:.string:_ZZNKSt7num_getIcSt19istreambuf_iteratorIcSt11char_traitsIcEEE8_GetifldEPcRS3_S6_NSt5_IosbIiE9_FmtflagsERKSt6localeEs)
                  4030129b    00000017                           : wlocale.obj (.const:.string:_ZZNKSt7num_getIwSt19istreambuf_iteratorIwSt11char_traitsIwEEE8_GetifldEPcRS3_S6_NSt5_IosbIiE9_FmtflagsERKSt6localeEs)
                  403012b2    00000016                           : ios.obj (.const:.typeinfo:_ZTSNSt8ios_base7failureE)
                  403012c8    00000016                           : xlocale.obj (.const:.typeinfo:_ZTSSt10moneypunctIcLb0EE)
                  403012de    00000016                           : xlocale.obj (.const:.typeinfo:_ZTSSt10moneypunctIcLb1EE)
                  403012f4    00000016                           : wlocale.obj (.const:.typeinfo:_ZTSSt10moneypunctIwLb0EE)
                  4030130a    00000016                           : wlocale.obj (.const:.typeinfo:_ZTSSt10moneypunctIwLb1EE)
                  40301320    00000014                           : locale0.obj (.const:.typeinfo:_ZTSNSt6locale7_LocimpE)
                  40301334    00000014                           : xlocale.obj (.const:_ZTVSt8time_putIcSt19ostreambuf_iteratorIcSt11char_traitsIcEEE)
                  40301348    00000014                           : wlocale.obj (.const:_ZTVSt8time_putIwSt19ostreambuf_iteratorIwSt11char_traitsIwEEE)
                  4030135c    00000012     SimpleClass.obj (.const:.typeinfo:_ZTSNSt6locale5facetE)
                  4030136e    00000012     rtsv7A8_A_le_eabi.lib : wlocale.obj (.const:.typeinfo:_ZTSSt13messages_base)
                  40301380    00000012                           : ios.obj (.const:.typeinfo:_ZTSSt13runtime_error)
                  40301392    00000011                           : iostream.obj (.const:.typeinfo:_ZTSSt12codecvt_base)
                  403013a3    00000011                           : string.obj (.const:.typeinfo:_ZTSSt12length_error)
                  403013b4    00000011                           : string.obj (.const:.typeinfo:_ZTSSt12out_of_range)
                  403013c5    00000003     SimpleClass.obj (.const:.string:_ZZNKSt7num_putIcSt19ostreambuf_iteratorIcSt11char_traitsIcEEE6do_putES3_RSt8ios_basecPKvEs)
                  403013c8    00000010     rtsv7A8_A_le_eabi.lib : typeinfo_.obj (.const:.typeinfo:_ZTIPKe)
                  403013d8    00000010                           : string.obj (.const:.typeinfo:_ZTSSt11logic_error)
                  403013e8    00000010                           : iostream.obj (.const:.typeinfo:_ZTSSt7codecvtIcciE)
                  403013f8    00000010                           : wiostrea.obj (.const:.typeinfo:_ZTSSt7codecvtIwciE)
                  40301408    00000010                           : typeinfo_.obj (.const:_ZTVN10__cxxabiv117__class_type_infoE)
                  40301418    00000010                           : typeinfo_.obj (.const:_ZTVN10__cxxabiv119__pointer_type_infoE)
                  40301428    00000010                           : typeinfo_.obj (.const:_ZTVN10__cxxabiv120__si_class_type_infoE)
                  40301438    00000010                           : typeinfo_.obj (.const:_ZTVN10__cxxabiv121__vmi_class_type_infoE)
                  40301448    00000010                           : typeinfo_.obj (.const:_ZTVN10__cxxabiv123__fundamental_type_infoE)
                  40301458    00000010     SimpleClass.obj (.const:_ZTVNSt6locale5facetE)
                  40301468    00000010     rtsv7A8_A_le_eabi.lib : locale0.obj (.const:_ZTVNSt6locale7_LocimpE)
                  40301478    00000010     SimpleClass.obj (.const:_ZTVSt10ctype_base)
                  40301488    00000010     rtsv7A8_A_le_eabi.lib : wlocale.obj (.const:_ZTVSt10money_base)
                  40301498    00000010                           : wlocale.obj (.const:_ZTVSt13messages_base)
                  403014a8    00000010                           : ios.obj (.const:_ZTVSt8ios_base)
                  403014b8    00000010                           : iostream.obj (.const:_ZTVSt9basic_iosIcSt11char_traitsIcEE)
                  403014c8    00000010                           : wiostrea.obj (.const:_ZTVSt9basic_iosIwSt11char_traitsIwEE)
                  403014d8    00000010                           : wlocale.obj (.const:_ZTVSt9time_base)
                  403014e8    0000000f     SimpleClass.obj (.const:.typeinfo:_ZTSSt10ctype_base)
                  403014f7    0000000f     rtsv7A8_A_le_eabi.lib : wlocale.obj (.const:.typeinfo:_ZTSSt10money_base)
                  40301506    0000000f                           : xlocale.obj (.const:.typeinfo:_ZTSSt8messagesIcE)
                  40301515    0000000f                           : wlocale.obj (.const:.typeinfo:_ZTSSt8messagesIwE)
                  40301524    0000000f     SimpleClass.obj (.const:.typeinfo:_ZTSSt8numpunctIcE)
                  40301533    0000000f     rtsv7A8_A_le_eabi.lib : wlocale.obj (.const:.typeinfo:_ZTSSt8numpunctIwE)
                  40301542    0000000e                           : xlocale.obj (.const:.typeinfo:_ZTSSt7_MpunctIcE)
                  40301550    0000000e                           : wlocale.obj (.const:.typeinfo:_ZTSSt7_MpunctIwE)
                  4030155e    0000000e                           : xlocale.obj (.const:.typeinfo:_ZTSSt7collateIcE)
                  4030156c    0000000e                           : wlocale.obj (.const:.typeinfo:_ZTSSt7collateIwE)
                  4030157a    0000000d                           : locale.obj (.const:.typeinfo:_ZTSSt9bad_alloc)
                  40301587    0000000d                           : ios.obj (.const:.typeinfo:_ZTSSt9exception)
                  40301594    0000000d                           : wlocale.obj (.const:.typeinfo:_ZTSSt9time_base)
                  403015a1    0000000d                           : typeinfo_.obj (.const:.typeinfo:_ZTSSt9type_info)
                  403015ae    00000002     SimpleClass.obj (.const:.string:_ZZNKSt7num_putIcSt19ostreambuf_iteratorIcSt11char_traitsIcEEE5_FputES3_RSt8ios_basecPKcjjjjEs_0)
                  403015b0    0000000c     rtsv7A8_A_le_eabi.lib : typeinfo_.obj (.const:.typeinfo:_ZTIN10__cxxabiv117__class_type_infoE)
                  403015bc    0000000c                           : typeinfo_.obj (.const:.typeinfo:_ZTIN10__cxxabiv117__pbase_type_infoE)
                  403015c8    0000000c                           : typeinfo_.obj (.const:.typeinfo:_ZTIN10__cxxabiv119__pointer_type_infoE)
                  403015d4    0000000c                           : typeinfo_.obj (.const:.typeinfo:_ZTIN10__cxxabiv120__si_class_type_infoE)
                  403015e0    0000000c                           : typeinfo_.obj (.const:.typeinfo:_ZTIN10__cxxabiv121__vmi_class_type_infoE)
                  403015ec    0000000c                           : typeinfo_.obj (.const:.typeinfo:_ZTIN10__cxxabiv123__fundamental_type_infoE)
                  403015f8    0000000c                           : locale0.obj (.const:.typeinfo:_ZTINSt6locale7_LocimpE)
                  40301604    0000000c                           : ios.obj (.const:.typeinfo:_ZTINSt8ios_base7failureE)
                  40301610    0000000c     SimpleClass.obj (.const:.typeinfo:_ZTISt10ctype_base)
                  4030161c    0000000c     rtsv7A8_A_le_eabi.lib : wlocale.obj (.const:.typeinfo:_ZTISt10money_base)
                  40301628    0000000c                           : xlocale.obj (.const:.typeinfo:_ZTISt10moneypunctIcLb0EE)
                  40301634    0000000c                           : xlocale.obj (.const:.typeinfo:_ZTISt10moneypunctIcLb1EE)
                  40301640    0000000c                           : wlocale.obj (.const:.typeinfo:_ZTISt10moneypunctIwLb0EE)
                  4030164c    0000000c                           : wlocale.obj (.const:.typeinfo:_ZTISt10moneypunctIwLb1EE)
                  40301658    0000000c                           : string.obj (.const:.typeinfo:_ZTISt11logic_error)
                  40301664    0000000c                           : iostream.obj (.const:.typeinfo:_ZTISt12codecvt_base)
                  40301670    0000000c                           : string.obj (.const:.typeinfo:_ZTISt12length_error)
                  4030167c    0000000c                           : string.obj (.const:.typeinfo:_ZTISt12out_of_range)
                  40301688    0000000c                           : iostream.obj (.const:.typeinfo:_ZTISt13basic_filebufIcSt11char_traitsIcEE)
                  40301694    0000000c                           : wiostrea.obj (.const:.typeinfo:_ZTISt13basic_filebufIwSt11char_traitsIwEE)
                  403016a0    0000000c                           : wlocale.obj (.const:.typeinfo:_ZTISt13messages_base)
                  403016ac    0000000c                           : ios.obj (.const:.typeinfo:_ZTISt13runtime_error)
                  403016b8    0000000c     SimpleClass.obj (.const:.typeinfo:_ZTISt5ctypeIcE)
                  403016c4    0000000c     rtsv7A8_A_le_eabi.lib : wiostrea.obj (.const:.typeinfo:_ZTISt5ctypeIwE)
                  403016d0    0000000c                           : xlocale.obj (.const:.typeinfo:_ZTISt7_MpunctIcE)
                  403016dc    0000000c                           : wlocale.obj (.const:.typeinfo:_ZTISt7_MpunctIwE)
                  403016e8    0000000c                           : iostream.obj (.const:.typeinfo:_ZTISt7codecvtIcciE)
                  403016f4    0000000c                           : wiostrea.obj (.const:.typeinfo:_ZTISt7codecvtIwciE)
                  40301700    0000000c                           : xlocale.obj (.const:.typeinfo:_ZTISt7collateIcE)
                  4030170c    0000000c                           : wlocale.obj (.const:.typeinfo:_ZTISt7collateIwE)
                  40301718    0000000c                           : locale.obj (.const:.typeinfo:_ZTISt7num_getIcSt19istreambuf_iteratorIcSt11char_traitsIcEEE)
                  40301724    0000000c                           : wlocale.obj (.const:.typeinfo:_ZTISt7num_getIwSt19istreambuf_iteratorIwSt11char_traitsIwEEE)
                  40301730    0000000c     SimpleClass.obj (.const:.typeinfo:_ZTISt7num_putIcSt19ostreambuf_iteratorIcSt11char_traitsIcEEE)
                  4030173c    0000000c     rtsv7A8_A_le_eabi.lib : wlocale.obj (.const:.typeinfo:_ZTISt7num_putIwSt19ostreambuf_iteratorIwSt11char_traitsIwEEE)
                  40301748    0000000c                           : ios.obj (.const:.typeinfo:_ZTISt8ios_base)
                  40301754    0000000c                           : xlocale.obj (.const:.typeinfo:_ZTISt8messagesIcE)
                  40301760    0000000c                           : wlocale.obj (.const:.typeinfo:_ZTISt8messagesIwE)
                  4030176c    0000000c     SimpleClass.obj (.const:.typeinfo:_ZTISt8numpunctIcE)
                  40301778    0000000c     rtsv7A8_A_le_eabi.lib : wlocale.obj (.const:.typeinfo:_ZTISt8numpunctIwE)
                  40301784    0000000c                           : xlocale.obj (.const:.typeinfo:_ZTISt8time_getIcSt19istreambuf_iteratorIcSt11char_traitsIcEEE)
                  40301790    0000000c                           : wlocale.obj (.const:.typeinfo:_ZTISt8time_getIwSt19istreambuf_iteratorIwSt11char_traitsIwEEE)
                  4030179c    0000000c                           : xlocale.obj (.const:.typeinfo:_ZTISt8time_putIcSt19ostreambuf_iteratorIcSt11char_traitsIcEEE)
                  403017a8    0000000c                           : wlocale.obj (.const:.typeinfo:_ZTISt8time_putIwSt19ostreambuf_iteratorIwSt11char_traitsIwEEE)
                  403017b4    0000000c                           : locale.obj (.const:.typeinfo:_ZTISt9bad_alloc)
                  403017c0    0000000c                           : iostream.obj (.const:.typeinfo:_ZTISt9basic_iosIcSt11char_traitsIcEE)
                  403017cc    0000000c                           : wiostrea.obj (.const:.typeinfo:_ZTISt9basic_iosIwSt11char_traitsIwEE)
                  403017d8    0000000c                           : xlocale.obj (.const:.typeinfo:_ZTISt9money_getIcSt19istreambuf_iteratorIcSt11char_traitsIcEEE)
                  403017e4    0000000c                           : wlocale.obj (.const:.typeinfo:_ZTISt9money_getIwSt19istreambuf_iteratorIwSt11char_traitsIwEEE)
                  403017f0    0000000c                           : xlocale.obj (.const:.typeinfo:_ZTISt9money_putIcSt19ostreambuf_iteratorIcSt11char_traitsIcEEE)
                  403017fc    0000000c                           : wlocale.obj (.const:.typeinfo:_ZTISt9money_putIwSt19ostreambuf_iteratorIwSt11char_traitsIwEEE)
                  40301808    0000000c                           : wlocale.obj (.const:.typeinfo:_ZTISt9time_base)
                  40301814    0000000c                           : ios.obj (.const:.typeinfo:_ZTSSt5_IosbIiE)
                  40301820    0000000c     SimpleClass.obj (.const:.typeinfo:_ZTSSt5ctypeIcE)
                  4030182c    0000000c     rtsv7A8_A_le_eabi.lib : wiostrea.obj (.const:.typeinfo:_ZTSSt5ctypeIwE)
                  40301838    0000000c                           : ios.obj (.const:.typeinfo:_ZTSSt8ios_base)
                  40301844    00000009     SimpleClass.obj (.const)
                  4030184d    00000003     SimpleClass.obj (.const:.string:_ZZNKSt7num_putIcSt19ostreambuf_iteratorIcSt11char_traitsIcEEE6do_putES3_RSt8ios_baseclEs)
                  40301850    00000008     rtsv7A8_A_le_eabi.lib : setlocale.obj (.const:.string)
                  40301858    00000008     SimpleClass.obj (.const:.typeinfo:_ZTINSt6locale5facetE)
                  40301860    00000008     rtsv7A8_A_le_eabi.lib : iostream.obj (.const:.typeinfo:_ZTISt15basic_streambufIcSt11char_traitsIcEE)
                  40301868    00000008                           : wiostrea.obj (.const:.typeinfo:_ZTISt15basic_streambufIwSt11char_traitsIwEE)
                  40301870    00000008                           : ios.obj (.const:.typeinfo:_ZTISt5_IosbIiE)
                  40301878    00000008                           : ios.obj (.const:.typeinfo:_ZTISt9exception)
                  40301880    00000008                           : typeinfo_.obj (.const:.typeinfo:_ZTISt9type_info)
                  40301888    00000008                           : typeinfo_.obj (.const:.typeinfo:_ZTIe)
                  40301890    00000006     SimpleClass.obj (.const:.string:_ZZNKSt8_Locinfo9_GetfalseEvEs)
                  40301896    00000006     rtsv7A8_A_le_eabi.lib : xlocale.obj (.const:.string:_ZZNKSt9money_putIcSt19ostreambuf_iteratorIcSt11char_traitsIcEEE6do_putES3_bRSt8ios_baseceEs)
                  4030189c    00000006                           : wlocale.obj (.const:.string:_ZZNKSt9money_putIwSt19ostreambuf_iteratorIwSt11char_traitsIwEEE6do_putES3_bRSt8ios_baseweEs)
                  403018a2    00000005                           : xlocale.obj (.const:.string:_ZZNSt7_MpunctIcE7_MakpatERNSt10money_base7patternEjjjEs)
                  403018a7    00000005                           : wlocale.obj (.const:.string:_ZZNSt7_MpunctIwE7_MakpatERNSt10money_base7patternEjjjEs)
                  403018ac    00000005                           : wlocale.obj (.const:.string)
                  403018b1    00000005                           : xlocale.obj (.const:.string)
                  403018b6    00000004                           : typeinfo_.obj (.const:.typeinfo:_ZTSPKe)
                  403018ba    00000002                           : wlocale.obj (.const:.string:_ZZNKSt7num_putIwSt19ostreambuf_iteratorIwSt11char_traitsIwEEE5_FputES3_RSt8ios_basewPKcjjjjEs)
                  403018bc    00000004                           : ios.obj (.const)
                  403018c0    00000003     SimpleClass.obj (.const:.string:_ZZNKSt7num_putIcSt19ostreambuf_iteratorIcSt11char_traitsIcEEE6do_putES3_RSt8ios_basecmEs)
                  403018c3    00000003     SimpleClass.obj (.const:.string:_ZZNKSt7num_putIcSt19ostreambuf_iteratorIcSt11char_traitsIcEEE6do_putES3_RSt8ios_basecxEs)
                  403018c6    00000003     SimpleClass.obj (.const:.string:_ZZNKSt7num_putIcSt19ostreambuf_iteratorIcSt11char_traitsIcEEE6do_putES3_RSt8ios_basecyEs)
                  403018c9    00000003     rtsv7A8_A_le_eabi.lib : wlocale.obj (.const:.string:_ZZNKSt7num_putIwSt19ostreambuf_iteratorIwSt11char_traitsIwEEE6do_putES3_RSt8ios_basewPKvEs)
                  403018cc    00000003                           : wlocale.obj (.const:.string:_ZZNKSt7num_putIwSt19ostreambuf_iteratorIwSt11char_traitsIwEEE6do_putES3_RSt8ios_basewlEs)
                  403018cf    00000003                           : wlocale.obj (.const:.string:_ZZNKSt7num_putIwSt19ostreambuf_iteratorIwSt11char_traitsIwEEE6do_putES3_RSt8ios_basewmEs)
                  403018d2    00000003                           : wlocale.obj (.const:.string:_ZZNKSt7num_putIwSt19ostreambuf_iteratorIwSt11char_traitsIwEEE6do_putES3_RSt8ios_basewxEs)
                  403018d5    00000003                           : wlocale.obj (.const:.string:_ZZNKSt7num_putIwSt19ostreambuf_iteratorIwSt11char_traitsIwEEE6do_putES3_RSt8ios_basewyEs)
                  403018d8    00000003                           : iostream.obj (.const:.typeinfo:_ZTSSi)
                  403018db    00000003                           : iostream.obj (.const:.typeinfo:_ZTSSo)
                  403018de    00000002                           : wlocale.obj (.const:.string:_ZZNKSt7num_putIwSt19ostreambuf_iteratorIwSt11char_traitsIwEEE5_FputES3_RSt8ios_basewPKcjjjjEs_0)
                  403018e0    00000002                           : xlocale.obj (.const:.string:_ZZNSt7_MpunctIcE5_InitERKSt8_LocinfoEs_0)
                  403018e2    00000002                           : wlocale.obj (.const:.string:_ZZNSt7_MpunctIwE5_InitERKSt8_LocinfoEs_0)
                  403018e4    00000002                           : typeinfo_.obj (.const:.typeinfo:_ZTSe)

.stack     0    403018e8    00000800     UNINITIALIZED
                  403018e8    00000800     --HOLE--

.sysmem    0    403020e8    00000800     UNINITIALIZED
                  403020e8    00000008     rtsv7A8_A_le_eabi.lib : memory.obj (.sysmem)
                  403020f0    000007f8     --HOLE--

.data      0    403028e8    000007cc     UNINITIALIZED
                  403028e8    000001b8     rtsv7A8_A_le_eabi.lib : iostream.obj (.data)
                  40302aa0    000001b8                           : wiostrea.obj (.data)
                  40302c58    000000f0                           : defs.obj (.data:_ftable)
                  40302d48    000000d0                           : lowlev.obj (.data)
                  40302e18    000000b0                           : signal.obj (.data:sigtable)
                  40302ec8    00000080                           : xvalues.obj (.data)
                  40302f48    00000054                           : ios.obj (.data)
                  40302f9c    00000034                           : setlocale.obj (.data:C_locale)
                  40302fd0    00000020                           : locale0.obj (.data)
                  40302ff0    00000010                           : defs.obj (.data)
                  40303000    00000010                           : tmzone.obj (.data)
                  40303010    0000000c                           : memory.obj (.data)
                  4030301c    00000008                           : _lock.obj (.data)
                  40303024    00000008                           : exit.obj (.data)
                  4030302c    00000008                           : feraiseexcept.obj (.data)
                  40303034    00000004                           : xlocale.obj (.data:_ZNSt9_FacetptrISt10moneypunctIcLb0EEE6_PsaveE)
                  40303038    00000004                           : xlocale.obj (.data:_ZNSt9_FacetptrISt10moneypunctIcLb1EEE6_PsaveE)
                  4030303c    00000004                           : wlocale.obj (.data:_ZNSt9_FacetptrISt10moneypunctIwLb0EEE6_PsaveE)
                  40303040    00000004                           : wlocale.obj (.data:_ZNSt9_FacetptrISt10moneypunctIwLb1EEE6_PsaveE)
                  40303044    00000004     SimpleClass.obj (.data:_ZNSt9_FacetptrISt5ctypeIcEE6_PsaveE)
                  40303048    00000004     rtsv7A8_A_le_eabi.lib : wiostrea.obj (.data:_ZNSt9_FacetptrISt5ctypeIwEE6_PsaveE)
                  4030304c    00000004                           : iostream.obj (.data:_ZNSt9_FacetptrISt7codecvtIcciEE6_PsaveE)
                  40303050    00000004                           : wiostrea.obj (.data:_ZNSt9_FacetptrISt7codecvtIwciEE6_PsaveE)
                  40303054    00000004                           : xlocale.obj (.data:_ZNSt9_FacetptrISt7collateIcEE6_PsaveE)
                  40303058    00000004                           : wlocale.obj (.data:_ZNSt9_FacetptrISt7collateIwEE6_PsaveE)
                  4030305c    00000004                           : locale.obj (.data:_ZNSt9_FacetptrISt7num_getIcSt19istreambuf_iteratorIcSt11char_traitsIcEEEE6_PsaveE)
                  40303060    00000004                           : wlocale.obj (.data:_ZNSt9_FacetptrISt7num_getIwSt19istreambuf_iteratorIwSt11char_traitsIwEEEE6_PsaveE)
                  40303064    00000004     SimpleClass.obj (.data:_ZNSt9_FacetptrISt7num_putIcSt19ostreambuf_iteratorIcSt11char_traitsIcEEEE6_PsaveE)
                  40303068    00000004     rtsv7A8_A_le_eabi.lib : wlocale.obj (.data:_ZNSt9_FacetptrISt7num_putIwSt19ostreambuf_iteratorIwSt11char_traitsIwEEEE6_PsaveE)
                  4030306c    00000004                           : xlocale.obj (.data:_ZNSt9_FacetptrISt8messagesIcEE6_PsaveE)
                  40303070    00000004                           : wlocale.obj (.data:_ZNSt9_FacetptrISt8messagesIwEE6_PsaveE)
                  40303074    00000004     SimpleClass.obj (.data:_ZNSt9_FacetptrISt8numpunctIcEE6_PsaveE)
                  40303078    00000004     rtsv7A8_A_le_eabi.lib : wlocale.obj (.data:_ZNSt9_FacetptrISt8numpunctIwEE6_PsaveE)
                  4030307c    00000004                           : xlocale.obj (.data:_ZNSt9_FacetptrISt8time_getIcSt19istreambuf_iteratorIcSt11char_traitsIcEEEE6_PsaveE)
                  40303080    00000004                           : wlocale.obj (.data:_ZNSt9_FacetptrISt8time_getIwSt19istreambuf_iteratorIwSt11char_traitsIwEEEE6_PsaveE)
                  40303084    00000004                           : xlocale.obj (.data:_ZNSt9_FacetptrISt8time_putIcSt19ostreambuf_iteratorIcSt11char_traitsIcEEEE6_PsaveE)
                  40303088    00000004                           : wlocale.obj (.data:_ZNSt9_FacetptrISt8time_putIwSt19ostreambuf_iteratorIwSt11char_traitsIwEEEE6_PsaveE)
                  4030308c    00000004                           : xlocale.obj (.data:_ZNSt9_FacetptrISt9money_getIcSt19istreambuf_iteratorIcSt11char_traitsIcEEEE6_PsaveE)
                  40303090    00000004                           : wlocale.obj (.data:_ZNSt9_FacetptrISt9money_getIwSt19istreambuf_iteratorIwSt11char_traitsIwEEEE6_PsaveE)
                  40303094    00000004                           : xlocale.obj (.data:_ZNSt9_FacetptrISt9money_putIcSt19ostreambuf_iteratorIcSt11char_traitsIcEEEE6_PsaveE)
                  40303098    00000004                           : wlocale.obj (.data:_ZNSt9_FacetptrISt9money_putIwSt19ostreambuf_iteratorIwSt11char_traitsIwEEEE6_PsaveE)
                  4030309c    00000004                           : dtor_list.obj (.data)
                  403030a0    00000004                           : errno.obj (.data)
                  403030a4    00000004                           : fopen.obj (.data)
                  403030a8    00000004                           : raisehan.obj (.data)
                  403030ac    00000004                           : stkdepth_vars.obj (.data)
                  403030b0    00000004                           : vars.obj (.data)

.bss       0    403030b4    000002bc     UNINITIALIZED
                  403030b4    00000120     rtsv7A8_A_le_eabi.lib : trgmsg.obj (.bss:__CIOBUF_)
                  403031d4    000000a0                           : defs.obj (.bss:__TI_tmpnams)
                  40303274    0000000c     (.common:tstr_out)
                  40303280    00000008                           : locale.obj (.bss)
                  40303288    00000008     (.common:_ZZNSt6locale7_Locimp7_AddfacEPNS_5facetEjE5nomem)
                  40303290    00000008     (.common:_ZZNSt6locale7_LocimpC1ERKS0_E5nomem)
                  40303298    00000008     (.common:parmbuf)
                  403032a0    00000004                           : xlocale.obj (.bss:_ZGVNSt10moneypunctIcLb0EE2idE)
                  403032a4    00000004                           : xlocale.obj (.bss:_ZGVNSt10moneypunctIcLb1EE2idE)
                  403032a8    00000004                           : wlocale.obj (.bss:_ZGVNSt10moneypunctIwLb0EE2idE)
                  403032ac    00000004                           : wlocale.obj (.bss:_ZGVNSt10moneypunctIwLb1EE2idE)
                  403032b0    00000004                           : iostream.obj (.bss:_ZGVNSt7codecvtIcciE2idE)
                  403032b4    00000004                           : xlocale.obj (.bss:_ZGVNSt7collateIcE2idE)
                  403032b8    00000004                           : wlocale.obj (.bss:_ZGVNSt7collateIwE2idE)
                  403032bc    00000004                           : locale.obj (.bss:_ZGVNSt7num_getIcSt19istreambuf_iteratorIcSt11char_traitsIcEEE2idE)
                  403032c0    00000004                           : wlocale.obj (.bss:_ZGVNSt7num_getIwSt19istreambuf_iteratorIwSt11char_traitsIwEEE2idE)
                  403032c4    00000004     SimpleClass.obj (.bss:_ZGVNSt7num_putIcSt19ostreambuf_iteratorIcSt11char_traitsIcEEE2idE)
                  403032c8    00000004     rtsv7A8_A_le_eabi.lib : wlocale.obj (.bss:_ZGVNSt7num_putIwSt19ostreambuf_iteratorIwSt11char_traitsIwEEE2idE)
                  403032cc    00000004                           : xlocale.obj (.bss:_ZGVNSt8messagesIcE2idE)
                  403032d0    00000004                           : wlocale.obj (.bss:_ZGVNSt8messagesIwE2idE)
                  403032d4    00000004     SimpleClass.obj (.bss:_ZGVNSt8numpunctIcE2idE)
                  403032d8    00000004     rtsv7A8_A_le_eabi.lib : wlocale.obj (.bss:_ZGVNSt8numpunctIwE2idE)
                  403032dc    00000004                           : xlocale.obj (.bss:_ZGVNSt8time_getIcSt19istreambuf_iteratorIcSt11char_traitsIcEEE2idE)
                  403032e0    00000004                           : wlocale.obj (.bss:_ZGVNSt8time_getIwSt19istreambuf_iteratorIwSt11char_traitsIwEEE2idE)
                  403032e4    00000004                           : xlocale.obj (.bss:_ZGVNSt8time_putIcSt19ostreambuf_iteratorIcSt11char_traitsIcEEE2idE)
                  403032e8    00000004                           : xlocale.obj (.bss:_ZGVNSt9money_getIcSt19istreambuf_iteratorIcSt11char_traitsIcEEE2idE)
                  403032ec    00000004                           : wlocale.obj (.bss:_ZGVNSt9money_getIwSt19istreambuf_iteratorIwSt11char_traitsIwEEE2idE)
                  403032f0    00000004                           : xlocale.obj (.bss:_ZGVNSt9money_putIcSt19ostreambuf_iteratorIcSt11char_traitsIcEEE2idE)
                  403032f4    00000004                           : wlocale.obj (.bss:_ZGVNSt9money_putIwSt19ostreambuf_iteratorIwSt11char_traitsIwEEE2idE)
                  403032f8    00000004                           : xlocale.obj (.bss:_ZNSt10moneypunctIcLb0EE2idE)
                  403032fc    00000004                           : xlocale.obj (.bss:_ZNSt10moneypunctIcLb1EE2idE)
                  40303300    00000004                           : wlocale.obj (.bss:_ZNSt10moneypunctIwLb0EE2idE)
                  40303304    00000004                           : wlocale.obj (.bss:_ZNSt10moneypunctIwLb1EE2idE)
                  40303308    00000004                           : iostream.obj (.bss:_ZNSt13basic_filebufIcSt11char_traitsIcEE7_StinitE)
                  4030330c    00000004                           : wiostrea.obj (.bss:_ZNSt13basic_filebufIwSt11char_traitsIwEE7_StinitE)
                  40303310    00000004                           : iostream.obj (.bss:_ZNSt4fposIiE4_StzE)
                  40303314    00000004                           : iostream.obj (.bss:_ZNSt7codecvtIcciE2idE)
                  40303318    00000004                           : xlocale.obj (.bss:_ZNSt7collateIcE2idE)
                  4030331c    00000004                           : wlocale.obj (.bss:_ZNSt7collateIwE2idE)
                  40303320    00000004                           : locale.obj (.bss:_ZNSt7num_getIcSt19istreambuf_iteratorIcSt11char_traitsIcEEE2idE)
                  40303324    00000004                           : wlocale.obj (.bss:_ZNSt7num_getIwSt19istreambuf_iteratorIwSt11char_traitsIwEEE2idE)
                  40303328    00000004     SimpleClass.obj (.bss:_ZNSt7num_putIcSt19ostreambuf_iteratorIcSt11char_traitsIcEEE2idE)
                  4030332c    00000004     rtsv7A8_A_le_eabi.lib : wlocale.obj (.bss:_ZNSt7num_putIwSt19ostreambuf_iteratorIwSt11char_traitsIwEEE2idE)
                  40303330    00000004                           : xlocale.obj (.bss:_ZNSt8messagesIcE2idE)
                  40303334    00000004                           : wlocale.obj (.bss:_ZNSt8messagesIwE2idE)
                  40303338    00000004     SimpleClass.obj (.bss:_ZNSt8numpunctIcE2idE)
                  4030333c    00000004     rtsv7A8_A_le_eabi.lib : wlocale.obj (.bss:_ZNSt8numpunctIwE2idE)
                  40303340    00000004                           : xlocale.obj (.bss:_ZNSt8time_getIcSt19istreambuf_iteratorIcSt11char_traitsIcEEE2idE)
                  40303344    00000004                           : wlocale.obj (.bss:_ZNSt8time_getIwSt19istreambuf_iteratorIwSt11char_traitsIwEEE2idE)
                  40303348    00000004                           : xlocale.obj (.bss:_ZNSt8time_putIcSt19ostreambuf_iteratorIcSt11char_traitsIcEEE2idE)
                  4030334c    00000004                           : wlocale.obj (.bss:_ZNSt8time_putIwSt19ostreambuf_iteratorIwSt11char_traitsIwEEE2idE)
                  40303350    00000004                           : xlocale.obj (.bss:_ZNSt9money_getIcSt19istreambuf_iteratorIcSt11char_traitsIcEEE2idE)
                  40303354    00000004                           : wlocale.obj (.bss:_ZNSt9money_getIwSt19istreambuf_iteratorIwSt11char_traitsIwEEE2idE)
                  40303358    00000004                           : xlocale.obj (.bss:_ZNSt9money_putIcSt19ostreambuf_iteratorIcSt11char_traitsIcEEE2idE)
                  4030335c    00000004                           : wlocale.obj (.bss:_ZNSt9money_putIwSt19ostreambuf_iteratorIwSt11char_traitsIwEEE2idE)
                  40303360    00000004                           : wlocale.obj (.bss)
                  40303364    00000004     (.common:_ZSt16__dummy_typeinfo)
                  40303368    00000004     (.common:__dso_handle)
                  4030336c    00000002     SimpleClass.obj (.bss)
                  4030336e    00000002     rtsv7A8_A_le_eabi.lib : wiostrea.obj (.bss)

.text      0    80000000    00023e3c     
                  80000000    00001a70     rtsv7A8_A_le_eabi.lib : _printfi.obj (.text)
                  80001a70    000017b8                           : locale.obj (.text)
                  80003228    00000fe4                           : xlocale.obj (.text:_ZNKSt9money_getIcSt19istreambuf_iteratorIcSt11char_traitsIcEEE8_GetmfldERS3_S5_bRSt8ios_base)
                  8000420c    00000fd4                           : wlocale.obj (.text)
                  800051e0    00000fa8                           : wlocale.obj (.text:_ZNKSt9money_getIwSt19istreambuf_iteratorIwSt11char_traitsIwEEE8_GetmfldERS3_S5_bRSt8ios_base)
                  80006188    00000cb8                           : locale.obj (.text:_ZNKSt7num_getIcSt19istreambuf_iteratorIcSt11char_traitsIcEEE8_GetffldEPcRS3_S6_RKSt6locale)
                  80006e40    00000c04                           : wlocale.obj (.text:_ZNKSt9money_putIwSt19ostreambuf_iteratorIwSt11char_traitsIwEEE8_PutmfldES3_bRSt8ios_basewbSbIwS2_SaIwEE)
                  80007a44    00000b68                           : xlocale.obj (.text:_ZNKSt9money_putIcSt19ostreambuf_iteratorIcSt11char_traitsIcEEE8_PutmfldES3_bRSt8ios_basecbSs)
                  800085ac    00000a8c                           : xlocale.obj (.text)
                  80009038    000009bc                           : wlocale.obj (.text:_ZNKSt7num_getIwSt19istreambuf_iteratorIwSt11char_traitsIwEEE8_GetffldEPcRS3_S6_RKSt6locale)
                  800099f4    00000984                           : locale0.obj (.text)
                  8000a378    00000908                           : wlocale.obj (.text:_ZNKSt7num_putIwSt19ostreambuf_iteratorIwSt11char_traitsIwEEE5_FputES3_RSt8ios_basewPKcjjjj)
                  8000ac80    000008d8                           : ios.obj (.text)
                  8000b558    00000850                           : wiostrea.obj (.text)
                  8000bda8    00000720                           : locale.obj (.text:_ZNKSt7num_getIcSt19istreambuf_iteratorIcSt11char_traitsIcEEE8_GetifldEPcRS3_S6_NSt5_IosbIiE9_FmtflagsERKSt6locale)
                  8000c4c8    0000070c     SimpleClass.obj (.text:_ZNKSt7num_putIcSt19ostreambuf_iteratorIcSt11char_traitsIcEEE5_FputES3_RSt8ios_basecPKcjjjj)
                  8000cbd4    00000708     rtsv7A8_A_le_eabi.lib : wlocale.obj (.text:_ZNKSt8time_getIwSt19istreambuf_iteratorIwSt11char_traitsIwEEE11do_get_dateES3_S3_RSt8ios_baseRNSt5_IosbIiE8_IostateEPSt2tm)
                  8000d2dc    00000688                           : iostream.obj (.text)
                  8000d964    0000067c                           : xlocale.obj (.text:_ZNKSt8time_getIcSt19istreambuf_iteratorIcSt11char_traitsIcEEE11do_get_dateES3_S3_RSt8ios_baseRNSt5_IosbIiE8_IostateEPSt2tm)
                  8000dfe0    0000063c                           : memory.obj (.text)
                  8000e61c    00000620                           : wlocale.obj (.text:_ZNKSt7num_getIwSt19istreambuf_iteratorIwSt11char_traitsIwEEE8_GetifldEPcRS3_S6_NSt5_IosbIiE9_FmtflagsERKSt6locale)
                  8000ec3c    00000548                           : lowlev.obj (.text)
                  8000f184    00000518                           : strftime.obj (.text)
                  8000f69c    000004cc                           : trgdrv.obj (.text)
                  8000fb68    00000454                           : wlocale.obj (.text:_ZNKSt7num_getIwSt19istreambuf_iteratorIwSt11char_traitsIwEEE6do_getES3_S3_RSt8ios_baseRNSt5_IosbIiE8_IostateERb)
                  8000ffbc    000003e4                           : wlocale.obj (.text:_ZNKSt8time_getIwSt19istreambuf_iteratorIwSt11char_traitsIwEEE7_GetintERS3_S5_iiRi)
                  800103a0    000003c8                           : wlocale.obj (.text:_ZNKSt9money_putIwSt19ostreambuf_iteratorIwSt11char_traitsIwEEE6do_putES3_bRSt8ios_basewe)
                  80010768    000003a4                           : wlocale.obj (.text:_ZNKSt9money_getIwSt19istreambuf_iteratorIwSt11char_traitsIwEEE6do_getES3_S3_bRSt8ios_baseRNSt5_IosbIiE8_IostateERe)
                  80010b0c    000003a4                           : wiostrea.obj (.text:_ZNSt13basic_filebufIwSt11char_traitsIwEE8overflowEi)
                  80010eb0    000003a0                           : wlocale.obj (.text:_ZNKSt9money_putIwSt19ostreambuf_iteratorIwSt11char_traitsIwEEE6do_putES3_bRSt8ios_basewRKSbIwS2_SaIwEE)
                  80011250    000003a0     SimpleClass.obj (.text:_ZStlsISt11char_traitsIcEERSt13basic_ostreamIcT_ES5_PKc)
                  800115f0    00000398     rtsv7A8_A_le_eabi.lib : iostream.obj (.text:_ZNSt13basic_filebufIcSt11char_traitsIcEE8overflowEi)
                  80011988    0000038c                           : wlocale.obj (.text:_ZNKSt7num_putIwSt19ostreambuf_iteratorIwSt11char_traitsIwEEE6do_putES3_RSt8ios_basewb)
                  80011d14    00000388     SimpleClass.obj (.text:_ZNKSt7num_putIcSt19ostreambuf_iteratorIcSt11char_traitsIcEEE5_IputES3_RSt8ios_basecPcj)
                  8001209c    00000378     rtsv7A8_A_le_eabi.lib : iostream.obj (.text:_ZNSt13basic_filebufIcSt11char_traitsIcEE5uflowEv)
                  80012414    00000378                           : wiostrea.obj (.text:_ZNSt13basic_filebufIwSt11char_traitsIwEE5uflowEv)
                  8001278c    00000368                           : xlocale.obj (.text:_ZNKSt9money_putIcSt19ostreambuf_iteratorIcSt11char_traitsIcEEE6do_putES3_bRSt8ios_basece)
                  80012af4    00000360                           : xlocale.obj (.text:_ZNKSt8time_getIcSt19istreambuf_iteratorIcSt11char_traitsIcEEE7_GetintERS3_S5_iiRi)
                  80012e54    00000344                           : strtod.obj (.text)
                  80013198    000002fc                           : iostream.obj (.text:_ZNSt13basic_filebufIcSt11char_traitsIcEE9_EndwriteEv)
                  80013494    000002fc                           : wiostrea.obj (.text:_ZNSt13basic_filebufIwSt11char_traitsIwEE9_EndwriteEv)
                  80013790    000002e4                           : strtoll.obj (.text)
                  80013a74    000002d4                           : fopen.obj (.text)
                  80013d48    000002c8                           : locale.obj (.text:_ZNKSt7num_getIcSt19istreambuf_iteratorIcSt11char_traitsIcEEE6do_getES3_S3_RSt8ios_baseRNSt5_IosbIiE8_IostateERb)
                  80014010    000002c4                           : wlocale.obj (.text:_ZNKSt8time_putIwSt19ostreambuf_iteratorIwSt11char_traitsIwEEE6do_putES3_RSt8ios_basewPKSt2tmcc)
                  800142d4    000002c0                           : wlocale.obj (.text:_ZNKSt7num_putIwSt19ostreambuf_iteratorIwSt11char_traitsIwEEE5_IputES3_RSt8ios_basewPcj)
                  80014594    000002c0                           : wlocale.obj (.text:_ZSt10_GetloctxtIwSt19istreambuf_iteratorIwSt11char_traitsIwEEEiRT0_S5_jPKT_)
                  80014854    000002b8                           : ull_div32.obj (.text)
                  80014b0c    000002b4     SimpleClass.obj (.text)
                  80014dc0    000002a0     SimpleClass.obj (.text:_ZNKSt7num_putIcSt19ostreambuf_iteratorIcSt11char_traitsIcEEE6do_putES3_RSt8ios_basecd)
                  80015060    000002a0     SimpleClass.obj (.text:_ZNKSt7num_putIcSt19ostreambuf_iteratorIcSt11char_traitsIcEEE6do_putES3_RSt8ios_basece)
                  80015300    00000298     rtsv7A8_A_le_eabi.lib : locale.obj (.text:_ZSt10_GetloctxtIcSt19istreambuf_iteratorIcSt11char_traitsIcEEEiRT0_S5_jPKT_)
                  80015598    00000258                           : xlocale.obj (.text:_ZNKSt9money_putIcSt19ostreambuf_iteratorIcSt11char_traitsIcEEE6do_putES3_bRSt8ios_basecRKSs)
                  800157f0    00000244                           : fwrite.obj (.text)
                  80015a34    00000244                           : strtoull.obj (.text)
                  80015c78    0000023c     SimpleClass.obj (.text:_ZNKSt7num_putIcSt19ostreambuf_iteratorIcSt11char_traitsIcEEE6do_putES3_RSt8ios_basecb)
                  80015eb4    00000234     rtsv7A8_A_le_eabi.lib : xlocale.obj (.text:_ZNKSt9money_getIcSt19istreambuf_iteratorIcSt11char_traitsIcEEE6do_getES3_S3_bRSt8ios_baseRNSt5_IosbIiE8_IostateERe)
                  800160e8    00000220                           : wlocale.obj (.text:_ZNKSt7num_putIwSt19ostreambuf_iteratorIwSt11char_traitsIwEEE6do_putES3_RSt8ios_basewd)
                  80016308    00000220                           : wlocale.obj (.text:_ZNKSt7num_putIwSt19ostreambuf_iteratorIwSt11char_traitsIwEEE6do_putES3_RSt8ios_basewe)
                  80016528    0000021c                           : xlocale.obj (.text:_ZNKSt8time_putIcSt19ostreambuf_iteratorIcSt11char_traitsIcEEE6do_putES3_RSt8ios_basecPKSt2tmcc)
                  80016744    00000214                           : fd_add32.obj (.text)
                  80016958    00000210                           : wchar.obj (.text)
                  80016b68    00000208                           : xlocale.obj (.text:_ZNKSt7collateIcE12do_transformEPKcS2_)
                  80016d70    00000204                           : wlocale.obj (.text:_ZNKSt7collateIwE12do_transformEPKwS2_)
                  80016f74    000001f8                           : strtol.obj (.text)
                  8001716c    000001cc                           : string.obj (.text)
                  80017338    000001c8                           : fputs.obj (.text)
                  80017500    000001c0                           : strtoul.obj (.text)
                  800176c0    000001a8                           : xdscale.obj (.text)
                  80017868    000001a0                           : wiostrea.obj (.text:_ZNSt9basic_iosIwSt11char_traitsIwEE4initEPSt15basic_streambufIwS1_Eb)
                  80017a08    0000019c                           : wlocale.obj (.text:_ZNKSt9money_getIwSt19istreambuf_iteratorIwSt11char_traitsIwEEE6do_getES3_S3_bRSt8ios_baseRNSt5_IosbIiE8_IostateERSbIwS2_SaIwEE)
                  80017ba4    0000019c                           : iostream.obj (.text:_ZNSt9basic_iosIcSt11char_traitsIcEE4initEPSt15basic_streambufIcS1_Eb)
                  80017d40    00000198                           : xlocale.obj (.text:_ZNKSt9money_getIcSt19istreambuf_iteratorIcSt11char_traitsIcEEE6do_getES3_S3_bRSt8ios_baseRNSt5_IosbIiE8_IostateERSs)
                  80017ed8    00000194     SimpleClass.obj (.text:_ZNSolsEi)
                  8001806c    00000194     rtsv7A8_A_le_eabi.lib : dtor_list.obj (.text)
                  80018200    00000190                           : wlocale.obj (.text:_ZNSt7_MpunctIwE5_InitERKSt8_Locinfo)
                  80018390    00000190                           : fd_div32.obj (.text)
                  80018520    00000184                           : wlocale.obj (.text:_ZNKSt7_MpunctIwE11do_groupingEv)
                  800186a4    00000184                           : wlocale.obj (.text:_ZNKSt8numpunctIwE11do_groupingEv)
                  80018828    00000180                           : memcpy32.obj (.text)
                  800189a8    00000170                           : wlocale.obj (.text:_ZNKSt8time_getIwSt19istreambuf_iteratorIwSt11char_traitsIwEEE11do_get_timeES3_S3_RSt8ios_baseRNSt5_IosbIiE8_IostateEPSt2tm)
                  80018b18    00000160                           : xlocale.obj (.text:_ZNSt7_MpunctIcE5_InitERKSt8_Locinfo)
                  80018c78    00000160                           : xdnorm.obj (.text)
                  80018dd8    0000015c     SimpleClass.obj (.text:_ZNKSt7num_putIcSt19ostreambuf_iteratorIcSt11char_traitsIcEEE5_IfmtEPcPKcNSt5_IosbIiE9_FmtflagsE)
                  80018f34    00000158     rtsv7A8_A_le_eabi.lib : setvbuf.obj (.text)
                  8001908c    00000154                           : typeinfo_.obj (.text)
                  800191e0    0000014c                           : wiostrea.obj (.text:_ZNSt13basic_filebufIwSt11char_traitsIwEE5imbueERKSt6locale)
                  8001932c    00000148                           : iostream.obj (.text:_ZNSt13basic_filebufIcSt11char_traitsIcEE5imbueERKSt6locale)
                  80019474    00000144                           : xlocale.obj (.text:_ZNKSt8time_getIcSt19istreambuf_iteratorIcSt11char_traitsIcEEE11do_get_timeES3_S3_RSt8ios_baseRNSt5_IosbIiE8_IostateEPSt2tm)
                  800195b8    00000134                           : iostream.obj (.text:_ZNSt13basic_filebufIcSt11char_traitsIcEE7seekoffElNSt5_IosbIiE8_SeekdirENS4_9_OpenmodeE)
                  800196ec    00000134                           : wiostrea.obj (.text:_ZNSt13basic_filebufIwSt11char_traitsIwEE7seekoffElNSt5_IosbIiE8_SeekdirENS4_9_OpenmodeE)
                  80019820    00000130     SimpleClass.obj (.text:_ZNKSt7num_putIcSt19ostreambuf_iteratorIcSt11char_traitsIcEEE5_FfmtEPccNSt5_IosbIiE9_FmtflagsE)
                  80019950    00000130     rtsv7A8_A_le_eabi.lib : fflush.obj (.text)
                  80019a80    0000012c     SimpleClass.obj (.text:_ZNSt8numpunctIcE5_InitERKSt8_Locinfo)
                  80019bac    00000128     rtsv7A8_A_le_eabi.lib : iostream.obj (.text:_ZNSt13basic_filebufIcSt11char_traitsIcEE7seekposESt4fposIiENSt5_IosbIiE9_OpenmodeE)
                  80019cd4    00000128                           : wiostrea.obj (.text:_ZNSt13basic_filebufIwSt11char_traitsIwEE7seekposESt4fposIiENSt5_IosbIiE9_OpenmodeE)
                  80019dfc    00000128                           : fd_mul32.obj (.text)
                  80019f24    0000011c     SimpleClass.obj (.text:_ZNKSt7num_putIcSt19ostreambuf_iteratorIcSt11char_traitsIcEEE11_PutgroupedES3_PKcjc)
                  8001a040    0000011c     rtsv7A8_A_le_eabi.lib : wlocale.obj (.text:_ZNSbIwSt11char_traitsIwESaIwEE6insertEjjw)
                  8001a15c    00000118                           : _io_perm.obj (.text)
                  8001a274    00000114                           : wlocale.obj (.text:_ZNKSt7_MpunctIwE14do_curr_symbolEv)
                  8001a388    00000114                           : wlocale.obj (.text:_ZNKSt7_MpunctIwE16do_negative_signEv)
                  8001a49c    00000114                           : wlocale.obj (.text:_ZNKSt7_MpunctIwE16do_positive_signEv)
                  8001a5b0    00000114                           : locale.obj (.text:_ZNKSt7num_getIcSt19istreambuf_iteratorIcSt11char_traitsIcEEE6do_getES3_S3_RSt8ios_baseRNSt5_IosbIiE8_IostateERt)
                  8001a6c4    00000114                           : wlocale.obj (.text:_ZNKSt7num_getIwSt19istreambuf_iteratorIwSt11char_traitsIwEEE6do_getES3_S3_RSt8ios_baseRNSt5_IosbIiE8_IostateERt)
                  8001a7d8    00000114                           : wlocale.obj (.text:_ZNKSt8numpunctIwE11do_truenameEv)
                  8001a8ec    00000114                           : wlocale.obj (.text:_ZNKSt8numpunctIwE12do_falsenameEv)
                  8001aa00    00000114                           : i_div32.obj (.text)
                  8001ab14    00000110     SimpleClass.obj (.text:_ZNSs5_CopyEjj)
                  8001ac24    0000010c     rtsv7A8_A_le_eabi.lib : wlocale.obj (.text:_ZNSbIwSt11char_traitsIwESaIwEE6assignERKS2_jj)
                  8001ad30    00000108                           : locale.obj (.text:_ZNKSt7num_getIcSt19istreambuf_iteratorIcSt11char_traitsIcEEE6do_getES3_S3_RSt8ios_baseRNSt5_IosbIiE8_IostateERj)
                  8001ae38    00000108                           : wlocale.obj (.text:_ZNKSt7num_getIwSt19istreambuf_iteratorIwSt11char_traitsIwEEE6do_getES3_S3_RSt8ios_baseRNSt5_IosbIiE8_IostateERj)
                  8001af40    00000100     SimpleClass.obj (.text:_ZNSs6appendERKSsjj)
                  8001b040    00000100     rtsv7A8_A_le_eabi.lib : xlocale.obj (.text:_ZSt9use_facetISt10moneypunctIcLb1EEERKT_RKSt6locale)
                  8001b140    00000100                           : wlocale.obj (.text:_ZSt9use_facetISt10moneypunctIwLb1EEERKT_RKSt6locale)
                  8001b240    00000100                           : fputc.obj (.text)
                  8001b340    000000fc                           : wlocale.obj (.text:_ZNKSt7num_putIwSt19ostreambuf_iteratorIwSt11char_traitsIwEEE11_PutgroupedES3_PKcjw)
                  8001b43c    000000fc     SimpleClass.obj (.text:_ZNSs6insertEjjc)
                  8001b538    000000fc     rtsv7A8_A_le_eabi.lib : wlocale.obj (.text:_ZNSt8numpunctIwE5_InitERKSt8_Locinfo)
                  8001b634    000000fc                           : xlocale.obj (.text:_ZSt9use_facetISt10moneypunctIcLb0EEERKT_RKSt6locale)
                  8001b730    000000fc                           : wlocale.obj (.text:_ZSt9use_facetISt10moneypunctIwLb0EEERKT_RKSt6locale)
                  8001b82c    000000fc                           : fclose.obj (.text)
                  8001b928    000000f8                           : wlocale.obj (.text:_ZSt9use_facetISt5ctypeIwEERKT_RKSt6locale)
                  8001ba20    000000f4     SimpleClass.obj (.text:_ZNSs6assignERKSsjj)
                  8001bb14    000000f0     rtsv7A8_A_le_eabi.lib : _bufread.obj (.text)
                  8001bc04    000000f0                           : u_div32.obj (.text)
                  8001bcf4    000000f0                           : xlocinfo.obj (.text)
                  8001bde4    000000ec                           : locale.obj (.text:_ZNKSt7num_getIcSt19istreambuf_iteratorIcSt11char_traitsIcEEE6do_getES3_S3_RSt8ios_baseRNSt5_IosbIiE8_IostateERPv)
                  8001bed0    000000ec                           : locale.obj (.text:_ZNKSt7num_getIcSt19istreambuf_iteratorIcSt11char_traitsIcEEE6do_getES3_S3_RSt8ios_baseRNSt5_IosbIiE8_IostateERx)
                  8001bfbc    000000ec                           : locale.obj (.text:_ZNKSt7num_getIcSt19istreambuf_iteratorIcSt11char_traitsIcEEE6do_getES3_S3_RSt8ios_baseRNSt5_IosbIiE8_IostateERy)
                  8001c0a8    000000ec                           : wlocale.obj (.text:_ZNKSt7num_getIwSt19istreambuf_iteratorIwSt11char_traitsIwEEE6do_getES3_S3_RSt8ios_baseRNSt5_IosbIiE8_IostateERPv)
                  8001c194    000000ec                           : wlocale.obj (.text:_ZNKSt7num_getIwSt19istreambuf_iteratorIwSt11char_traitsIwEEE6do_getES3_S3_RSt8ios_baseRNSt5_IosbIiE8_IostateERx)
                  8001c280    000000ec                           : wlocale.obj (.text:_ZNKSt7num_getIwSt19istreambuf_iteratorIwSt11char_traitsIwEEE6do_getES3_S3_RSt8ios_baseRNSt5_IosbIiE8_IostateERy)
                  8001c36c    000000ec     SimpleClass.obj (.text:_ZNSo6sentryC1ERSo)
                  8001c458    000000ec     rtsv7A8_A_le_eabi.lib : multibyte.obj (.text)
                  8001c544    000000e8                           : locale.obj (.text:_ZNKSt7num_getIcSt19istreambuf_iteratorIcSt11char_traitsIcEEE6do_getES3_S3_RSt8ios_baseRNSt5_IosbIiE8_IostateERl)
                  8001c62c    000000e8                           : locale.obj (.text:_ZNKSt7num_getIcSt19istreambuf_iteratorIcSt11char_traitsIcEEE6do_getES3_S3_RSt8ios_baseRNSt5_IosbIiE8_IostateERm)
                  8001c714    000000e8                           : wlocale.obj (.text:_ZNKSt7num_getIwSt19istreambuf_iteratorIwSt11char_traitsIwEEE6do_getES3_S3_RSt8ios_baseRNSt5_IosbIiE8_IostateERl)
                  8001c7fc    000000e8                           : wlocale.obj (.text:_ZNKSt7num_getIwSt19istreambuf_iteratorIwSt11char_traitsIwEEE6do_getES3_S3_RSt8ios_baseRNSt5_IosbIiE8_IostateERm)
                  8001c8e4    000000e4                           : locale.obj (.text:_ZNKSt7num_getIcSt19istreambuf_iteratorIcSt11char_traitsIcEEE6do_getES3_S3_RSt8ios_baseRNSt5_IosbIiE8_IostateERd)
                  8001c9c8    000000e4                           : locale.obj (.text:_ZNKSt7num_getIcSt19istreambuf_iteratorIcSt11char_traitsIcEEE6do_getES3_S3_RSt8ios_baseRNSt5_IosbIiE8_IostateERe)
                  8001caac    000000e4                           : wlocale.obj (.text:_ZNKSt7num_getIwSt19istreambuf_iteratorIwSt11char_traitsIwEEE6do_getES3_S3_RSt8ios_baseRNSt5_IosbIiE8_IostateERd)
                  8001cb90    000000e4                           : wlocale.obj (.text:_ZNKSt7num_getIwSt19istreambuf_iteratorIwSt11char_traitsIwEEE6do_getES3_S3_RSt8ios_baseRNSt5_IosbIiE8_IostateERe)
                  8001cc74    000000e4                           : wlocale.obj (.text:_ZNKSt8messagesIwE6do_getEiiiRKSbIwSt11char_traitsIwESaIwEE)
                  8001cd58    000000e4     SimpleClass.obj (.text:_ZNSs5eraseEjj)
                  8001ce3c    000000e0     rtsv7A8_A_le_eabi.lib : locale.obj (.text:_ZNKSt7num_getIcSt19istreambuf_iteratorIcSt11char_traitsIcEEE6do_getES3_S3_RSt8ios_baseRNSt5_IosbIiE8_IostateERf)
                  8001cf1c    000000e0                           : wlocale.obj (.text:_ZNKSt7num_getIwSt19istreambuf_iteratorIwSt11char_traitsIwEEE6do_getES3_S3_RSt8ios_baseRNSt5_IosbIiE8_IostateERf)
                  8001cffc    000000e0                           : xlocale.obj (.text:_ZNKSt8messagesIcE6do_getEiiiRKSs)
                  8001d0dc    000000e0                           : wiostrea.obj (.text:_ZNSt13basic_filebufIwSt11char_traitsIwEED0Ev)
                  8001d1bc    000000e0                           : wlocale.obj (.text:_ZSt9use_facetISt8numpunctIwEERKT_RKSt6locale)
                  8001d29c    000000e0                           : fd_cmp32.obj (.text:__aeabi_cdcmple)
                  8001d37c    000000e0                           : fd_cmp32.obj (.text:__aeabi_cdrcmple)
                  8001d45c    000000e0                           : fgetc.obj (.text)
                  8001d53c    000000dc     SimpleClass.obj (.text:_ZNSs6appendEPKcj)
                  8001d618    000000d8     rtsv7A8_A_le_eabi.lib : wiostrea.obj (.text:_ZNKSt7codecvtIwciE6do_outERiPKwS3_RS3_PcS5_RS5_)
                  8001d6f0    000000d8                           : wiostrea.obj (.text:_ZNSt13basic_filebufIwSt11char_traitsIwEED1Ev)
                  8001d7c8    000000d4     SimpleClass.obj (.text:_ZNSs5_GrowEjb)
                  8001d89c    000000d0     rtsv7A8_A_le_eabi.lib : wlocale.obj (.text:_ZNSbIwSt11char_traitsIwESaIwEE6appendEjw)
                  8001d96c    000000d0                           : wiostrea.obj (.text:_ZNSt13basic_filebufIwSt11char_traitsIwEE6setbufEPwi)
                  8001da3c    000000cc     SimpleClass.obj (.text:_ZNSo3putEc)
                  8001db08    000000cc     SimpleClass.obj (.text:_ZSt9use_facetISt5ctypeIcEERKT_RKSt6locale)
                  8001dbd4    000000cc     SimpleClass.obj (.text:_ZSt9use_facetISt7num_putIcSt19ostreambuf_iteratorIcSt11char_traitsIcEEEERKT_RKSt6locale)
                  8001dca0    000000cc     SimpleClass.obj (.text:_ZSt9use_facetISt8numpunctIcEERKT_RKSt6locale)
                  8001dd6c    000000c8     rtsv7A8_A_le_eabi.lib : wlocale.obj (.text:_ZNSbIwSt11char_traitsIwESaIwEE5_CopyEjj)
                  8001de34    000000c8                           : iostream.obj (.text:_ZNSt13basic_filebufIcSt11char_traitsIcEE9pbackfailEi)
                  8001defc    000000c8                           : wiostrea.obj (.text:_ZNSt13basic_filebufIwSt11char_traitsIwEE9pbackfailEi)
                  8001dfc4    000000c8                           : ungetc.obj (.text)
                  8001e08c    000000c0                           : wiostrea.obj (.text:_ZNKSt7codecvtIwciE5do_inERiPKcS3_RS3_PwS5_RS5_)
                  8001e14c    000000b8                           : stox.obj (.text)
                  8001e204    000000b8                           : xdunscal.obj (.text)
                  8001e2bc    000000b0     SimpleClass.obj (.text:_ZNKSt7num_putIcSt19ostreambuf_iteratorIcSt11char_traitsIcEEE6do_putES3_RSt8ios_basecPKv)
                  8001e36c    000000b0     rtsv7A8_A_le_eabi.lib : wiostrea.obj (.text:_ZNSt15basic_streambufIwSt11char_traitsIwEE6xsputnEPKwi)
                  8001e41c    000000b0                           : wlocale.obj (.text:_ZSt10_MaklocstrIwEPT_PKcS1_RKSt7_Cvtvec)
                  8001e4cc    000000b0                           : memset32.obj (.text)
                  8001e57c    000000ac     SimpleClass.obj (.text:_ZNSo12_Sentry_baseC1ERSo)
                  8001e628    000000ac     rtsv7A8_A_le_eabi.lib : wiostrea.obj (.text:_ZNSt15basic_streambufIwSt11char_traitsIwEE6xsgetnEPwi)
                  8001e6d4    000000a8                           : xlocale.obj (.text:_ZNKSt8time_getIcSt19istreambuf_iteratorIcSt11char_traitsIcEEE11do_get_yearES3_S3_RSt8ios_baseRNSt5_IosbIiE8_IostateEPSt2tm)
                  8001e77c    000000a8                           : wlocale.obj (.text:_ZNKSt8time_getIwSt19istreambuf_iteratorIwSt11char_traitsIwEEE11do_get_yearES3_S3_RSt8ios_baseRNSt5_IosbIiE8_IostateEPSt2tm)
                  8001e824    000000a8                           : iostream.obj (.text:_ZNSt13basic_filebufIcSt11char_traitsIcEE6setbufEPci)
                  8001e8cc    000000a8                           : iostream.obj (.text:_ZNSt15basic_streambufIcSt11char_traitsIcEE6xsputnEPKci)
                  8001e974    000000a8                           : fseek.obj (.text)
                  8001ea1c    000000a8                           : sprintf.obj (.text)
                  8001eac4    000000a4                           : iostream.obj (.text:_ZNSt15basic_streambufIcSt11char_traitsIcEE6xsgetnEPci)
                  8001eb68    000000a4     SimpleClass.obj (.text:_ZNSt5ctypeIcEC1EPKsbj)
                  8001ec0c    000000a4     rtsv7A8_A_le_eabi.lib : autoinit.obj (.text)
                  8001ecb0    000000a4                           : ftell.obj (.text)
                  8001ed54    000000a4                           : trgmsg.obj (.text)
                  8001edf8    000000a0                           : copy_decompress_rle.obj (.text)
                  8001ee98    0000009c                           : wlocale.obj (.text:_ZNSbIwSt11char_traitsIwESaIwEE5eraseEjj)
                  8001ef34    0000009c     SimpleClass.obj (.text:_ZNSo12_Sentry_baseD1Ev)
                  8001efd0    0000009c     SimpleClass.obj (.text:_ZNSs6appendEjc)
                  8001f06c    0000009c     rtsv7A8_A_le_eabi.lib : xlocale.obj (.text:_ZNSt8time_getIcSt19istreambuf_iteratorIcSt11char_traitsIcEEE5_InitERKSt8_Locinfo)
                  8001f108    00000098     SimpleClass.obj (.text:_ZNKSt7num_putIcSt19ostreambuf_iteratorIcSt11char_traitsIcEEE5_PutcES3_PKcj)
                  8001f1a0    00000098     SimpleClass.obj (.text:_ZNKSt7num_putIcSt19ostreambuf_iteratorIcSt11char_traitsIcEEE6do_putES3_RSt8ios_basecx)
                  8001f238    00000098     SimpleClass.obj (.text:_ZNKSt7num_putIcSt19ostreambuf_iteratorIcSt11char_traitsIcEEE6do_putES3_RSt8ios_basecy)
                  8001f2d0    00000094     SimpleClass.obj (.text:_ZNKSt7num_putIcSt19ostreambuf_iteratorIcSt11char_traitsIcEEE6do_putES3_RSt8ios_basecl)
                  8001f364    00000094     SimpleClass.obj (.text:_ZNKSt7num_putIcSt19ostreambuf_iteratorIcSt11char_traitsIcEEE6do_putES3_RSt8ios_basecm)
                  8001f3f8    00000094     SimpleClass.obj (.text:_ZNSs5_TidyEbj)
                  8001f48c    00000090     rtsv7A8_A_le_eabi.lib : wlocale.obj (.text:_ZNKSt7num_putIwSt19ostreambuf_iteratorIwSt11char_traitsIwEEE6do_putES3_RSt8ios_basewPKv)
                  8001f51c    00000090                           : wlocale.obj (.text:_ZNKSt7num_putIwSt19ostreambuf_iteratorIwSt11char_traitsIwEEE6do_putES3_RSt8ios_basewx)
                  8001f5ac    00000090                           : wlocale.obj (.text:_ZNKSt7num_putIwSt19ostreambuf_iteratorIwSt11char_traitsIwEEE6do_putES3_RSt8ios_basewy)
                  8001f63c    00000090     SimpleClass.obj (.text:_ZSt10_MaklocstrIcEPT_PKcS1_RKSt7_Cvtvec)
                  8001f6cc    0000008c     rtsv7A8_A_le_eabi.lib : locale0.obj (.text:_ZNKSs7compareEjjPKcj)
                  8001f758    0000008c                           : wlocale.obj (.text:_ZNKSt7num_putIwSt19ostreambuf_iteratorIwSt11char_traitsIwEEE6do_putES3_RSt8ios_basewl)
                  8001f7e4    0000008c                           : wlocale.obj (.text:_ZNKSt7num_putIwSt19ostreambuf_iteratorIwSt11char_traitsIwEEE6do_putES3_RSt8ios_basewm)
                  8001f870    0000008c                           : iostream.obj (.text:_ZNSt13basic_filebufIcSt11char_traitsIcEED0Ev)
                  8001f8fc    00000088                           : wiostrea.obj (.text:_ZNKSt7codecvtIwciE10do_unshiftERiPcS2_RS2_)
                  8001f984    00000088     SimpleClass.obj (.text:_ZNSo5flushEv)
                  8001fa0c    00000088     SimpleClass.obj (.text:_ZNSs6assignEPKcj)
                  8001fa94    00000088     rtsv7A8_A_le_eabi.lib : _tvaltostr.obj (.text)
                  8001fb1c    00000084                           : wiostrea.obj (.text:_ZNKSt7codecvtIwciE9do_lengthERKiPKcS4_j)
                  8001fba0    00000084                           : iostream.obj (.text:_ZNSt13basic_filebufIcSt11char_traitsIcEED1Ev)
                  8001fc24    00000084                           : atoi.obj (.text)
                  8001fca8    00000084                           : cpy_tbl.obj (.text)
                  8001fd2c    00000084                           : throw.obj (.text)
                  8001fdb0    00000080                           : ltoa.obj (.text)
                  8001fe30    0000007c     SimpleClass.obj (.text:_ZNKSt7num_putIcSt19ostreambuf_iteratorIcSt11char_traitsIcEEE4_PutES3_PKcj)
                  8001feac    0000007c     rtsv7A8_A_le_eabi.lib : locale.obj (.text:_ZNSt19istreambuf_iteratorIcSt11char_traitsIcEEppEv)
                  8001ff28    0000007c                           : wlocale.obj (.text:_ZNSt19istreambuf_iteratorIwSt11char_traitsIwEEppEv)
                  8001ffa4    00000078                           : wiostrea.obj (.text:_ZNKSt5ctypeIwE10do_toupperEPwPKw)
                  8002001c    00000078                           : wlocale.obj (.text:_ZNKSt7num_putIwSt19ostreambuf_iteratorIwSt11char_traitsIwEEE5_IfmtEPcPKcNSt5_IosbIiE9_FmtflagsE)
                  80020094    00000078                           : wlocale.obj (.text:_ZNKSt7num_putIwSt19ostreambuf_iteratorIwSt11char_traitsIwEEE5_PutcES3_PKcj)
                  8002010c    00000078                           : locale.obj (.text:_ZNSt19istreambuf_iteratorIcSt11char_traitsIcEE5_PeekEv)
                  80020184    00000078                           : wlocale.obj (.text:_ZNSt19istreambuf_iteratorIwSt11char_traitsIwEE5_PeekEv)
                  800201fc    00000078                           : exit.obj (.text)
                  80020274    00000074                           : string.obj (.text:_ZNSt12out_of_rangeC1ERKSs)
                  800202e8    00000074                           : wlocale.obj (.text:_ZNSt19ostreambuf_iteratorIwSt11char_traitsIwEEaSEw)
                  8002035c    00000074     SimpleClass.obj (.text:_ZNSt6locale5facet7_DecrefEv)
                  800203d0    00000070     rtsv7A8_A_le_eabi.lib : wlocale.obj (.text:_ZNKSt7num_putIwSt19ostreambuf_iteratorIwSt11char_traitsIwEEE5_FfmtEPccNSt5_IosbIiE9_FmtflagsE)
                  80020440    00000070     SimpleClass.obj (.text:_ZNSt19ostreambuf_iteratorIcSt11char_traitsIcEEaSEc)
                  800204b0    00000070     rtsv7A8_A_le_eabi.lib : locale.obj (.text:_ZStneIcSt11char_traitsIcEEbRKSt19istreambuf_iteratorIT_T0_ES7_)
                  80020520    00000070                           : wlocale.obj (.text:_ZStneIwSt11char_traitsIwEEbRKSt19istreambuf_iteratorIT_T0_ES7_)
                  80020590    0000006c     SimpleClass.obj (.text:_ZNKSt7num_putIcSt19ostreambuf_iteratorIcSt11char_traitsIcEEE4_RepES3_cj)
                  800205fc    00000068     rtsv7A8_A_le_eabi.lib : wiostrea.obj (.text:_ZNKSt5ctypeIwE10do_tolowerEPwPKw)
                  80020664    00000068                           : string.obj (.text:_ZNSt11logic_errorC2ERKSs)
                  800206cc    00000068                           : iostream.obj (.text:_ZNSt13basic_filebufIcSt11char_traitsIcEE9underflowEv)
                  80020734    00000068                           : wiostrea.obj (.text:_ZNSt13basic_filebufIwSt11char_traitsIwEE9underflowEv)
                  8002079c    00000068                           : ldexp.obj (.text)
                  80020804    00000064                           : xlocale.obj (.text:_ZNKSt7collateIcE10do_compareEPKcS2_S2_S2_)
                  80020868    00000064                           : wlocale.obj (.text:_ZNKSt7collateIwE10do_compareEPKwS2_S2_S2_)
                  800208cc    00000064     SimpleClass.obj (.text:_ZNKSt7num_putIcSt19ostreambuf_iteratorIcSt11char_traitsIcEEE3putES3_RSt8ios_basecl)
                  80020930    00000064     SimpleClass.obj (.text:_ZNSs9_ChassignEjjc)
                  80020994    00000064     SimpleClass.obj (.text:_ZNSt5ctypeIcE7_GetcatEPPKNSt6locale5facetE)
                  800209f8    00000064     SimpleClass.obj (.text:_ZNSt6locale2idcvjEv)
                  80020a5c    00000064     rtsv7A8_A_le_eabi.lib : locale.obj (.text:_ZSteqIcSt11char_traitsIcEEbRKSt19istreambuf_iteratorIT_T0_ES7_)
                  80020ac0    00000064                           : wlocale.obj (.text:_ZSteqIwSt11char_traitsIwEEbRKSt19istreambuf_iteratorIT_T0_ES7_)
                  80020b24    00000064                           : signal.obj (.text)
                  80020b88    00000060     SimpleClass.obj (.text:_ZNKSt5ctypeIcE10do_tolowerEPcPKc)
                  80020be8    00000060     SimpleClass.obj (.text:_ZNKSt5ctypeIcE10do_toupperEPcPKc)
                  80020c48    00000060     rtsv7A8_A_le_eabi.lib : xlocale.obj (.text:_ZNKSt8time_getIcSt19istreambuf_iteratorIcSt11char_traitsIcEEE14do_get_weekdayES3_S3_RSt8ios_baseRNSt5_IosbIiE8_IostateEPSt2tm)
                  80020ca8    00000060                           : xlocale.obj (.text:_ZNKSt8time_getIcSt19istreambuf_iteratorIcSt11char_traitsIcEEE16do_get_monthnameES3_S3_RSt8ios_baseRNSt5_IosbIiE8_IostateEPSt2tm)
                  80020d08    00000060                           : wlocale.obj (.text:_ZNKSt8time_getIwSt19istreambuf_iteratorIwSt11char_traitsIwEEE14do_get_weekdayES3_S3_RSt8ios_baseRNSt5_IosbIiE8_IostateEPSt2tm)
                  80020d68    00000060                           : wlocale.obj (.text:_ZNKSt8time_getIwSt19istreambuf_iteratorIwSt11char_traitsIwEEE16do_get_monthnameES3_S3_RSt8ios_baseRNSt5_IosbIiE8_IostateEPSt2tm)
                  80020dc8    00000060                           : iostream.obj (.text:_ZNSt15basic_streambufIcSt11char_traitsIcEE5_InitEv)
                  80020e28    00000060     SimpleClass.obj (.text:_ZNSt15basic_streambufIcSt11char_traitsIcEE5sputcEc)
                  80020e88    00000060     rtsv7A8_A_le_eabi.lib : xlocale.obj (.text:_ZNSt7_MpunctIcE7_MakpatERNSt10money_base7patternEjjj)
                  80020ee8    00000060                           : wlocale.obj (.text:_ZNSt7_MpunctIwE7_MakpatERNSt10money_base7patternEjjj)
                  80020f48    0000005c                           : wiostrea.obj (.text:_ZNKSt5ctypeIwE8do_widenEPKcS2_Pw)
                  80020fa4    0000005c                           : wiostrea.obj (.text:_ZNKSt5ctypeIwE9do_narrowEPKwS2_cPc)
                  80021000    0000005c     SimpleClass.obj (.text:_ZNSt7num_putIcSt19ostreambuf_iteratorIcSt11char_traitsIcEEE7_GetcatEPPKNSt6locale5facetE)
                  8002105c    0000005c     SimpleClass.obj (.text:_ZNSt7num_putIcSt19ostreambuf_iteratorIcSt11char_traitsIcEEEC1Ej)
                  800210b8    0000005c     SimpleClass.obj (.text:_ZNSt8numpunctIcE7_GetcatEPPKNSt6locale5facetE)
                  80021114    0000005c     SimpleClass.obj (.text:_ZNSt8numpunctIcEC1Ej)
                  80021170    0000005c     rtsv7A8_A_le_eabi.lib : fd_toi32.obj (.text)
                  800211cc    0000005c                           : fd_tos32.obj (.text)
                  80021228    00000058                           : wlocale.obj (.text:_ZNSt8time_getIwSt19istreambuf_iteratorIwSt11char_traitsIwEEE5_InitERKSt8_Locinfo)
                  80021280    00000058                           : feraiseexcept.obj (.text)
                  800212d8    00000054                           : ios.obj (.text:_ZNSt6localeaSERKS_)
                  8002132c    00000054     SimpleClass.obj (.text:_ZSt4endlIcSt11char_traitsIcEERSt13basic_ostreamIT_T0_ES6_)
                  80021380    00000054     rtsv7A8_A_le_eabi.lib : boot.obj (.text)
                  800213d4    00000050                           : wiostrea.obj (.text:_ZNKSt5ctypeIwE5do_isEPKwS2_Ps)
                  80021424    00000050                           : wlocale.obj (.text:_ZNKSt7num_putIwSt19ostreambuf_iteratorIwSt11char_traitsIwEEE4_RepES3_wj)
                  80021474    00000050     SimpleClass.obj (.text:_ZNKSt9basic_iosIcSt11char_traitsIcEE5widenEc)
                  800214c4    00000050     SimpleClass.obj (.text:_ZNSs7_InsideEPKc)
                  80021514    00000050     rtsv7A8_A_le_eabi.lib : ios.obj (.text:_ZNSt13runtime_errorD0Ev)
                  80021564    00000050                           : ios.obj (.text:_ZNSt8ios_base7failureD0Ev)
                  800215b4    00000050                           : xlocale.obj (.text:_ZNSt9money_putIcSt19ostreambuf_iteratorIcSt11char_traitsIcEEE4_PutES3_St22_String_const_iteratorIcS2_SaIcEEj)
                  80021604    00000050                           : xlocale.obj (.text:_ZNSt9money_putIcSt19ostreambuf_iteratorIcSt11char_traitsIcEEE4_RepES3_cj)
                  80021654    00000050                           : wlocale.obj (.text:_ZNSt9money_putIwSt19ostreambuf_iteratorIwSt11char_traitsIwEEE4_PutES3_St22_String_const_iteratorIwS2_SaIwEEj)
                  800216a4    00000050                           : wlocale.obj (.text:_ZNSt9money_putIwSt19ostreambuf_iteratorIwSt11char_traitsIwEEE4_RepES3_wj)
                  800216f4    0000004c                           : wiostrea.obj (.text:_ZNKSt5ctypeIwE11do_scan_notEsPKwS2_)
                  80021740    0000004c                           : iostream.obj (.text:_ZNSt13basic_filebufIcSt11char_traitsIcEE4syncEv)
                  8002178c    0000004c                           : wiostrea.obj (.text:_ZNSt13basic_filebufIwSt11char_traitsIwEE4syncEv)
                  800217d8    0000004c                           : iostream.obj (.text:_ZNSt15basic_streambufIcSt11char_traitsIcEE7seekposESt4fposIiENSt5_IosbIiE9_OpenmodeE)
                  80021824    0000004c                           : wiostrea.obj (.text:_ZNSt15basic_streambufIwSt11char_traitsIwEE7seekposESt4fposIiENSt5_IosbIiE9_OpenmodeE)
                  80021870    0000004c     SimpleClass.obj (.text:_ZNSt6localeD1Ev)
                  800218bc    0000004c     rtsv7A8_A_le_eabi.lib : new_.obj (.text)
                  80021908    0000004c                           : raise.obj (.text)
                  80021954    00000048     SimpleClass.obj (.text:_ZNKSt15basic_streambufIcSt11char_traitsIcEE8_PnavailEv)
                  8002199c    00000048     rtsv7A8_A_le_eabi.lib : wiostrea.obj (.text:_ZNKSt5ctypeIwE10do_toupperEw)
                  800219e4    00000048     SimpleClass.obj (.text:_ZNSt5ctypeIcE5_TidyEv)
                  80021a2c    00000048     rtsv7A8_A_le_eabi.lib : setlocale.obj (.text)
                  80021a74    00000048                           : strncpy.obj (.text)
                  80021abc    00000044                           : wiostrea.obj (.text:_ZNKSt5ctypeIwE10do_scan_isEsPKwS2_)
                  80021b00    00000044     SimpleClass.obj (.text:_ZNKSt8_Locinfo9_GetctypeEv)
                  80021b44    00000044     SimpleClass.obj (.text:_ZNSsC1EPKc)
                  80021b88    00000044     rtsv7A8_A_le_eabi.lib : xlocale.obj (.text:_ZNSt10moneypunctIcLb0EED0Ev)
                  80021bcc    00000044                           : xlocale.obj (.text:_ZNSt10moneypunctIcLb1EED0Ev)
                  80021c10    00000044                           : wlocale.obj (.text:_ZNSt10moneypunctIwLb0EED0Ev)
                  80021c54    00000044                           : wlocale.obj (.text:_ZNSt10moneypunctIwLb1EED0Ev)
                  80021c98    00000044                           : string.obj (.text:_ZNSt11logic_errorD0Ev)
                  80021cdc    00000044                           : string.obj (.text:_ZNSt12length_errorD0Ev)
                  80021d20    00000044                           : string.obj (.text:_ZNSt12out_of_rangeD0Ev)
                  80021d64    00000044                           : ios.obj (.text:_ZNSt13runtime_errorD1Ev)
                  80021da8    00000044                           : iostream.obj (.text:_ZNSt15basic_streambufIcSt11char_traitsIcEE7seekoffElNSt5_IosbIiE8_SeekdirENS4_9_OpenmodeE)
                  80021dec    00000044                           : wiostrea.obj (.text:_ZNSt15basic_streambufIwSt11char_traitsIwEE7seekoffElNSt5_IosbIiE8_SeekdirENS4_9_OpenmodeE)
                  80021e30    00000044                           : xlocale.obj (.text:_ZNSt7_MpunctIcED0Ev)
                  80021e74    00000044                           : wlocale.obj (.text:_ZNSt7_MpunctIwED0Ev)
                  80021eb8    00000044                           : ios.obj (.text:_ZNSt8ios_base7failureD1Ev)
                  80021efc    00000044                           : strcspn.obj (.text)
                  80021f40    00000044                           : xferaise.obj (.text)
                  80021f84    00000040                           : wiostrea.obj (.text:_ZNKSt5ctypeIwE10do_tolowerEw)
                  80021fc4    00000040                           : wlocale.obj (.text:_ZNSbIwSt11char_traitsIwESaIwEE9_ChassignEjjw)
                  80022004    00000040     SimpleClass.obj (.text:_ZNSt6locale5facet7_IncrefEv)
                  80022044    00000040     SimpleClass.obj (.text:_ZNSt9basic_iosIcSt11char_traitsIcEE5clearENSt5_IosbIiE8_IostateEb)
                  80022084    00000040     SimpleClass.obj (.text:_ZNSt9basic_iosIcSt11char_traitsIcEE8setstateENSt5_IosbIiE8_IostateEb)
                  800220c4    0000003c     SimpleClass.obj (.text:_ZNKSt5ctypeIcE8do_widenEPKcS2_Pc)
                  80022100    0000003c     SimpleClass.obj (.text:_ZNKSt5ctypeIcE9do_narrowEPKcS2_cPc)
                  8002213c    0000003c     rtsv7A8_A_le_eabi.lib : xlocale.obj (.text:_ZNKSt7_MpunctIcE11do_groupingEv)
                  80022178    0000003c                           : xlocale.obj (.text:_ZNKSt7_MpunctIcE14do_curr_symbolEv)
                  800221b4    0000003c                           : xlocale.obj (.text:_ZNKSt7_MpunctIcE16do_negative_signEv)
                  800221f0    0000003c                           : xlocale.obj (.text:_ZNKSt7_MpunctIcE16do_positive_signEv)
                  8002222c    0000003c                           : ios.obj (.text:_ZNKSt9exception6_RaiseEv)
                  80022268    0000003c     SimpleClass.obj (.text:_ZNSo5_OsfxEv)
                  800222a4    0000003c     rtsv7A8_A_le_eabi.lib : xlocale.obj (.text:_ZNSt10moneypunctIcLb0EED1Ev)
                  800222e0    0000003c                           : xlocale.obj (.text:_ZNSt10moneypunctIcLb1EED1Ev)
                  8002231c    0000003c                           : wlocale.obj (.text:_ZNSt10moneypunctIwLb0EED1Ev)
                  80022358    0000003c                           : wlocale.obj (.text:_ZNSt10moneypunctIwLb1EED1Ev)
                  80022394    0000003c                           : string.obj (.text:_ZNSt11logic_errorD1Ev)
                  800223d0    0000003c                           : string.obj (.text:_ZNSt12length_errorD1Ev)
                  8002240c    0000003c                           : string.obj (.text:_ZNSt12out_of_rangeD1Ev)
                  80022448    0000003c                           : xlocale.obj (.text:_ZNSt7_MpunctIcED1Ev)
                  80022484    0000003c                           : wlocale.obj (.text:_ZNSt7_MpunctIwED1Ev)
                  800224c0    0000003c                           : wlocale.obj (.text:_ZNSt8numpunctIwED0Ev)
                  800224fc    0000003c                           : i_tofd32.obj (.text)
                  80022538    00000038                           : wiostrea.obj (.text:_ZNKSt5ctypeIwE5do_isEsw)
                  80022570    00000038     SimpleClass.obj (.text:_ZNSs4_EosEj)
                  800225a8    00000038     rtsv7A8_A_le_eabi.lib : iostream.obj (.text:_ZNSt15basic_streambufIcSt11char_traitsIcEE5uflowEv)
                  800225e0    00000038                           : wiostrea.obj (.text:_ZNSt15basic_streambufIwSt11char_traitsIwEE5uflowEv)
                  80022618    00000038                           : wiostrea.obj (.text:_ZNSt5ctypeIwED0Ev)
                  80022650    00000038                           : memmov.obj (.text)
                  80022688    00000038                           : xdclass.obj (.text)
                  800226c0    00000034     SimpleClass.obj (.text:_ZNKSs6_MyptrEv)
                  800226f4    00000034     SimpleClass.obj (.text:_ZNKSs8max_sizeEv)
                  80022728    00000034     rtsv7A8_A_le_eabi.lib : wiostrea.obj (.text:_ZNKSt5ctypeIwE8do_widenEc)
                  8002275c    00000034     SimpleClass.obj (.text:_ZNSs6_MyptrEv)
                  80022790    00000034     SimpleClass.obj (.text:_ZNSsC1Ev)
                  800227c4    00000034     SimpleClass.obj (.text:_ZNSt11char_traitsIcE11eq_int_typeERKiS2_)
                  800227f8    00000034     SimpleClass.obj (.text:_ZNSt6locale5facetC1Ej)
                  8002282c    00000034     rtsv7A8_A_le_eabi.lib : wlocale.obj (.text:_ZNSt8numpunctIwED1Ev)
                  80022860    00000034                           : xlocale.obj (.text:_ZNSt8time_getIcSt19istreambuf_iteratorIcSt11char_traitsIcEEED0Ev)
                  80022894    00000034                           : wlocale.obj (.text:_ZNSt8time_getIwSt19istreambuf_iteratorIwSt11char_traitsIwEEED0Ev)
                  800228c8    00000034                           : guard.obj (.text)
                  800228fc    00000034                           : memcmp.obj (.text)
                  80022930    00000030     SimpleClass.obj (.text:_ZNKSaIcE8max_sizeEv)
                  80022960    00000030     rtsv7A8_A_le_eabi.lib : wiostrea.obj (.text:_ZNKSt5ctypeIwE9do_narrowEwc)
                  80022990    00000030     SimpleClass.obj (.text:_ZNSt10ctype_baseC1Ej)
                  800229c0    00000030     SimpleClass.obj (.text:_ZNSt15basic_streambufIcSt11char_traitsIcEE5sputnEPKci)
                  800229f0    00000030     SimpleClass.obj (.text:_ZNSt19ostreambuf_iteratorIcSt11char_traitsIcEEC1EPSt15basic_streambufIcS1_E)
                  80022a20    00000030     SimpleClass.obj (.text:_ZNSt5ctypeIcED1Ev)
                  80022a50    00000030     rtsv7A8_A_le_eabi.lib : wiostrea.obj (.text:_ZNSt5ctypeIwED1Ev)
                  80022a80    00000030     SimpleClass.obj (.text:_ZNSt6localeC1ERKS_)
                  80022ab0    00000030     SimpleClass.obj (.text:_ZNSt8ios_base5widthEi)
                  80022ae0    00000030     SimpleClass.obj (.text:_ZNSt8numpunctIcE5_TidyEv)
                  80022b10    00000030     SimpleClass.obj (.text:_ZNSt8numpunctIcED1Ev)
                  80022b40    00000030     rtsv7A8_A_le_eabi.lib : wlocale.obj (.text:_ZSt10_MaklocchrIwET_cPS0_RKSt7_Cvtvec)
                  80022b70    00000030     SimpleClass.obj (.text:_ZStoRRNSt5_IosbIiE8_IostateES1_)
                  80022ba0    00000030     rtsv7A8_A_le_eabi.lib : fgetpos.obj (.text)
                  80022bd0    00000030                           : frexp.obj (.text)
                  80022c00    0000002c                           : iostream.obj (.text:_ZNSt15basic_streambufIcSt11char_traitsIcEED0Ev)
                  80022c2c    0000002c                           : wiostrea.obj (.text:_ZNSt15basic_streambufIwSt11char_traitsIwEED0Ev)
                  80022c58    0000002c                           : xlocale.obj (.text:_ZNSt8time_getIcSt19istreambuf_iteratorIcSt11char_traitsIcEEED1Ev)
                  80022c84    0000002c                           : wlocale.obj (.text:_ZNSt8time_getIwSt19istreambuf_iteratorIwSt11char_traitsIwEEED1Ev)
                  80022cb0    0000002c                           : memccpy.obj (.text)
                  80022cdc    0000002c                           : memchr.obj (.text)
                  80022d08    0000002c                           : strcat.obj (.text)
                  80022d34    00000028     SimpleClass.obj (.text:_ZNKSt5ctypeIcE5widenEc)
                  80022d5c    00000028     rtsv7A8_A_le_eabi.lib : wlocale.obj (.text:_ZNKSt7collateIwE7do_hashEPKwS2_)
                  80022d84    00000028     SimpleClass.obj (.text:_ZNKSt8ios_base4failEv)
                  80022dac    00000028     SimpleClass.obj (.text:_ZNKSt8ios_base4goodEv)
                  80022dd4    00000028     SimpleClass.obj (.text:_ZNKSt8numpunctIcE8groupingEv)
                  80022dfc    00000028     SimpleClass.obj (.text:_ZNKSt8numpunctIcE8truenameEv)
                  80022e24    00000028     SimpleClass.obj (.text:_ZNKSt8numpunctIcE9falsenameEv)
                  80022e4c    00000028     SimpleClass.obj (.text:_ZNSs6assignEPKc)
                  80022e74    00000028     SimpleClass.obj (.text:_ZNSt10ctype_baseD0Ev)
                  80022e9c    00000028     SimpleClass.obj (.text:_ZNSt5ctypeIcED0Ev)
                  80022ec4    00000028     SimpleClass.obj (.text:_ZNSt6locale5facetD0Ev)
                  80022eec    00000028     SimpleClass.obj (.text:_ZNSt7num_putIcSt19ostreambuf_iteratorIcSt11char_traitsIcEEED0Ev)
                  80022f14    00000028     SimpleClass.obj (.text:_ZNSt8numpunctIcED0Ev)
                  80022f3c    00000028     rtsv7A8_A_le_eabi.lib : iostream.obj (.text:_ZTv0_n12_NSiD0Ev)
                  80022f64    00000028                           : iostream.obj (.text:_ZTv0_n12_NSoD0Ev)
                  80022f8c    00000028                           : wiostrea.obj (.text:_ZTv0_n12_NSt13basic_istreamIwSt11char_traitsIwEED0Ev)
                  80022fb4    00000028                           : wiostrea.obj (.text:_ZTv0_n12_NSt13basic_ostreamIwSt11char_traitsIwEED0Ev)
                  80022fdc    00000028                           : strchr.obj (.text)
                  80023004    00000028                           : strcmp.obj (.text)
                  8002302c    00000024     SimpleClass.obj (.text:_ZNKSt5ctypeIcE10do_tolowerEc)
                  80023050    00000024     SimpleClass.obj (.text:_ZNKSt5ctypeIcE10do_toupperEc)
                  80023074    00000024     rtsv7A8_A_le_eabi.lib : xlocale.obj (.text:_ZNKSt7collateIcE7do_hashEPKcS2_)
                  80023098    00000024     SimpleClass.obj (.text:_ZNKSt8_Locinfo7_GetcvtEv)
                  800230bc    00000024     SimpleClass.obj (.text:_ZNSo6sentryD1Ev)
                  800230e0    00000024     SimpleClass.obj (.text:_ZNSs6assignERKSs)
                  80023104    00000024     SimpleClass.obj (.text:_ZNSt11char_traitsIcE4copyEPcPKcj)
                  80023128    00000024     SimpleClass.obj (.text:_ZNSt11char_traitsIcE4moveEPcPKcj)
                  8002314c    00000024     SimpleClass.obj (.text:_ZNSt11char_traitsIcE6assignEPcjc)
                  80023170    00000024     SimpleClass.obj (.text:_ZNSt11char_traitsIcE6assignERcRKc)
                  80023194    00000024     SimpleClass.obj (.text:_ZNSt15basic_streambufIcSt11char_traitsIcEE6_PnincEv)
                  800231b8    00000024     rtsv7A8_A_le_eabi.lib : iostream.obj (.text:_ZNSt15basic_streambufIcSt11char_traitsIcEED1Ev)
                  800231dc    00000024                           : wiostrea.obj (.text:_ZNSt15basic_streambufIwSt11char_traitsIwEED1Ev)
                  80023200    00000024     SimpleClass.obj (.text:_ZNSt6locale2idC1Ej)
                  80023224    00000024     rtsv7A8_A_le_eabi.lib : _lock.obj (.text)
                  80023248    00000020     SimpleClass.obj (.text:_ZNKSt8ios_base6getlocEv)
                  80023268    00000020     SimpleClass.obj (.text:_ZNKSt8numpunctIcE11do_groupingEv)
                  80023288    00000020     SimpleClass.obj (.text:_ZNKSt8numpunctIcE11do_truenameEv)
                  800232a8    00000020     SimpleClass.obj (.text:_ZNKSt8numpunctIcE12do_falsenameEv)
                  800232c8    00000020     SimpleClass.obj (.text:_ZNKSt8numpunctIcE13decimal_pointEv)
                  800232e8    00000020     SimpleClass.obj (.text:_ZNKSt8numpunctIcE13thousands_sepEv)
                  80023308    00000020     rtsv7A8_A_le_eabi.lib : iostream.obj (.text:_ZNSiD0Ev)
                  80023328    00000020                           : iostream.obj (.text:_ZNSoD0Ev)
                  80023348    00000020     SimpleClass.obj (.text:_ZNSsD1Ev)
                  80023368    00000020     SimpleClass.obj (.text:_ZNSsixEj)
                  80023388    00000020     SimpleClass.obj (.text:_ZNSt11_String_valIcSaIcEEC1ES0_)
                  800233a8    00000020     rtsv7A8_A_le_eabi.lib : wiostrea.obj (.text:_ZNSt13basic_istreamIwSt11char_traitsIwEED0Ev)
                  800233c8    00000020                           : wiostrea.obj (.text:_ZNSt13basic_ostreamIwSt11char_traitsIwEED0Ev)
                  800233e8    00000020     SimpleClass.obj (.text:_ZNSt15basic_streambufIcSt11char_traitsIcEE7pubsyncEv)
                  80023408    00000020     SimpleClass.obj (.text:_ZNSt5ctypeIcE5_InitERKSt8_Locinfo)
                  80023428    00000020     SimpleClass.obj (.text:_ZNSt7num_putIcSt19ostreambuf_iteratorIcSt11char_traitsIcEEE5_InitERKSt8_Locinfo)
                  80023448    00000020     SimpleClass.obj (.text:_ZStanNSt5_IosbIiE9_FmtflagsES1_)
                  80023468    00000020     rtsv7A8_A_le_eabi.lib : iostream.obj (.text:_ZTv0_n12_NSiD1Ev)
                  80023488    00000020                           : iostream.obj (.text:_ZTv0_n12_NSoD1Ev)
                  800234a8    00000020                           : wiostrea.obj (.text:_ZTv0_n12_NSt13basic_istreamIwSt11char_traitsIwEED1Ev)
                  800234c8    00000020                           : wiostrea.obj (.text:_ZTv0_n12_NSt13basic_ostreamIwSt11char_traitsIwEED1Ev)
                  800234e8    00000020                           : args_main.obj (.text)
                  80023508    0000001c     SimpleClass.obj (.text:_ZNKSt5ctypeIcE9do_narrowEcc)
                  80023524    0000001c     rtsv7A8_A_le_eabi.lib : iostream.obj (.text:_ZNKSt7codecvtIcciE5do_inERiPKcS3_RS3_PcS5_RS5_)
                  80023540    0000001c                           : iostream.obj (.text:_ZNKSt7codecvtIcciE6do_outERiPKcS3_RS3_PcS5_RS5_)
                  8002355c    0000001c     SimpleClass.obj (.text:_ZNSaIcE10deallocateEPcj)
                  80023578    0000001c     SimpleClass.obj (.text:_ZNSaIcE8allocateEj)
                  80023594    0000001c     SimpleClass.obj (.text:_ZNSolsEPFRSoS_E)
                  800235b0    0000001c     SimpleClass.obj (.text:_ZSt10_MaklocchrIcET_cPS0_RKSt7_Cvtvec)
                  800235cc    0000001c     SimpleClass.obj (.text:_ZSt8_ToloweriPKSt9_Ctypevec)
                  800235e8    0000001c     SimpleClass.obj (.text:_ZSt8_ToupperiPKSt9_Ctypevec)
                  80023604    0000001c     rtsv7A8_A_le_eabi.lib : strlen.obj (.text)
                  80023620    00000018     SimpleClass.obj (.text:_ZNKSo6sentrycvbEv)
                  80023638    00000018     SimpleClass.obj (.text:_ZNKSs4sizeEv)
                  80023650    00000018     rtsv7A8_A_le_eabi.lib : string.obj (.text:_ZNKSt11logic_error4whatEv)
                  80023668    00000018                           : ios.obj (.text:_ZNKSt13runtime_error4whatEv)
                  80023680    00000018     SimpleClass.obj (.text:_ZNKSt19ostreambuf_iteratorIcSt11char_traitsIcEE6failedEv)
                  80023698    00000018     SimpleClass.obj (.text:_ZNKSt5ctypeIcE8do_widenEc)
                  800236b0    00000018     SimpleClass.obj (.text:_ZNKSt8_Locinfo8_GettrueEv)
                  800236c8    00000018     SimpleClass.obj (.text:_ZNKSt8_Locinfo9_GetfalseEv)
                  800236e0    00000018     SimpleClass.obj (.text:_ZNKSt8ios_base5flagsEv)
                  800236f8    00000018     SimpleClass.obj (.text:_ZNKSt8ios_base5widthEv)
                  80023710    00000018     SimpleClass.obj (.text:_ZNKSt8ios_base7rdstateEv)
                  80023728    00000018     SimpleClass.obj (.text:_ZNKSt8ios_base9precisionEv)
                  80023740    00000018     SimpleClass.obj (.text:_ZNKSt8numpunctIcE16do_decimal_pointEv)
                  80023758    00000018     SimpleClass.obj (.text:_ZNKSt8numpunctIcE16do_thousands_sepEv)
                  80023770    00000018     SimpleClass.obj (.text:_ZNKSt9basic_iosIcSt11char_traitsIcEE3tieEv)
                  80023788    00000018     SimpleClass.obj (.text:_ZNKSt9basic_iosIcSt11char_traitsIcEE4fillEv)
                  800237a0    00000018     SimpleClass.obj (.text:_ZNKSt9basic_iosIcSt11char_traitsIcEE5rdbufEv)
                  800237b8    00000018     SimpleClass.obj (.text:_ZNSaIcEC1ERKS_)
                  800237d0    00000018     rtsv7A8_A_le_eabi.lib : iostream.obj (.text:_ZNSiD1Ev)
                  800237e8    00000018                           : iostream.obj (.text:_ZNSoD1Ev)
                  80023800    00000018     SimpleClass.obj (.text:_ZNSt10ctype_baseD1Ev)
                  80023818    00000018     SimpleClass.obj (.text:_ZNSt11char_traitsIcE11to_int_typeERKc)
                  80023830    00000018     rtsv7A8_A_le_eabi.lib : wiostrea.obj (.text:_ZNSt13basic_istreamIwSt11char_traitsIwEED1Ev)
                  80023848    00000018                           : wiostrea.obj (.text:_ZNSt13basic_ostreamIwSt11char_traitsIwEED1Ev)
                  80023860    00000018     SimpleClass.obj (.text:_ZNSt7_LockitC1Ei)
                  80023878    00000018     SimpleClass.obj (.text:_ZNSt7num_putIcSt19ostreambuf_iteratorIcSt11char_traitsIcEEED1Ev)
                  80023890    00000018     rtsv7A8_A_le_eabi.lib : iostream.obj (.text:_ZNSt9basic_iosIcSt11char_traitsIcEED0Ev)
                  800238a8    00000018                           : wiostrea.obj (.text:_ZNSt9basic_iosIwSt11char_traitsIwEED0Ev)
                  800238c0    00000018     SimpleClass.obj (.text:_ZSt9_AllocateIcEPT_jS1_)
                  800238d8    00000018     rtsv7A8_A_le_eabi.lib : strcpy.obj (.text)
                  800238f0    00000018                           : tolower.obj (.text)
                  80023908    00000018                           : toupper.obj (.text)
                  80023920    00000014     SimpleClass.obj (.text:_ZNKSs5c_strEv)
                  80023934    00000014     rtsv7A8_A_le_eabi.lib : wiostrea.obj (.text:_ZNKSt5ctypeIwE2isEsw)
                  80023948    00000014                           : wiostrea.obj (.text:_ZNKSt5ctypeIwE5widenEc)
                  8002395c    00000014                           : wiostrea.obj (.text:_ZNKSt5ctypeIwE6narrowEwc)
                  80023970    00000014                           : iostream.obj (.text:_ZNKSt7codecvtIcciE9do_lengthERKiPKcS4_j)
                  80023984    00000014                           : wlocale.obj (.text:_ZNKSt8numpunctIwE13thousands_sepEv)
                  80023998    00000014                           : wlocale.obj (.text:_ZNKSt8numpunctIwE8groupingEv)
                  800239ac    00000014                           : wlocale.obj (.text:_ZNKSt8numpunctIwE9falsenameEv)
                  800239c0    00000014     SimpleClass.obj (.text:_ZNSaIcEC1Ev)
                  800239d4    00000014     SimpleClass.obj (.text:_ZNSo12_Sentry_baseC2ERSo)
                  800239e8    00000014     SimpleClass.obj (.text:_ZNSt10ctype_baseC2Ej)
                  800239fc    00000014     SimpleClass.obj (.text:_ZNSt11_String_valIcSaIcEEC2ES0_)
                  80023a10    00000014     SimpleClass.obj (.text:_ZNSt11char_traitsIcE6lengthEPKc)
                  80023a24    00000014     SimpleClass.obj (.text:_ZNSt19ostreambuf_iteratorIcSt11char_traitsIcEEdeEv)
                  80023a38    00000014     SimpleClass.obj (.text:_ZNSt19ostreambuf_iteratorIcSt11char_traitsIcEEppEv)
                  80023a4c    00000014     SimpleClass.obj (.text:_ZNSt6locale5facetC2Ej)
                  80023a60    00000014     SimpleClass.obj (.text:_ZNSt6locale5facetD1Ev)
                  80023a74    00000014     SimpleClass.obj (.text:_ZNSt7_LockitD1Ev)
                  80023a88    00000014     rtsv7A8_A_le_eabi.lib : copy_decompress_none.obj (.text:decompress:none)
                  80023a9c    00000010                           : iostream.obj (.text:_ZNKSt7codecvtIcciE10do_unshiftERiPcS2_RS2_)
                  80023aac    00000010     SimpleClass.obj (.text:_ZNKSt8_Locinfo9_GetlconvEv)
                  80023abc    00000010     SimpleClass.obj (.text:_ZNSo12_Sentry_baseD2Ev)
                  80023acc    00000010     SimpleClass.obj (.text:_ZNSt10ctype_baseD2Ev)
                  80023adc    00000010     rtsv7A8_A_le_eabi.lib : wlocale.obj (.text:_ZNSt10money_baseD0Ev)
                  80023aec    00000010                           : iostream.obj (.text:_ZNSt12codecvt_baseD0Ev)
                  80023afc    00000010                           : wlocale.obj (.text:_ZNSt13messages_baseD0Ev)
                  80023b0c    00000010     SimpleClass.obj (.text:_ZNSt6locale5facetD2Ev)
                  80023b1c    00000010     rtsv7A8_A_le_eabi.lib : iostream.obj (.text:_ZNSt7codecvtIcciED0Ev)
                  80023b2c    00000010                           : wiostrea.obj (.text:_ZNSt7codecvtIwciED0Ev)
                  80023b3c    00000010                           : xlocale.obj (.text:_ZNSt7collateIcED0Ev)
                  80023b4c    00000010                           : wlocale.obj (.text:_ZNSt7collateIwED0Ev)
                  80023b5c    00000010                           : locale.obj (.text:_ZNSt7num_getIcSt19istreambuf_iteratorIcSt11char_traitsIcEEED0Ev)
                  80023b6c    00000010                           : wlocale.obj (.text:_ZNSt7num_getIwSt19istreambuf_iteratorIwSt11char_traitsIwEEED0Ev)
                  80023b7c    00000010                           : wlocale.obj (.text:_ZNSt7num_putIwSt19ostreambuf_iteratorIwSt11char_traitsIwEEED0Ev)
                  80023b8c    00000010                           : xlocale.obj (.text:_ZNSt8messagesIcED0Ev)
                  80023b9c    00000010                           : wlocale.obj (.text:_ZNSt8messagesIwED0Ev)
                  80023bac    00000010                           : xlocale.obj (.text:_ZNSt8time_putIcSt19ostreambuf_iteratorIcSt11char_traitsIcEEED0Ev)
                  80023bbc    00000010                           : wlocale.obj (.text:_ZNSt8time_putIwSt19ostreambuf_iteratorIwSt11char_traitsIwEEED0Ev)
                  80023bcc    00000010                           : locale.obj (.text:_ZNSt9bad_allocD0Ev)
                  80023bdc    00000010                           : ios.obj (.text:_ZNSt9exceptionD0Ev)
                  80023bec    00000010                           : xlocale.obj (.text:_ZNSt9money_getIcSt19istreambuf_iteratorIcSt11char_traitsIcEEED0Ev)
                  80023bfc    00000010                           : wlocale.obj (.text:_ZNSt9money_getIwSt19istreambuf_iteratorIwSt11char_traitsIwEEED0Ev)
                  80023c0c    00000010                           : xlocale.obj (.text:_ZNSt9money_putIcSt19ostreambuf_iteratorIcSt11char_traitsIcEEED0Ev)
                  80023c1c    00000010                           : wlocale.obj (.text:_ZNSt9money_putIwSt19ostreambuf_iteratorIwSt11char_traitsIwEEED0Ev)
                  80023c2c    00000010                           : wlocale.obj (.text:_ZNSt9time_baseD0Ev)
                  80023c3c    00000010                           : copy_zero_init.obj (.text:decompress:ZI)
                  80023c4c    00000010                           : delete.obj (.text)
                  80023c5c    0000000c                           : fsetpos.obj (.text)
                  80023c68    00000008                           : iostream.obj (.text:_ZNKSt12codecvt_base11do_encodingEv)
                  80023c70    00000008                           : iostream.obj (.text:_ZNKSt12codecvt_base13do_max_lengthEv)
                  80023c78    00000008                           : iostream.obj (.text:_ZNKSt12codecvt_base16do_always_noconvEv)
                  80023c80    00000008                           : xlocale.obj (.text:_ZNKSt7_MpunctIcE13do_neg_formatEv)
                  80023c88    00000008                           : xlocale.obj (.text:_ZNKSt7_MpunctIcE13do_pos_formatEv)
                  80023c90    00000008                           : xlocale.obj (.text:_ZNKSt7_MpunctIcE14do_frac_digitsEv)
                  80023c98    00000008                           : xlocale.obj (.text:_ZNKSt7_MpunctIcE16do_decimal_pointEv)
                  80023ca0    00000008                           : xlocale.obj (.text:_ZNKSt7_MpunctIcE16do_thousands_sepEv)
                  80023ca8    00000008                           : wlocale.obj (.text:_ZNKSt7_MpunctIwE13do_neg_formatEv)
                  80023cb0    00000008                           : wlocale.obj (.text:_ZNKSt7_MpunctIwE13do_pos_formatEv)
                  80023cb8    00000008                           : wlocale.obj (.text:_ZNKSt7_MpunctIwE14do_frac_digitsEv)
                  80023cc0    00000008                           : wlocale.obj (.text:_ZNKSt7_MpunctIwE16do_decimal_pointEv)
                  80023cc8    00000008                           : wlocale.obj (.text:_ZNKSt7_MpunctIwE16do_thousands_sepEv)
                  80023cd0    00000008                           : wiostrea.obj (.text:_ZNKSt7codecvtIwciE11do_encodingEv)
                  80023cd8    00000008                           : wiostrea.obj (.text:_ZNKSt7codecvtIwciE13do_max_lengthEv)
                  80023ce0    00000008                           : wiostrea.obj (.text:_ZNKSt7codecvtIwciE16do_always_noconvEv)
                  80023ce8    00000008                           : xlocale.obj (.text:_ZNKSt8messagesIcE7do_openERKSsRKSt6locale)
                  80023cf0    00000008                           : wlocale.obj (.text:_ZNKSt8messagesIwE7do_openERKSsRKSt6locale)
                  80023cf8    00000008                           : wlocale.obj (.text:_ZNKSt8numpunctIwE16do_decimal_pointEv)
                  80023d00    00000008                           : wlocale.obj (.text:_ZNKSt8numpunctIwE16do_thousands_sepEv)
                  80023d08    00000008                           : xlocale.obj (.text:_ZNKSt8time_getIcSt19istreambuf_iteratorIcSt11char_traitsIcEEE13do_date_orderEv)
                  80023d10    00000008                           : wlocale.obj (.text:_ZNKSt8time_getIwSt19istreambuf_iteratorIwSt11char_traitsIwEEE13do_date_orderEv)
                  80023d18    00000008                           : ios.obj (.text:_ZNKSt9exception4whatEv)
                  80023d20    00000008     SimpleClass.obj (.text:_ZNSt11char_traitsIcE3eofEv)
                  80023d28    00000008     rtsv7A8_A_le_eabi.lib : iostream.obj (.text:_ZNSt15basic_streambufIcSt11char_traitsIcEE4syncEv)
                  80023d30    00000008                           : iostream.obj (.text:_ZNSt15basic_streambufIcSt11char_traitsIcEE8overflowEi)
                  80023d38    00000008                           : iostream.obj (.text:_ZNSt15basic_streambufIcSt11char_traitsIcEE9pbackfailEi)
                  80023d40    00000008                           : iostream.obj (.text:_ZNSt15basic_streambufIcSt11char_traitsIcEE9showmanycEv)
                  80023d48    00000008                           : iostream.obj (.text:_ZNSt15basic_streambufIcSt11char_traitsIcEE9underflowEv)
                  80023d50    00000008                           : wiostrea.obj (.text:_ZNSt15basic_streambufIwSt11char_traitsIwEE4syncEv)
                  80023d58    00000008                           : wiostrea.obj (.text:_ZNSt15basic_streambufIwSt11char_traitsIwEE8overflowEi)
                  80023d60    00000008                           : wiostrea.obj (.text:_ZNSt15basic_streambufIwSt11char_traitsIwEE9pbackfailEi)
                  80023d68    00000008                           : wiostrea.obj (.text:_ZNSt15basic_streambufIwSt11char_traitsIwEE9showmanycEv)
                  80023d70    00000008                           : wiostrea.obj (.text:_ZNSt15basic_streambufIwSt11char_traitsIwEE9underflowEv)
                  80023d78    00000008                           : copy_decompress_rle.obj (.text:decompress:rle24)
                  80023d80    00000008                           : placenew.obj (.text)
                  80023d88    00000008                           : pre_init.obj (.text)
                  80023d90    00000004                           : string.obj (.text:_ZNKSt11logic_error8_DoraiseEv)
                  80023d94    00000004                           : string.obj (.text:_ZNKSt12length_error8_DoraiseEv)
                  80023d98    00000004                           : string.obj (.text:_ZNKSt12out_of_range8_DoraiseEv)
                  80023d9c    00000004                           : ios.obj (.text:_ZNKSt13runtime_error8_DoraiseEv)
                  80023da0    00000004                           : ios.obj (.text:_ZNKSt8ios_base7failure8_DoraiseEv)
                  80023da4    00000004                           : xlocale.obj (.text:_ZNKSt8messagesIcE8do_closeEi)
                  80023da8    00000004                           : wlocale.obj (.text:_ZNKSt8messagesIwE8do_closeEi)
                  80023dac    00000004                           : locale.obj (.text:_ZNKSt9bad_alloc8_DoraiseEv)
                  80023db0    00000004                           : ios.obj (.text:_ZNKSt9exception8_DoraiseEv)
                  80023db4    00000004                           : wlocale.obj (.text:_ZNSt10money_baseD1Ev)
                  80023db8    00000004                           : iostream.obj (.text:_ZNSt12codecvt_baseD1Ev)
                  80023dbc    00000004                           : wlocale.obj (.text:_ZNSt13messages_baseD1Ev)
                  80023dc0    00000004                           : iostream.obj (.text:_ZNSt15basic_streambufIcSt11char_traitsIcEE5_LockEv)
                  80023dc4    00000004                           : iostream.obj (.text:_ZNSt15basic_streambufIcSt11char_traitsIcEE5imbueERKSt6locale)
                  80023dc8    00000004                           : iostream.obj (.text:_ZNSt15basic_streambufIcSt11char_traitsIcEE6setbufEPci)
                  80023dcc    00000004                           : iostream.obj (.text:_ZNSt15basic_streambufIcSt11char_traitsIcEE7_UnlockEv)
                  80023dd0    00000004                           : wiostrea.obj (.text:_ZNSt15basic_streambufIwSt11char_traitsIwEE5_LockEv)
                  80023dd4    00000004                           : wiostrea.obj (.text:_ZNSt15basic_streambufIwSt11char_traitsIwEE5imbueERKSt6locale)
                  80023dd8    00000004                           : wiostrea.obj (.text:_ZNSt15basic_streambufIwSt11char_traitsIwEE6setbufEPwi)
                  80023ddc    00000004                           : wiostrea.obj (.text:_ZNSt15basic_streambufIwSt11char_traitsIwEE7_UnlockEv)
                  80023de0    00000004                           : iostream.obj (.text:_ZNSt7codecvtIcciED1Ev)
                  80023de4    00000004                           : wiostrea.obj (.text:_ZNSt7codecvtIwciED1Ev)
                  80023de8    00000004                           : xlocale.obj (.text:_ZNSt7collateIcED1Ev)
                  80023dec    00000004                           : wlocale.obj (.text:_ZNSt7collateIwED1Ev)
                  80023df0    00000004                           : locale.obj (.text:_ZNSt7num_getIcSt19istreambuf_iteratorIcSt11char_traitsIcEEED1Ev)
                  80023df4    00000004                           : wlocale.obj (.text:_ZNSt7num_getIwSt19istreambuf_iteratorIwSt11char_traitsIwEEED1Ev)
                  80023df8    00000004                           : wlocale.obj (.text:_ZNSt7num_putIwSt19ostreambuf_iteratorIwSt11char_traitsIwEEED1Ev)
                  80023dfc    00000004                           : xlocale.obj (.text:_ZNSt8messagesIcED1Ev)
                  80023e00    00000004                           : wlocale.obj (.text:_ZNSt8messagesIwED1Ev)
                  80023e04    00000004                           : xlocale.obj (.text:_ZNSt8time_putIcSt19ostreambuf_iteratorIcSt11char_traitsIcEEED1Ev)
                  80023e08    00000004                           : wlocale.obj (.text:_ZNSt8time_putIwSt19ostreambuf_iteratorIwSt11char_traitsIwEEED1Ev)
                  80023e0c    00000004                           : locale.obj (.text:_ZNSt9bad_allocD1Ev)
                  80023e10    00000004                           : iostream.obj (.text:_ZNSt9basic_iosIcSt11char_traitsIcEED1Ev)
                  80023e14    00000004                           : wiostrea.obj (.text:_ZNSt9basic_iosIwSt11char_traitsIwEED1Ev)
                  80023e18    00000004                           : ios.obj (.text:_ZNSt9exceptionD1Ev)
                  80023e1c    00000004                           : xlocale.obj (.text:_ZNSt9money_getIcSt19istreambuf_iteratorIcSt11char_traitsIcEEED1Ev)
                  80023e20    00000004                           : wlocale.obj (.text:_ZNSt9money_getIwSt19istreambuf_iteratorIwSt11char_traitsIwEEED1Ev)
                  80023e24    00000004                           : xlocale.obj (.text:_ZNSt9money_putIcSt19ostreambuf_iteratorIcSt11char_traitsIcEEED1Ev)
                  80023e28    00000004                           : wlocale.obj (.text:_ZNSt9money_putIwSt19ostreambuf_iteratorIwSt11char_traitsIwEEED1Ev)
                  80023e2c    00000004                           : wlocale.obj (.text:_ZNSt9time_baseD1Ev)
                  80023e30    00000004                           : i_div0.obj (.text)
                  80023e34    00000004                           : newhandler.obj (.text)
                  80023e38    00000004                           : xatexit.obj (.text)

.TI.persistent 
*          0    403028e8    00000000     UNINITIALIZED

.TI.noinit 
*          0    403030b4    00000000     UNINITIALIZED

.init_array 
*          0    40303370    0000001c     
                  40303370    00000004     SimpleClass.obj (.init_array)
                  40303374    00000004     rtsv7A8_A_le_eabi.lib : iostream.obj (.init_array)
                  40303378    00000004                           : locale.obj (.init_array)
                  4030337c    00000004                           : locale0.obj (.init_array)
                  40303380    00000004                           : wiostrea.obj (.init_array)
                  40303384    00000004                           : wlocale.obj (.init_array)
                  40303388    00000004                           : xlocale.obj (.init_array)

.cinit     0    40303390    00000128     
                  40303390    00000101     (.cinit..data.load) [load image, compression = rle]
                  40303491    00000003     --HOLE-- [fill = 0]
                  40303494    0000000c     (__TI_handler_table)
                  403034a0    00000008     (.cinit..bss.load) [load image, compression = zero_init]
                  403034a8    00000010     (__TI_cinit_table)


LINKER GENERATED COPY TABLES

__TI_cinit_table @ 403034a8 records: 2, size/record: 8, table size: 16
	.data: load addr=40303390, load size=00000101 bytes, run addr=403028e8, run size=000007cc bytes, compression=rle
	.bss: load addr=403034a0, load size=00000008 bytes, run addr=403030b4, run size=000002bc bytes, compression=zero_init


LINKER GENERATED HANDLER TABLE

__TI_handler_table @ 40303494 records: 3, size/record: 4, table size: 12
	index: 0, handler: __TI_zero_init
	index: 1, handler: __TI_decompress_rle24
	index: 2, handler: __TI_decompress_none


GLOBAL SYMBOLS: SORTED ALPHABETICALLY BY Name 

address   name                                                                                                                            
-------   ----                                                                                                                            
800201fc  C$$EXIT                                                                                                                         
8001ed9c  C$$IO$$                                                                                                                         
8000fafc  HOSTclock                                                                                                                       
8000fa94  HOSTclose                                                                                                                       
8000fa2c  HOSTgetenv                                                                                                                      
8000f98c  HOSTlseek                                                                                                                       
8000f900  HOSTopen                                                                                                                        
8000f87c  HOSTread                                                                                                                        
8000f7e4  HOSTrename                                                                                                                      
8000f784  HOSTtime                                                                                                                        
8000f720  HOSTunlink                                                                                                                      
8000f69c  HOSTwrite                                                                                                                       
40303370  SHT$$INIT_ARRAY$$Base                                                                                                           
4030338c  SHT$$INIT_ARRAY$$Limit                                                                                                          
80023e38  _Atexit                                                                                                                         
80022688  _Dclass                                                                                                                         
80009b44  _Deletegloballocale                                                                                                             
40302ec8  _Denorm                                                                                                                         
80018c78  _Dnorm                                                                                                                          
800176c0  _Dscale                                                                                                                         
8001e204  _Dunscale                                                                                                                       
40302ed8  _Eps                                                                                                                            
403030a0  _Errno                                                                                                                          
80009aec  _Fac_tidy                                                                                                                       
4030302c  _Fenv                                                                                                                           
80021f40  _Feraise                                                                                                                        
8001bcf4  _Getctyptab                                                                                                                     
80009df4  _Getgloballocale                                                                                                                
40302ee8  _Hugeval                                                                                                                        
40302ef8  _Inf                                                                                                                            
40302f08  _Nan                                                                                                                            
40302f28  _Rteps                                                                                                                          
80009ef8  _Setgloballocale                                                                                                                
40302f18  _Snan                                                                                                                           
8001e1a4  _Stodx                                                                                                                          
8001e1ec  _Stofx                                                                                                                          
8001e15c  _Stoldx                                                                                                                         
8001e158  _Stollx                                                                                                                         
8001e154  _Stolx                                                                                                                          
8001e150  _Stoullx                                                                                                                        
8001e14c  _Stoulx                                                                                                                         
40303030  _Tls_setup__Fenv                                                                                                                
40302f38  _Xbig                                                                                                                           
80023e34  _Z21__default_new_handlerv                                                                                                      
403032a0  _ZGVNSt10moneypunctIcLb0EE2idE                                                                                                  
403032a4  _ZGVNSt10moneypunctIcLb1EE2idE                                                                                                  
403032a8  _ZGVNSt10moneypunctIwLb0EE2idE                                                                                                  
403032ac  _ZGVNSt10moneypunctIwLb1EE2idE                                                                                                  
403032b0  _ZGVNSt7codecvtIcciE2idE                                                                                                        
403032b4  _ZGVNSt7collateIcE2idE                                                                                                          
403032b8  _ZGVNSt7collateIwE2idE                                                                                                          
403032bc  _ZGVNSt7num_getIcSt19istreambuf_iteratorIcSt11char_traitsIcEEE2idE                                                              
403032c0  _ZGVNSt7num_getIwSt19istreambuf_iteratorIwSt11char_traitsIwEEE2idE                                                              
403032c4  _ZGVNSt7num_putIcSt19ostreambuf_iteratorIcSt11char_traitsIcEEE2idE                                                              
403032c8  _ZGVNSt7num_putIwSt19ostreambuf_iteratorIwSt11char_traitsIwEEE2idE                                                              
403032cc  _ZGVNSt8messagesIcE2idE                                                                                                         
403032d0  _ZGVNSt8messagesIwE2idE                                                                                                         
403032d4  _ZGVNSt8numpunctIcE2idE                                                                                                         
403032d8  _ZGVNSt8numpunctIwE2idE                                                                                                         
403032dc  _ZGVNSt8time_getIcSt19istreambuf_iteratorIcSt11char_traitsIcEEE2idE                                                             
403032e0  _ZGVNSt8time_getIwSt19istreambuf_iteratorIwSt11char_traitsIwEEE2idE                                                             
403032e4  _ZGVNSt8time_putIcSt19ostreambuf_iteratorIcSt11char_traitsIcEEE2idE                                                             
403032e8  _ZGVNSt9money_getIcSt19istreambuf_iteratorIcSt11char_traitsIcEEE2idE                                                            
403032ec  _ZGVNSt9money_getIwSt19istreambuf_iteratorIwSt11char_traitsIwEEE2idE                                                            
403032f0  _ZGVNSt9money_putIcSt19ostreambuf_iteratorIcSt11char_traitsIcEEE2idE                                                            
403032f4  _ZGVNSt9money_putIwSt19ostreambuf_iteratorIwSt11char_traitsIwEEE2idE                                                            
800191c8  _ZN10__cxxabiv116__enum_type_infoD0Ev                                                                                           
800191c4  _ZN10__cxxabiv116__enum_type_infoD1Ev                                                                                           
800191c4  _ZN10__cxxabiv116__enum_type_infoD2Ev                                                                                           
800191b4  _ZN10__cxxabiv117__array_type_infoD0Ev                                                                                          
800191b0  _ZN10__cxxabiv117__array_type_infoD1Ev                                                                                          
800191b0  _ZN10__cxxabiv117__array_type_infoD2Ev                                                                                          
800191a0  _ZN10__cxxabiv117__class_type_infoD0Ev                                                                                          
8001919c  _ZN10__cxxabiv117__class_type_infoD1Ev                                                                                          
8001919c  _ZN10__cxxabiv117__class_type_infoD2Ev                                                                                          
8001918c  _ZN10__cxxabiv117__pbase_type_infoD0Ev                                                                                          
80019188  _ZN10__cxxabiv117__pbase_type_infoD1Ev                                                                                          
80019188  _ZN10__cxxabiv117__pbase_type_infoD2Ev                                                                                          
80019178  _ZN10__cxxabiv119__pointer_type_infoD0Ev                                                                                        
80019174  _ZN10__cxxabiv119__pointer_type_infoD1Ev                                                                                        
80019174  _ZN10__cxxabiv119__pointer_type_infoD2Ev                                                                                        
80019164  _ZN10__cxxabiv120__function_type_infoD0Ev                                                                                       
80019160  _ZN10__cxxabiv120__function_type_infoD1Ev                                                                                       
80019160  _ZN10__cxxabiv120__function_type_infoD2Ev                                                                                       
80019150  _ZN10__cxxabiv120__si_class_type_infoD0Ev                                                                                       
8001914c  _ZN10__cxxabiv120__si_class_type_infoD1Ev                                                                                       
8001914c  _ZN10__cxxabiv120__si_class_type_infoD2Ev                                                                                       
8001913c  _ZN10__cxxabiv121__vmi_class_type_infoD0Ev                                                                                      
80019138  _ZN10__cxxabiv121__vmi_class_type_infoD1Ev                                                                                      
80019138  _ZN10__cxxabiv121__vmi_class_type_infoD2Ev                                                                                      
80019128  _ZN10__cxxabiv123__fundamental_type_infoD0Ev                                                                                    
80019124  _ZN10__cxxabiv123__fundamental_type_infoD1Ev                                                                                    
80019124  _ZN10__cxxabiv123__fundamental_type_infoD2Ev                                                                                    
80019114  _ZN10__cxxabiv129__pointer_to_member_type_infoD0Ev                                                                              
80019110  _ZN10__cxxabiv129__pointer_to_member_type_infoD1Ev                                                                              
80019110  _ZN10__cxxabiv129__pointer_to_member_type_infoD2Ev                                                                              
80014be8  _ZN4Date3setEiii                                                                                                                
80014c64  _ZN4Date5printEv                                                                                                                
80014b68  _ZN4DateC1Eiii                                                                                                                  
80014b68  _ZN4DateC2Eiii                                                                                                                  
80022930  _ZNKSaIcE8max_sizeEv                                                                                                            
80023620  _ZNKSo6sentrycvbEv                                                                                                              
80023638  _ZNKSs4sizeEv                                                                                                                   
80023920  _ZNKSs5c_strEv                                                                                                                  
800226c0  _ZNKSs6_MyptrEv                                                                                                                 
8001f6cc  _ZNKSs7compareEjjPKcj                                                                                                           
800226f4  _ZNKSs8max_sizeEv                                                                                                               
80023650  _ZNKSt11logic_error4whatEv                                                                                                      
80023d90  _ZNKSt11logic_error8_DoraiseEv                                                                                                  
8001716c  _ZNKSt12_String_base5_XlenEv                                                                                                    
800171f0  _ZNKSt12_String_base5_XranEv                                                                                                    
80023c68  _ZNKSt12codecvt_base11do_encodingEv                                                                                             
80023c70  _ZNKSt12codecvt_base13do_max_lengthEv                                                                                           
80023c78  _ZNKSt12codecvt_base16do_always_noconvEv                                                                                        
80023d94  _ZNKSt12length_error8_DoraiseEv                                                                                                 
80023d98  _ZNKSt12out_of_range8_DoraiseEv                                                                                                 
80023668  _ZNKSt13runtime_error4whatEv                                                                                                    
80023d9c  _ZNKSt13runtime_error8_DoraiseEv                                                                                                
80021954  _ZNKSt15basic_streambufIcSt11char_traitsIcEE8_PnavailEv                                                                         
80023680  _ZNKSt19ostreambuf_iteratorIcSt11char_traitsIcEE6failedEv                                                                       
80020b88  _ZNKSt5ctypeIcE10do_tolowerEPcPKc                                                                                               
8002302c  _ZNKSt5ctypeIcE10do_tolowerEc                                                                                                   
80020be8  _ZNKSt5ctypeIcE10do_toupperEPcPKc                                                                                               
80023050  _ZNKSt5ctypeIcE10do_toupperEc                                                                                                   
80022d34  _ZNKSt5ctypeIcE5widenEc                                                                                                         
800220c4  _ZNKSt5ctypeIcE8do_widenEPKcS2_Pc                                                                                               
80023698  _ZNKSt5ctypeIcE8do_widenEc                                                                                                      
80022100  _ZNKSt5ctypeIcE9do_narrowEPKcS2_cPc                                                                                             
80023508  _ZNKSt5ctypeIcE9do_narrowEcc                                                                                                    
80021abc  _ZNKSt5ctypeIwE10do_scan_isEsPKwS2_                                                                                             
800205fc  _ZNKSt5ctypeIwE10do_tolowerEPwPKw                                                                                               
80021f84  _ZNKSt5ctypeIwE10do_tolowerEw                                                                                                   
8001ffa4  _ZNKSt5ctypeIwE10do_toupperEPwPKw                                                                                               
8002199c  _ZNKSt5ctypeIwE10do_toupperEw                                                                                                   
800216f4  _ZNKSt5ctypeIwE11do_scan_notEsPKwS2_                                                                                            
80023934  _ZNKSt5ctypeIwE2isEsw                                                                                                           
800213d4  _ZNKSt5ctypeIwE5do_isEPKwS2_Ps                                                                                                  
80022538  _ZNKSt5ctypeIwE5do_isEsw                                                                                                        
80023948  _ZNKSt5ctypeIwE5widenEc                                                                                                         
8002395c  _ZNKSt5ctypeIwE6narrowEwc                                                                                                       
80020f48  _ZNKSt5ctypeIwE8do_widenEPKcS2_Pw                                                                                               
80022728  _ZNKSt5ctypeIwE8do_widenEc                                                                                                      
80020fa4  _ZNKSt5ctypeIwE9do_narrowEPKwS2_cPc                                                                                             
80022960  _ZNKSt5ctypeIwE9do_narrowEwc                                                                                                    
8000a2f8  _ZNKSt6locale9_GetfacetEj                                                                                                       
8000a114  _ZNKSt6localeeqERKS_                                                                                                            
8002213c  _ZNKSt7_MpunctIcE11do_groupingEv                                                                                                
80023c80  _ZNKSt7_MpunctIcE13do_neg_formatEv                                                                                              
80023c88  _ZNKSt7_MpunctIcE13do_pos_formatEv                                                                                              
80022178  _ZNKSt7_MpunctIcE14do_curr_symbolEv                                                                                             
80023c90  _ZNKSt7_MpunctIcE14do_frac_digitsEv                                                                                             
80023c98  _ZNKSt7_MpunctIcE16do_decimal_pointEv                                                                                           
800221b4  _ZNKSt7_MpunctIcE16do_negative_signEv                                                                                           
800221f0  _ZNKSt7_MpunctIcE16do_positive_signEv                                                                                           
80023ca0  _ZNKSt7_MpunctIcE16do_thousands_sepEv                                                                                           
80018520  _ZNKSt7_MpunctIwE11do_groupingEv                                                                                                
80023ca8  _ZNKSt7_MpunctIwE13do_neg_formatEv                                                                                              
80023cb0  _ZNKSt7_MpunctIwE13do_pos_formatEv                                                                                              
8001a274  _ZNKSt7_MpunctIwE14do_curr_symbolEv                                                                                             
80023cb8  _ZNKSt7_MpunctIwE14do_frac_digitsEv                                                                                             
80023cc0  _ZNKSt7_MpunctIwE16do_decimal_pointEv                                                                                           
8001a388  _ZNKSt7_MpunctIwE16do_negative_signEv                                                                                           
8001a49c  _ZNKSt7_MpunctIwE16do_positive_signEv                                                                                           
80023cc8  _ZNKSt7_MpunctIwE16do_thousands_sepEv                                                                                           
80023a9c  _ZNKSt7codecvtIcciE10do_unshiftERiPcS2_RS2_                                                                                     
80023524  _ZNKSt7codecvtIcciE5do_inERiPKcS3_RS3_PcS5_RS5_                                                                                 
80023540  _ZNKSt7codecvtIcciE6do_outERiPKcS3_RS3_PcS5_RS5_                                                                                
80023970  _ZNKSt7codecvtIcciE9do_lengthERKiPKcS4_j                                                                                        
8001f8fc  _ZNKSt7codecvtIwciE10do_unshiftERiPcS2_RS2_                                                                                     
80023cd0  _ZNKSt7codecvtIwciE11do_encodingEv                                                                                              
80023cd8  _ZNKSt7codecvtIwciE13do_max_lengthEv                                                                                            
80023ce0  _ZNKSt7codecvtIwciE16do_always_noconvEv                                                                                         
8001e08c  _ZNKSt7codecvtIwciE5do_inERiPKcS3_RS3_PwS5_RS5_                                                                                 
8001d618  _ZNKSt7codecvtIwciE6do_outERiPKwS3_RS3_PcS5_RS5_                                                                                
8001fb1c  _ZNKSt7codecvtIwciE9do_lengthERKiPKcS4_j                                                                                        
80020804  _ZNKSt7collateIcE10do_compareEPKcS2_S2_S2_                                                                                      
80016b68  _ZNKSt7collateIcE12do_transformEPKcS2_                                                                                          
80023074  _ZNKSt7collateIcE7do_hashEPKcS2_                                                                                                
80020868  _ZNKSt7collateIwE10do_compareEPKwS2_S2_S2_                                                                                      
80016d70  _ZNKSt7collateIwE12do_transformEPKwS2_                                                                                          
80022d5c  _ZNKSt7collateIwE7do_hashEPKwS2_                                                                                                
8001bde4  _ZNKSt7num_getIcSt19istreambuf_iteratorIcSt11char_traitsIcEEE6do_getES3_S3_RSt8ios_baseRNSt5_IosbIiE8_IostateERPv               
80013d48  _ZNKSt7num_getIcSt19istreambuf_iteratorIcSt11char_traitsIcEEE6do_getES3_S3_RSt8ios_baseRNSt5_IosbIiE8_IostateERb                
8001c8e4  _ZNKSt7num_getIcSt19istreambuf_iteratorIcSt11char_traitsIcEEE6do_getES3_S3_RSt8ios_baseRNSt5_IosbIiE8_IostateERd                
8001c9c8  _ZNKSt7num_getIcSt19istreambuf_iteratorIcSt11char_traitsIcEEE6do_getES3_S3_RSt8ios_baseRNSt5_IosbIiE8_IostateERe                
8001ce3c  _ZNKSt7num_getIcSt19istreambuf_iteratorIcSt11char_traitsIcEEE6do_getES3_S3_RSt8ios_baseRNSt5_IosbIiE8_IostateERf                
8001ad30  _ZNKSt7num_getIcSt19istreambuf_iteratorIcSt11char_traitsIcEEE6do_getES3_S3_RSt8ios_baseRNSt5_IosbIiE8_IostateERj                
8001c544  _ZNKSt7num_getIcSt19istreambuf_iteratorIcSt11char_traitsIcEEE6do_getES3_S3_RSt8ios_baseRNSt5_IosbIiE8_IostateERl                
8001c62c  _ZNKSt7num_getIcSt19istreambuf_iteratorIcSt11char_traitsIcEEE6do_getES3_S3_RSt8ios_baseRNSt5_IosbIiE8_IostateERm                
8001a5b0  _ZNKSt7num_getIcSt19istreambuf_iteratorIcSt11char_traitsIcEEE6do_getES3_S3_RSt8ios_baseRNSt5_IosbIiE8_IostateERt                
8001bed0  _ZNKSt7num_getIcSt19istreambuf_iteratorIcSt11char_traitsIcEEE6do_getES3_S3_RSt8ios_baseRNSt5_IosbIiE8_IostateERx                
8001bfbc  _ZNKSt7num_getIcSt19istreambuf_iteratorIcSt11char_traitsIcEEE6do_getES3_S3_RSt8ios_baseRNSt5_IosbIiE8_IostateERy                
80006188  _ZNKSt7num_getIcSt19istreambuf_iteratorIcSt11char_traitsIcEEE8_GetffldEPcRS3_S6_RKSt6locale                                     
8000bda8  _ZNKSt7num_getIcSt19istreambuf_iteratorIcSt11char_traitsIcEEE8_GetifldEPcRS3_S6_NSt5_IosbIiE9_FmtflagsERKSt6locale              
8001c0a8  _ZNKSt7num_getIwSt19istreambuf_iteratorIwSt11char_traitsIwEEE6do_getES3_S3_RSt8ios_baseRNSt5_IosbIiE8_IostateERPv               
8000fb68  _ZNKSt7num_getIwSt19istreambuf_iteratorIwSt11char_traitsIwEEE6do_getES3_S3_RSt8ios_baseRNSt5_IosbIiE8_IostateERb                
8001caac  _ZNKSt7num_getIwSt19istreambuf_iteratorIwSt11char_traitsIwEEE6do_getES3_S3_RSt8ios_baseRNSt5_IosbIiE8_IostateERd                
8001cb90  _ZNKSt7num_getIwSt19istreambuf_iteratorIwSt11char_traitsIwEEE6do_getES3_S3_RSt8ios_baseRNSt5_IosbIiE8_IostateERe                
8001cf1c  _ZNKSt7num_getIwSt19istreambuf_iteratorIwSt11char_traitsIwEEE6do_getES3_S3_RSt8ios_baseRNSt5_IosbIiE8_IostateERf                
8001ae38  _ZNKSt7num_getIwSt19istreambuf_iteratorIwSt11char_traitsIwEEE6do_getES3_S3_RSt8ios_baseRNSt5_IosbIiE8_IostateERj                
8001c714  _ZNKSt7num_getIwSt19istreambuf_iteratorIwSt11char_traitsIwEEE6do_getES3_S3_RSt8ios_baseRNSt5_IosbIiE8_IostateERl                
8001c7fc  _ZNKSt7num_getIwSt19istreambuf_iteratorIwSt11char_traitsIwEEE6do_getES3_S3_RSt8ios_baseRNSt5_IosbIiE8_IostateERm                
8001a6c4  _ZNKSt7num_getIwSt19istreambuf_iteratorIwSt11char_traitsIwEEE6do_getES3_S3_RSt8ios_baseRNSt5_IosbIiE8_IostateERt                
8001c194  _ZNKSt7num_getIwSt19istreambuf_iteratorIwSt11char_traitsIwEEE6do_getES3_S3_RSt8ios_baseRNSt5_IosbIiE8_IostateERx                
8001c280  _ZNKSt7num_getIwSt19istreambuf_iteratorIwSt11char_traitsIwEEE6do_getES3_S3_RSt8ios_baseRNSt5_IosbIiE8_IostateERy                
80009038  _ZNKSt7num_getIwSt19istreambuf_iteratorIwSt11char_traitsIwEEE8_GetffldEPcRS3_S6_RKSt6locale                                     
8000e61c  _ZNKSt7num_getIwSt19istreambuf_iteratorIwSt11char_traitsIwEEE8_GetifldEPcRS3_S6_NSt5_IosbIiE9_FmtflagsERKSt6locale              
80019f24  _ZNKSt7num_putIcSt19ostreambuf_iteratorIcSt11char_traitsIcEEE11_PutgroupedES3_PKcjc                                             
800208cc  _ZNKSt7num_putIcSt19ostreambuf_iteratorIcSt11char_traitsIcEEE3putES3_RSt8ios_basecl                                             
8001fe30  _ZNKSt7num_putIcSt19ostreambuf_iteratorIcSt11char_traitsIcEEE4_PutES3_PKcj                                                      
80020590  _ZNKSt7num_putIcSt19ostreambuf_iteratorIcSt11char_traitsIcEEE4_RepES3_cj                                                        
80019820  _ZNKSt7num_putIcSt19ostreambuf_iteratorIcSt11char_traitsIcEEE5_FfmtEPccNSt5_IosbIiE9_FmtflagsE                                  
8000c4c8  _ZNKSt7num_putIcSt19ostreambuf_iteratorIcSt11char_traitsIcEEE5_FputES3_RSt8ios_basecPKcjjjj                                     
80018dd8  _ZNKSt7num_putIcSt19ostreambuf_iteratorIcSt11char_traitsIcEEE5_IfmtEPcPKcNSt5_IosbIiE9_FmtflagsE                                
80011d14  _ZNKSt7num_putIcSt19ostreambuf_iteratorIcSt11char_traitsIcEEE5_IputES3_RSt8ios_basecPcj                                         
8001f108  _ZNKSt7num_putIcSt19ostreambuf_iteratorIcSt11char_traitsIcEEE5_PutcES3_PKcj                                                     
8001e2bc  _ZNKSt7num_putIcSt19ostreambuf_iteratorIcSt11char_traitsIcEEE6do_putES3_RSt8ios_basecPKv                                        
80015c78  _ZNKSt7num_putIcSt19ostreambuf_iteratorIcSt11char_traitsIcEEE6do_putES3_RSt8ios_basecb                                          
80014dc0  _ZNKSt7num_putIcSt19ostreambuf_iteratorIcSt11char_traitsIcEEE6do_putES3_RSt8ios_basecd                                          
80015060  _ZNKSt7num_putIcSt19ostreambuf_iteratorIcSt11char_traitsIcEEE6do_putES3_RSt8ios_basece                                          
8001f2d0  _ZNKSt7num_putIcSt19ostreambuf_iteratorIcSt11char_traitsIcEEE6do_putES3_RSt8ios_basecl                                          
8001f364  _ZNKSt7num_putIcSt19ostreambuf_iteratorIcSt11char_traitsIcEEE6do_putES3_RSt8ios_basecm                                          
8001f1a0  _ZNKSt7num_putIcSt19ostreambuf_iteratorIcSt11char_traitsIcEEE6do_putES3_RSt8ios_basecx                                          
8001f238  _ZNKSt7num_putIcSt19ostreambuf_iteratorIcSt11char_traitsIcEEE6do_putES3_RSt8ios_basecy                                          
8001b340  _ZNKSt7num_putIwSt19ostreambuf_iteratorIwSt11char_traitsIwEEE11_PutgroupedES3_PKcjw                                             
80021424  _ZNKSt7num_putIwSt19ostreambuf_iteratorIwSt11char_traitsIwEEE4_RepES3_wj                                                        
800203d0  _ZNKSt7num_putIwSt19ostreambuf_iteratorIwSt11char_traitsIwEEE5_FfmtEPccNSt5_IosbIiE9_FmtflagsE                                  
8000a378  _ZNKSt7num_putIwSt19ostreambuf_iteratorIwSt11char_traitsIwEEE5_FputES3_RSt8ios_basewPKcjjjj                                     
8002001c  _ZNKSt7num_putIwSt19ostreambuf_iteratorIwSt11char_traitsIwEEE5_IfmtEPcPKcNSt5_IosbIiE9_FmtflagsE                                
800142d4  _ZNKSt7num_putIwSt19ostreambuf_iteratorIwSt11char_traitsIwEEE5_IputES3_RSt8ios_basewPcj                                         
80020094  _ZNKSt7num_putIwSt19ostreambuf_iteratorIwSt11char_traitsIwEEE5_PutcES3_PKcj                                                     
8001f48c  _ZNKSt7num_putIwSt19ostreambuf_iteratorIwSt11char_traitsIwEEE6do_putES3_RSt8ios_basewPKv                                        
80011988  _ZNKSt7num_putIwSt19ostreambuf_iteratorIwSt11char_traitsIwEEE6do_putES3_RSt8ios_basewb                                          
800160e8  _ZNKSt7num_putIwSt19ostreambuf_iteratorIwSt11char_traitsIwEEE6do_putES3_RSt8ios_basewd                                          
80016308  _ZNKSt7num_putIwSt19ostreambuf_iteratorIwSt11char_traitsIwEEE6do_putES3_RSt8ios_basewe                                          
8001f758  _ZNKSt7num_putIwSt19ostreambuf_iteratorIwSt11char_traitsIwEEE6do_putES3_RSt8ios_basewl                                          
8001f7e4  _ZNKSt7num_putIwSt19ostreambuf_iteratorIwSt11char_traitsIwEEE6do_putES3_RSt8ios_basewm                                          
8001f51c  _ZNKSt7num_putIwSt19ostreambuf_iteratorIwSt11char_traitsIwEEE6do_putES3_RSt8ios_basewx                                          
8001f5ac  _ZNKSt7num_putIwSt19ostreambuf_iteratorIwSt11char_traitsIwEEE6do_putES3_RSt8ios_basewy                                          
80023098  _ZNKSt8_Locinfo7_GetcvtEv                                                                                                       
800236b0  _ZNKSt8_Locinfo8_GettrueEv                                                                                                      
80021b00  _ZNKSt8_Locinfo9_GetctypeEv                                                                                                     
800236c8  _ZNKSt8_Locinfo9_GetfalseEv                                                                                                     
80023aac  _ZNKSt8_Locinfo9_GetlconvEv                                                                                                     
80022d84  _ZNKSt8ios_base4failEv                                                                                                          
80022dac  _ZNKSt8ios_base4goodEv                                                                                                          
800236e0  _ZNKSt8ios_base5flagsEv                                                                                                         
800236f8  _ZNKSt8ios_base5widthEv                                                                                                         
80023248  _ZNKSt8ios_base6getlocEv                                                                                                        
80023da0  _ZNKSt8ios_base7failure8_DoraiseEv                                                                                              
80023710  _ZNKSt8ios_base7rdstateEv                                                                                                       
80023728  _ZNKSt8ios_base9precisionEv                                                                                                     
8001cffc  _ZNKSt8messagesIcE6do_getEiiiRKSs                                                                                               
80023ce8  _ZNKSt8messagesIcE7do_openERKSsRKSt6locale                                                                                      
80023da4  _ZNKSt8messagesIcE8do_closeEi                                                                                                   
8001cc74  _ZNKSt8messagesIwE6do_getEiiiRKSbIwSt11char_traitsIwESaIwEE                                                                     
80023cf0  _ZNKSt8messagesIwE7do_openERKSsRKSt6locale                                                                                      
80023da8  _ZNKSt8messagesIwE8do_closeEi                                                                                                   
80023268  _ZNKSt8numpunctIcE11do_groupingEv                                                                                               
80023288  _ZNKSt8numpunctIcE11do_truenameEv                                                                                               
800232a8  _ZNKSt8numpunctIcE12do_falsenameEv                                                                                              
800232c8  _ZNKSt8numpunctIcE13decimal_pointEv                                                                                             
800232e8  _ZNKSt8numpunctIcE13thousands_sepEv                                                                                             
80023740  _ZNKSt8numpunctIcE16do_decimal_pointEv                                                                                          
80023758  _ZNKSt8numpunctIcE16do_thousands_sepEv                                                                                          
80022dd4  _ZNKSt8numpunctIcE8groupingEv                                                                                                   
80022dfc  _ZNKSt8numpunctIcE8truenameEv                                                                                                   
80022e24  _ZNKSt8numpunctIcE9falsenameEv                                                                                                  
800186a4  _ZNKSt8numpunctIwE11do_groupingEv                                                                                               
8001a7d8  _ZNKSt8numpunctIwE11do_truenameEv                                                                                               
8001a8ec  _ZNKSt8numpunctIwE12do_falsenameEv                                                                                              
80023984  _ZNKSt8numpunctIwE13thousands_sepEv                                                                                             
80023cf8  _ZNKSt8numpunctIwE16do_decimal_pointEv                                                                                          
80023d00  _ZNKSt8numpunctIwE16do_thousands_sepEv                                                                                          
80023998  _ZNKSt8numpunctIwE8groupingEv                                                                                                   
800239ac  _ZNKSt8numpunctIwE9falsenameEv                                                                                                  
8000d964  _ZNKSt8time_getIcSt19istreambuf_iteratorIcSt11char_traitsIcEEE11do_get_dateES3_S3_RSt8ios_baseRNSt5_IosbIiE8_IostateEPSt2tm     
80019474  _ZNKSt8time_getIcSt19istreambuf_iteratorIcSt11char_traitsIcEEE11do_get_timeES3_S3_RSt8ios_baseRNSt5_IosbIiE8_IostateEPSt2tm     
8001e6d4  _ZNKSt8time_getIcSt19istreambuf_iteratorIcSt11char_traitsIcEEE11do_get_yearES3_S3_RSt8ios_baseRNSt5_IosbIiE8_IostateEPSt2tm     
80023d08  _ZNKSt8time_getIcSt19istreambuf_iteratorIcSt11char_traitsIcEEE13do_date_orderEv                                                 
80020c48  _ZNKSt8time_getIcSt19istreambuf_iteratorIcSt11char_traitsIcEEE14do_get_weekdayES3_S3_RSt8ios_baseRNSt5_IosbIiE8_IostateEPSt2tm  
80020ca8  _ZNKSt8time_getIcSt19istreambuf_iteratorIcSt11char_traitsIcEEE16do_get_monthnameES3_S3_RSt8ios_baseRNSt5_IosbIiE8_IostateEPSt2tm
80012af4  _ZNKSt8time_getIcSt19istreambuf_iteratorIcSt11char_traitsIcEEE7_GetintERS3_S5_iiRi                                              
8000cbd4  _ZNKSt8time_getIwSt19istreambuf_iteratorIwSt11char_traitsIwEEE11do_get_dateES3_S3_RSt8ios_baseRNSt5_IosbIiE8_IostateEPSt2tm     
800189a8  _ZNKSt8time_getIwSt19istreambuf_iteratorIwSt11char_traitsIwEEE11do_get_timeES3_S3_RSt8ios_baseRNSt5_IosbIiE8_IostateEPSt2tm     
8001e77c  _ZNKSt8time_getIwSt19istreambuf_iteratorIwSt11char_traitsIwEEE11do_get_yearES3_S3_RSt8ios_baseRNSt5_IosbIiE8_IostateEPSt2tm     
80023d10  _ZNKSt8time_getIwSt19istreambuf_iteratorIwSt11char_traitsIwEEE13do_date_orderEv                                                 
80020d08  _ZNKSt8time_getIwSt19istreambuf_iteratorIwSt11char_traitsIwEEE14do_get_weekdayES3_S3_RSt8ios_baseRNSt5_IosbIiE8_IostateEPSt2tm  
80020d68  _ZNKSt8time_getIwSt19istreambuf_iteratorIwSt11char_traitsIwEEE16do_get_monthnameES3_S3_RSt8ios_baseRNSt5_IosbIiE8_IostateEPSt2tm
8000ffbc  _ZNKSt8time_getIwSt19istreambuf_iteratorIwSt11char_traitsIwEEE7_GetintERS3_S5_iiRi                                              
80016528  _ZNKSt8time_putIcSt19ostreambuf_iteratorIcSt11char_traitsIcEEE6do_putES3_RSt8ios_basecPKSt2tmcc                                 
80014010  _ZNKSt8time_putIwSt19ostreambuf_iteratorIwSt11char_traitsIwEEE6do_putES3_RSt8ios_basewPKSt2tmcc                                 
80023dac  _ZNKSt9bad_alloc8_DoraiseEv                                                                                                     
80023770  _ZNKSt9basic_iosIcSt11char_traitsIcEE3tieEv                                                                                     
80023788  _ZNKSt9basic_iosIcSt11char_traitsIcEE4fillEv                                                                                    
800237a0  _ZNKSt9basic_iosIcSt11char_traitsIcEE5rdbufEv                                                                                   
80021474  _ZNKSt9basic_iosIcSt11char_traitsIcEE5widenEc                                                                                   
80023d18  _ZNKSt9exception4whatEv                                                                                                         
8002222c  _ZNKSt9exception6_RaiseEv                                                                                                       
80023db0  _ZNKSt9exception8_DoraiseEv                                                                                                     
80017d40  _ZNKSt9money_getIcSt19istreambuf_iteratorIcSt11char_traitsIcEEE6do_getES3_S3_bRSt8ios_baseRNSt5_IosbIiE8_IostateERSs            
80015eb4  _ZNKSt9money_getIcSt19istreambuf_iteratorIcSt11char_traitsIcEEE6do_getES3_S3_bRSt8ios_baseRNSt5_IosbIiE8_IostateERe             
8000322c  _ZNKSt9money_getIcSt19istreambuf_iteratorIcSt11char_traitsIcEEE8_GetmfldERS3_S5_bRSt8ios_base                                   
80017a08  _ZNKSt9money_getIwSt19istreambuf_iteratorIwSt11char_traitsIwEEE6do_getES3_S3_bRSt8ios_baseRNSt5_IosbIiE8_IostateERSbIwS2_SaIwEE 
80010768  _ZNKSt9money_getIwSt19istreambuf_iteratorIwSt11char_traitsIwEEE6do_getES3_S3_bRSt8ios_baseRNSt5_IosbIiE8_IostateERe             
800051e0  _ZNKSt9money_getIwSt19istreambuf_iteratorIwSt11char_traitsIwEEE8_GetmfldERS3_S5_bRSt8ios_base                                   
80015598  _ZNKSt9money_putIcSt19ostreambuf_iteratorIcSt11char_traitsIcEEE6do_putES3_bRSt8ios_basecRKSs                                    
8001278c  _ZNKSt9money_putIcSt19ostreambuf_iteratorIcSt11char_traitsIcEEE6do_putES3_bRSt8ios_basece                                       
80007a44  _ZNKSt9money_putIcSt19ostreambuf_iteratorIcSt11char_traitsIcEEE8_PutmfldES3_bRSt8ios_basecbSs                                   
80010eb0  _ZNKSt9money_putIwSt19ostreambuf_iteratorIwSt11char_traitsIwEEE6do_putES3_bRSt8ios_basewRKSbIwS2_SaIwEE                         
800103a0  _ZNKSt9money_putIwSt19ostreambuf_iteratorIwSt11char_traitsIwEEE6do_putES3_bRSt8ios_basewe                                       
80006e40  _ZNKSt9money_putIwSt19ostreambuf_iteratorIwSt11char_traitsIwEEE8_PutmfldES3_bRSt8ios_basewbSbIwS2_SaIwEE                        
800190b0  _ZNKSt9type_info4nameEv                                                                                                         
800190f8  _ZNKSt9type_info6beforeERKS_                                                                                                    
800190d8  _ZNKSt9type_infoeqERKS_                                                                                                         
800190b8  _ZNKSt9type_infoneERKS_                                                                                                         
8002355c  _ZNSaIcE10deallocateEPcj                                                                                                        
80023578  _ZNSaIcE8allocateEj                                                                                                             
800237b8  _ZNSaIcEC1ERKS_                                                                                                                 
800239c0  _ZNSaIcEC1Ev                                                                                                                    
8001dd6c  _ZNSbIwSt11char_traitsIwESaIwEE5_CopyEjj                                                                                        
8001ee98  _ZNSbIwSt11char_traitsIwESaIwEE5eraseEjj                                                                                        
8001d89c  _ZNSbIwSt11char_traitsIwESaIwEE6appendEjw                                                                                       
8001ac24  _ZNSbIwSt11char_traitsIwESaIwEE6assignERKS2_jj                                                                                  
8001a040  _ZNSbIwSt11char_traitsIwESaIwEE6insertEjjw                                                                                      
80021fc4  _ZNSbIwSt11char_traitsIwESaIwEE9_ChassignEjjw                                                                                   
80023308  _ZNSiD0Ev                                                                                                                       
800237d0  _ZNSiD1Ev                                                                                                                       
8001e57c  _ZNSo12_Sentry_baseC1ERSo                                                                                                       
800239d4  _ZNSo12_Sentry_baseC2ERSo                                                                                                       
8001ef34  _ZNSo12_Sentry_baseD1Ev                                                                                                         
80023abc  _ZNSo12_Sentry_baseD2Ev                                                                                                         
8001da3c  _ZNSo3putEc                                                                                                                     
80022268  _ZNSo5_OsfxEv                                                                                                                   
8001f984  _ZNSo5flushEv                                                                                                                   
8001c36c  _ZNSo6sentryC1ERSo                                                                                                              
800230bc  _ZNSo6sentryD1Ev                                                                                                                
80023328  _ZNSoD0Ev                                                                                                                       
800237e8  _ZNSoD1Ev                                                                                                                       
80023594  _ZNSolsEPFRSoS_E                                                                                                                
80017ed8  _ZNSolsEi                                                                                                                       
80022570  _ZNSs4_EosEj                                                                                                                    
8001ab14  _ZNSs5_CopyEjj                                                                                                                  
8001d7c8  _ZNSs5_GrowEjb                                                                                                                  
8001f3f8  _ZNSs5_TidyEbj                                                                                                                  
8001cd58  _ZNSs5eraseEjj                                                                                                                  
8002275c  _ZNSs6_MyptrEv                                                                                                                  
8001d53c  _ZNSs6appendEPKcj                                                                                                               
8001af40  _ZNSs6appendERKSsjj                                                                                                             
8001efd0  _ZNSs6appendEjc                                                                                                                 
80022e4c  _ZNSs6assignEPKc                                                                                                                
8001fa0c  _ZNSs6assignEPKcj                                                                                                               
800230e0  _ZNSs6assignERKSs                                                                                                               
8001ba20  _ZNSs6assignERKSsjj                                                                                                             
8001b43c  _ZNSs6insertEjjc                                                                                                                
800214c4  _ZNSs7_InsideEPKc                                                                                                               
80020930  _ZNSs9_ChassignEjjc                                                                                                             
80021b44  _ZNSsC1EPKc                                                                                                                     
80022790  _ZNSsC1Ev                                                                                                                       
80023348  _ZNSsD1Ev                                                                                                                       
80023368  _ZNSsixEj                                                                                                                       
80022990  _ZNSt10ctype_baseC1Ej                                                                                                           
800239e8  _ZNSt10ctype_baseC2Ej                                                                                                           
80022e74  _ZNSt10ctype_baseD0Ev                                                                                                           
80023800  _ZNSt10ctype_baseD1Ev                                                                                                           
80023acc  _ZNSt10ctype_baseD2Ev                                                                                                           
80023adc  _ZNSt10money_baseD0Ev                                                                                                           
80023db4  _ZNSt10money_baseD1Ev                                                                                                           
403032f8  _ZNSt10moneypunctIcLb0EE2idE                                                                                                    
80021b88  _ZNSt10moneypunctIcLb0EED0Ev                                                                                                    
800222a4  _ZNSt10moneypunctIcLb0EED1Ev                                                                                                    
403032fc  _ZNSt10moneypunctIcLb1EE2idE                                                                                                    
80021bcc  _ZNSt10moneypunctIcLb1EED0Ev                                                                                                    
800222e0  _ZNSt10moneypunctIcLb1EED1Ev                                                                                                    
40303300  _ZNSt10moneypunctIwLb0EE2idE                                                                                                    
80021c10  _ZNSt10moneypunctIwLb0EED0Ev                                                                                                    
8002231c  _ZNSt10moneypunctIwLb0EED1Ev                                                                                                    
40303304  _ZNSt10moneypunctIwLb1EE2idE                                                                                                    
80021c54  _ZNSt10moneypunctIwLb1EED0Ev                                                                                                    
80022358  _ZNSt10moneypunctIwLb1EED1Ev                                                                                                    
80023388  _ZNSt11_String_valIcSaIcEEC1ES0_                                                                                                
800239fc  _ZNSt11_String_valIcSaIcEEC2ES0_                                                                                                
800227c4  _ZNSt11char_traitsIcE11eq_int_typeERKiS2_                                                                                       
80023818  _ZNSt11char_traitsIcE11to_int_typeERKc                                                                                          
80023d20  _ZNSt11char_traitsIcE3eofEv                                                                                                     
80023104  _ZNSt11char_traitsIcE4copyEPcPKcj                                                                                               
80023128  _ZNSt11char_traitsIcE4moveEPcPKcj                                                                                               
8002314c  _ZNSt11char_traitsIcE6assignEPcjc                                                                                               
80023170  _ZNSt11char_traitsIcE6assignERcRKc                                                                                              
80023a10  _ZNSt11char_traitsIcE6lengthEPKc                                                                                                
80020664  _ZNSt11logic_errorC2ERKSs                                                                                                       
80021c98  _ZNSt11logic_errorD0Ev                                                                                                          
80022394  _ZNSt11logic_errorD1Ev                                                                                                          
80023aec  _ZNSt12codecvt_baseD0Ev                                                                                                         
80023db8  _ZNSt12codecvt_baseD1Ev                                                                                                         
80021cdc  _ZNSt12length_errorD0Ev                                                                                                         
800223d0  _ZNSt12length_errorD1Ev                                                                                                         
80020274  _ZNSt12out_of_rangeC1ERKSs                                                                                                      
80021d20  _ZNSt12out_of_rangeD0Ev                                                                                                         
8002240c  _ZNSt12out_of_rangeD1Ev                                                                                                         
80021740  _ZNSt13basic_filebufIcSt11char_traitsIcEE4syncEv                                                                                
8001932c  _ZNSt13basic_filebufIcSt11char_traitsIcEE5imbueERKSt6locale                                                                     
8001209c  _ZNSt13basic_filebufIcSt11char_traitsIcEE5uflowEv                                                                               
8001e824  _ZNSt13basic_filebufIcSt11char_traitsIcEE6setbufEPci                                                                            
40303308  _ZNSt13basic_filebufIcSt11char_traitsIcEE7_StinitE                                                                              
800195b8  _ZNSt13basic_filebufIcSt11char_traitsIcEE7seekoffElNSt5_IosbIiE8_SeekdirENS4_9_OpenmodeE                                        
80019bac  _ZNSt13basic_filebufIcSt11char_traitsIcEE7seekposESt4fposIiENSt5_IosbIiE9_OpenmodeE                                             
800115f0  _ZNSt13basic_filebufIcSt11char_traitsIcEE8overflowEi                                                                            
80013198  _ZNSt13basic_filebufIcSt11char_traitsIcEE9_EndwriteEv                                                                           
8001de34  _ZNSt13basic_filebufIcSt11char_traitsIcEE9pbackfailEi                                                                           
800206cc  _ZNSt13basic_filebufIcSt11char_traitsIcEE9underflowEv                                                                           
8001f870  _ZNSt13basic_filebufIcSt11char_traitsIcEED0Ev                                                                                   
8001fba0  _ZNSt13basic_filebufIcSt11char_traitsIcEED1Ev                                                                                   
8002178c  _ZNSt13basic_filebufIwSt11char_traitsIwEE4syncEv                                                                                
800191e0  _ZNSt13basic_filebufIwSt11char_traitsIwEE5imbueERKSt6locale                                                                     
80012414  _ZNSt13basic_filebufIwSt11char_traitsIwEE5uflowEv                                                                               
8001d96c  _ZNSt13basic_filebufIwSt11char_traitsIwEE6setbufEPwi                                                                            
4030330c  _ZNSt13basic_filebufIwSt11char_traitsIwEE7_StinitE                                                                              
800196ec  _ZNSt13basic_filebufIwSt11char_traitsIwEE7seekoffElNSt5_IosbIiE8_SeekdirENS4_9_OpenmodeE                                        
80019cd4  _ZNSt13basic_filebufIwSt11char_traitsIwEE7seekposESt4fposIiENSt5_IosbIiE9_OpenmodeE                                             
80010b0c  _ZNSt13basic_filebufIwSt11char_traitsIwEE8overflowEi                                                                            
80013494  _ZNSt13basic_filebufIwSt11char_traitsIwEE9_EndwriteEv                                                                           
8001defc  _ZNSt13basic_filebufIwSt11char_traitsIwEE9pbackfailEi                                                                           
80020734  _ZNSt13basic_filebufIwSt11char_traitsIwEE9underflowEv                                                                           
8001d0dc  _ZNSt13basic_filebufIwSt11char_traitsIwEED0Ev                                                                                   
8001d6f0  _ZNSt13basic_filebufIwSt11char_traitsIwEED1Ev                                                                                   
800233a8  _ZNSt13basic_istreamIwSt11char_traitsIwEED0Ev                                                                                   
80023830  _ZNSt13basic_istreamIwSt11char_traitsIwEED1Ev                                                                                   
800233c8  _ZNSt13basic_ostreamIwSt11char_traitsIwEED0Ev                                                                                   
80023848  _ZNSt13basic_ostreamIwSt11char_traitsIwEED1Ev                                                                                   
80023afc  _ZNSt13messages_baseD0Ev                                                                                                        
80023dbc  _ZNSt13messages_baseD1Ev                                                                                                        
80021514  _ZNSt13runtime_errorD0Ev                                                                                                        
80021d64  _ZNSt13runtime_errorD1Ev                                                                                                        
80023d28  _ZNSt15basic_streambufIcSt11char_traitsIcEE4syncEv                                                                              
80020dc8  _ZNSt15basic_streambufIcSt11char_traitsIcEE5_InitEv                                                                             
80023dc0  _ZNSt15basic_streambufIcSt11char_traitsIcEE5_LockEv                                                                             
80023dc4  _ZNSt15basic_streambufIcSt11char_traitsIcEE5imbueERKSt6locale                                                                   
80020e28  _ZNSt15basic_streambufIcSt11char_traitsIcEE5sputcEc                                                                             
800229c0  _ZNSt15basic_streambufIcSt11char_traitsIcEE5sputnEPKci                                                                          
800225a8  _ZNSt15basic_streambufIcSt11char_traitsIcEE5uflowEv                                                                             
80023194  _ZNSt15basic_streambufIcSt11char_traitsIcEE6_PnincEv                                                                            
80023dc8  _ZNSt15basic_streambufIcSt11char_traitsIcEE6setbufEPci                                                                          
8001eac4  _ZNSt15basic_streambufIcSt11char_traitsIcEE6xsgetnEPci                                                                          
8001e8cc  _ZNSt15basic_streambufIcSt11char_traitsIcEE6xsputnEPKci                                                                         
80023dcc  _ZNSt15basic_streambufIcSt11char_traitsIcEE7_UnlockEv                                                                           
800233e8  _ZNSt15basic_streambufIcSt11char_traitsIcEE7pubsyncEv                                                                           
80021da8  _ZNSt15basic_streambufIcSt11char_traitsIcEE7seekoffElNSt5_IosbIiE8_SeekdirENS4_9_OpenmodeE                                      
800217d8  _ZNSt15basic_streambufIcSt11char_traitsIcEE7seekposESt4fposIiENSt5_IosbIiE9_OpenmodeE                                           
80023d30  _ZNSt15basic_streambufIcSt11char_traitsIcEE8overflowEi                                                                          
80023d38  _ZNSt15basic_streambufIcSt11char_traitsIcEE9pbackfailEi                                                                         
80023d40  _ZNSt15basic_streambufIcSt11char_traitsIcEE9showmanycEv                                                                         
80023d48  _ZNSt15basic_streambufIcSt11char_traitsIcEE9underflowEv                                                                         
80022c00  _ZNSt15basic_streambufIcSt11char_traitsIcEED0Ev                                                                                 
800231b8  _ZNSt15basic_streambufIcSt11char_traitsIcEED1Ev                                                                                 
80023d50  _ZNSt15basic_streambufIwSt11char_traitsIwEE4syncEv                                                                              
80023dd0  _ZNSt15basic_streambufIwSt11char_traitsIwEE5_LockEv                                                                             
80023dd4  _ZNSt15basic_streambufIwSt11char_traitsIwEE5imbueERKSt6locale                                                                   
800225e0  _ZNSt15basic_streambufIwSt11char_traitsIwEE5uflowEv                                                                             
80023dd8  _ZNSt15basic_streambufIwSt11char_traitsIwEE6setbufEPwi                                                                          
8001e628  _ZNSt15basic_streambufIwSt11char_traitsIwEE6xsgetnEPwi                                                                          
8001e36c  _ZNSt15basic_streambufIwSt11char_traitsIwEE6xsputnEPKwi                                                                         
80023ddc  _ZNSt15basic_streambufIwSt11char_traitsIwEE7_UnlockEv                                                                           
80021dec  _ZNSt15basic_streambufIwSt11char_traitsIwEE7seekoffElNSt5_IosbIiE8_SeekdirENS4_9_OpenmodeE                                      
80021824  _ZNSt15basic_streambufIwSt11char_traitsIwEE7seekposESt4fposIiENSt5_IosbIiE9_OpenmodeE                                           
80023d58  _ZNSt15basic_streambufIwSt11char_traitsIwEE8overflowEi                                                                          
80023d60  _ZNSt15basic_streambufIwSt11char_traitsIwEE9pbackfailEi                                                                         
80023d68  _ZNSt15basic_streambufIwSt11char_traitsIwEE9showmanycEv                                                                         
80023d70  _ZNSt15basic_streambufIwSt11char_traitsIwEE9underflowEv                                                                         
80022c2c  _ZNSt15basic_streambufIwSt11char_traitsIwEED0Ev                                                                                 
800231dc  _ZNSt15basic_streambufIwSt11char_traitsIwEED1Ev                                                                                 
8002010c  _ZNSt19istreambuf_iteratorIcSt11char_traitsIcEE5_PeekEv                                                                         
8001feac  _ZNSt19istreambuf_iteratorIcSt11char_traitsIcEEppEv                                                                             
80020184  _ZNSt19istreambuf_iteratorIwSt11char_traitsIwEE5_PeekEv                                                                         
8001ff28  _ZNSt19istreambuf_iteratorIwSt11char_traitsIwEEppEv                                                                             
800229f0  _ZNSt19ostreambuf_iteratorIcSt11char_traitsIcEEC1EPSt15basic_streambufIcS1_E                                                    
80020440  _ZNSt19ostreambuf_iteratorIcSt11char_traitsIcEEaSEc                                                                             
80023a24  _ZNSt19ostreambuf_iteratorIcSt11char_traitsIcEEdeEv                                                                             
80023a38  _ZNSt19ostreambuf_iteratorIcSt11char_traitsIcEEppEv                                                                             
800202e8  _ZNSt19ostreambuf_iteratorIwSt11char_traitsIwEEaSEw                                                                             
40303310  _ZNSt4fposIiE4_StzE                                                                                                             
40302fe0  _ZNSt5ctypeIcE2idE                                                                                                              
80023408  _ZNSt5ctypeIcE5_InitERKSt8_Locinfo                                                                                              
800219e4  _ZNSt5ctypeIcE5_TidyEv                                                                                                          
80020994  _ZNSt5ctypeIcE7_GetcatEPPKNSt6locale5facetE                                                                                     
8001eb68  _ZNSt5ctypeIcEC1EPKsbj                                                                                                          
80022e9c  _ZNSt5ctypeIcED0Ev                                                                                                              
80022a20  _ZNSt5ctypeIcED1Ev                                                                                                              
40303360  _ZNSt5ctypeIwE2idE                                                                                                              
80022618  _ZNSt5ctypeIwED0Ev                                                                                                              
80022a50  _ZNSt5ctypeIwED1Ev                                                                                                              
40302aa0  _ZNSt6_Winit9_Init_cntE                                                                                                         
8000b6b8  _ZNSt6_WinitC1Ev                                                                                                                
8000b6b8  _ZNSt6_WinitC2Ev                                                                                                                
8000b558  _ZNSt6_WinitD1Ev                                                                                                                
8000b558  _ZNSt6_WinitD2Ev                                                                                                                
40302fd0  _ZNSt6locale2id7_Id_cntE                                                                                                        
80023200  _ZNSt6locale2idC1Ej                                                                                                             
800209f8  _ZNSt6locale2idcvjEv                                                                                                            
80009f28  _ZNSt6locale5_InitEv                                                                                                            
8000a0dc  _ZNSt6locale5emptyEv                                                                                                            
8002035c  _ZNSt6locale5facet7_DecrefEv                                                                                                    
80022004  _ZNSt6locale5facet7_IncrefEv                                                                                                    
8000a098  _ZNSt6locale5facet9_RegisterEv                                                                                                  
800227f8  _ZNSt6locale5facetC1Ej                                                                                                          
80023a4c  _ZNSt6locale5facetC2Ej                                                                                                          
80022ec4  _ZNSt6locale5facetD0Ev                                                                                                          
80023a60  _ZNSt6locale5facetD1Ev                                                                                                          
80023b0c  _ZNSt6locale5facetD2Ev                                                                                                          
800030cc  _ZNSt6locale6globalERKS_                                                                                                        
80002f84  _ZNSt6locale7_AddfacEPNS_5facetEjj                                                                                              
80001f70  _ZNSt6locale7_Locimp7_AddfacEPNS_5facetEj                                                                                       
40302fd8  _ZNSt6locale7_Locimp8_ClocptrE                                                                                                  
800020b0  _ZNSt6locale7_Locimp8_MakelocERKSt8_LocinfoiPS0_PKS_                                                                            
8000440c  _ZNSt6locale7_Locimp9_MakewlocERKSt8_LocinfoiPS0_PKS_                                                                           
80008758  _ZNSt6locale7_Locimp9_MakexlocERKSt8_LocinfoiPS0_PKS_                                                                           
800026e8  _ZNSt6locale7_LocimpC1ERKS0_                                                                                                    
80009e00  _ZNSt6locale7_LocimpC1Eb                                                                                                        
800026e8  _ZNSt6locale7_LocimpC2ERKS0_                                                                                                    
80009e00  _ZNSt6locale7_LocimpC2Eb                                                                                                        
80009ad4  _ZNSt6locale7_LocimpD0Ev                                                                                                        
80009a1c  _ZNSt6locale7_LocimpD1Ev                                                                                                        
80009a1c  _ZNSt6locale7_LocimpD2Ev                                                                                                        
8000a088  _ZNSt6locale7classicEv                                                                                                          
80002cc0  _ZNSt6localeC1EPKci                                                                                                             
80022a80  _ZNSt6localeC1ERKS_                                                                                                             
8000292c  _ZNSt6localeC1ERKS_PKci                                                                                                         
80002860  _ZNSt6localeC1ERKS_S1_i                                                                                                         
8000a054  _ZNSt6localeC1Ev                                                                                                                
80002cc0  _ZNSt6localeC2EPKci                                                                                                             
8000292c  _ZNSt6localeC2ERKS_PKci                                                                                                         
80002860  _ZNSt6localeC2ERKS_S1_i                                                                                                         
8000a054  _ZNSt6localeC2Ev                                                                                                                
80021870  _ZNSt6localeD1Ev                                                                                                                
800212d8  _ZNSt6localeaSERKS_                                                                                                             
80023860  _ZNSt7_LockitC1Ei                                                                                                               
80023a74  _ZNSt7_LockitD1Ev                                                                                                               
80018b18  _ZNSt7_MpunctIcE5_InitERKSt8_Locinfo                                                                                            
80020e88  _ZNSt7_MpunctIcE7_MakpatERNSt10money_base7patternEjjj                                                                           
80021e30  _ZNSt7_MpunctIcED0Ev                                                                                                            
80022448  _ZNSt7_MpunctIcED1Ev                                                                                                            
80018200  _ZNSt7_MpunctIwE5_InitERKSt8_Locinfo                                                                                            
80020ee8  _ZNSt7_MpunctIwE7_MakpatERNSt10money_base7patternEjjj                                                                           
80021e74  _ZNSt7_MpunctIwED0Ev                                                                                                            
80022484  _ZNSt7_MpunctIwED1Ev                                                                                                            
40303314  _ZNSt7codecvtIcciE2idE                                                                                                          
80023b1c  _ZNSt7codecvtIcciED0Ev                                                                                                          
80023de0  _ZNSt7codecvtIcciED1Ev                                                                                                          
40302fdc  _ZNSt7codecvtIwciE2idE                                                                                                          
80023b2c  _ZNSt7codecvtIwciED0Ev                                                                                                          
80023de4  _ZNSt7codecvtIwciED1Ev                                                                                                          
40303318  _ZNSt7collateIcE2idE                                                                                                            
80023b3c  _ZNSt7collateIcED0Ev                                                                                                            
80023de8  _ZNSt7collateIcED1Ev                                                                                                            
4030331c  _ZNSt7collateIwE2idE                                                                                                            
80023b4c  _ZNSt7collateIwED0Ev                                                                                                            
80023dec  _ZNSt7collateIwED1Ev                                                                                                            
40303320  _ZNSt7num_getIcSt19istreambuf_iteratorIcSt11char_traitsIcEEE2idE                                                                
80023b5c  _ZNSt7num_getIcSt19istreambuf_iteratorIcSt11char_traitsIcEEED0Ev                                                                
80023df0  _ZNSt7num_getIcSt19istreambuf_iteratorIcSt11char_traitsIcEEED1Ev                                                                
40303324  _ZNSt7num_getIwSt19istreambuf_iteratorIwSt11char_traitsIwEEE2idE                                                                
80023b6c  _ZNSt7num_getIwSt19istreambuf_iteratorIwSt11char_traitsIwEEED0Ev                                                                
80023df4  _ZNSt7num_getIwSt19istreambuf_iteratorIwSt11char_traitsIwEEED1Ev                                                                
40303328  _ZNSt7num_putIcSt19ostreambuf_iteratorIcSt11char_traitsIcEEE2idE                                                                
80023428  _ZNSt7num_putIcSt19ostreambuf_iteratorIcSt11char_traitsIcEEE5_InitERKSt8_Locinfo                                                
80021000  _ZNSt7num_putIcSt19ostreambuf_iteratorIcSt11char_traitsIcEEE7_GetcatEPPKNSt6locale5facetE                                       
8002105c  _ZNSt7num_putIcSt19ostreambuf_iteratorIcSt11char_traitsIcEEEC1Ej                                                                
80022eec  _ZNSt7num_putIcSt19ostreambuf_iteratorIcSt11char_traitsIcEEED0Ev                                                                
80023878  _ZNSt7num_putIcSt19ostreambuf_iteratorIcSt11char_traitsIcEEED1Ev                                                                
4030332c  _ZNSt7num_putIwSt19ostreambuf_iteratorIwSt11char_traitsIwEEE2idE                                                                
80023b7c  _ZNSt7num_putIwSt19ostreambuf_iteratorIwSt11char_traitsIwEEED0Ev                                                                
80023df8  _ZNSt7num_putIwSt19ostreambuf_iteratorIwSt11char_traitsIwEEED1Ev                                                                
80001b48  _ZNSt8_Locinfo8_AddcatsEiPKc                                                                                                    
80009c04  _ZNSt8_LocinfoC1EPKc                                                                                                            
80001dec  _ZNSt8_LocinfoC1EiPKc                                                                                                           
80009c04  _ZNSt8_LocinfoC2EPKc                                                                                                            
80001dec  _ZNSt8_LocinfoC2EiPKc                                                                                                           
80009b78  _ZNSt8_LocinfoD1Ev                                                                                                              
80009b78  _ZNSt8_LocinfoD2Ev                                                                                                              
8000b29c  _ZNSt8ios_base17register_callbackEPFvNS_5eventERS_iEi                                                                           
403028e8  _ZNSt8ios_base4Init9_Init_cntE                                                                                                  
8000d56c  _ZNSt8ios_base4InitC1Ev                                                                                                         
8000d56c  _ZNSt8ios_base4InitC2Ev                                                                                                         
8000d474  _ZNSt8ios_base4InitD1Ev                                                                                                         
8000d474  _ZNSt8ios_base4InitD2Ev                                                                                                         
8000b4e8  _ZNSt8ios_base5_InitEv                                                                                                          
40302f4c  _ZNSt8ios_base5_SyncE                                                                                                           
8000acd0  _ZNSt8ios_base5_TidyEv                                                                                                          
8000ad88  _ZNSt8ios_base5clearENSt5_IosbIiE8_IostateEb                                                                                    
8000b480  _ZNSt8ios_base5imbueERKSt6locale                                                                                                
80022ab0  _ZNSt8ios_base5widthEi                                                                                                          
40302f48  _ZNSt8ios_base6_IndexE                                                                                                          
8000b438  _ZNSt8ios_base7_AddstdEv                                                                                                        
8000b2ec  _ZNSt8ios_base7copyfmtERKS_                                                                                                     
80021564  _ZNSt8ios_base7failureD0Ev                                                                                                      
80021eb8  _ZNSt8ios_base7failureD1Ev                                                                                                      
8000ac98  _ZNSt8ios_base8_CallfnsENS_5eventE                                                                                              
8000b1a8  _ZNSt8ios_base8_FindarrEi                                                                                                       
8000ac80  _ZNSt8ios_baseD0Ev                                                                                                              
8000ad28  _ZNSt8ios_baseD1Ev                                                                                                              
8000ad28  _ZNSt8ios_baseD2Ev                                                                                                              
40303330  _ZNSt8messagesIcE2idE                                                                                                           
80023b8c  _ZNSt8messagesIcED0Ev                                                                                                           
80023dfc  _ZNSt8messagesIcED1Ev                                                                                                           
40303334  _ZNSt8messagesIwE2idE                                                                                                           
80023b9c  _ZNSt8messagesIwED0Ev                                                                                                           
80023e00  _ZNSt8messagesIwED1Ev                                                                                                           
40303338  _ZNSt8numpunctIcE2idE                                                                                                           
80019a80  _ZNSt8numpunctIcE5_InitERKSt8_Locinfo                                                                                           
80022ae0  _ZNSt8numpunctIcE5_TidyEv                                                                                                       
800210b8  _ZNSt8numpunctIcE7_GetcatEPPKNSt6locale5facetE                                                                                  
80021114  _ZNSt8numpunctIcEC1Ej                                                                                                           
80022f14  _ZNSt8numpunctIcED0Ev                                                                                                           
80022b10  _ZNSt8numpunctIcED1Ev                                                                                                           
4030333c  _ZNSt8numpunctIwE2idE                                                                                                           
8001b538  _ZNSt8numpunctIwE5_InitERKSt8_Locinfo                                                                                           
800224c0  _ZNSt8numpunctIwED0Ev                                                                                                           
8002282c  _ZNSt8numpunctIwED1Ev                                                                                                           
40303340  _ZNSt8time_getIcSt19istreambuf_iteratorIcSt11char_traitsIcEEE2idE                                                               
8001f06c  _ZNSt8time_getIcSt19istreambuf_iteratorIcSt11char_traitsIcEEE5_InitERKSt8_Locinfo                                               
80022860  _ZNSt8time_getIcSt19istreambuf_iteratorIcSt11char_traitsIcEEED0Ev                                                               
80022c58  _ZNSt8time_getIcSt19istreambuf_iteratorIcSt11char_traitsIcEEED1Ev                                                               
40303344  _ZNSt8time_getIwSt19istreambuf_iteratorIwSt11char_traitsIwEEE2idE                                                               
80021228  _ZNSt8time_getIwSt19istreambuf_iteratorIwSt11char_traitsIwEEE5_InitERKSt8_Locinfo                                               
80022894  _ZNSt8time_getIwSt19istreambuf_iteratorIwSt11char_traitsIwEEED0Ev                                                               
80022c84  _ZNSt8time_getIwSt19istreambuf_iteratorIwSt11char_traitsIwEEED1Ev                                                               
40303348  _ZNSt8time_putIcSt19ostreambuf_iteratorIcSt11char_traitsIcEEE2idE                                                               
80023bac  _ZNSt8time_putIcSt19ostreambuf_iteratorIcSt11char_traitsIcEEED0Ev                                                               
80023e04  _ZNSt8time_putIcSt19ostreambuf_iteratorIcSt11char_traitsIcEEED1Ev                                                               
4030334c  _ZNSt8time_putIwSt19ostreambuf_iteratorIwSt11char_traitsIwEEE2idE                                                               
80023bbc  _ZNSt8time_putIwSt19ostreambuf_iteratorIwSt11char_traitsIwEEED0Ev                                                               
80023e08  _ZNSt8time_putIwSt19ostreambuf_iteratorIwSt11char_traitsIwEEED1Ev                                                               
40303034  _ZNSt9_FacetptrISt10moneypunctIcLb0EEE6_PsaveE                                                                                  
40303038  _ZNSt9_FacetptrISt10moneypunctIcLb1EEE6_PsaveE                                                                                  
4030303c  _ZNSt9_FacetptrISt10moneypunctIwLb0EEE6_PsaveE                                                                                  
40303040  _ZNSt9_FacetptrISt10moneypunctIwLb1EEE6_PsaveE                                                                                  
40303044  _ZNSt9_FacetptrISt5ctypeIcEE6_PsaveE                                                                                            
40303048  _ZNSt9_FacetptrISt5ctypeIwEE6_PsaveE                                                                                            
4030304c  _ZNSt9_FacetptrISt7codecvtIcciEE6_PsaveE                                                                                        
40303050  _ZNSt9_FacetptrISt7codecvtIwciEE6_PsaveE                                                                                        
40303054  _ZNSt9_FacetptrISt7collateIcEE6_PsaveE                                                                                          
40303058  _ZNSt9_FacetptrISt7collateIwEE6_PsaveE                                                                                          
4030305c  _ZNSt9_FacetptrISt7num_getIcSt19istreambuf_iteratorIcSt11char_traitsIcEEEE6_PsaveE                                              
40303060  _ZNSt9_FacetptrISt7num_getIwSt19istreambuf_iteratorIwSt11char_traitsIwEEEE6_PsaveE                                              
40303064  _ZNSt9_FacetptrISt7num_putIcSt19ostreambuf_iteratorIcSt11char_traitsIcEEEE6_PsaveE                                              
40303068  _ZNSt9_FacetptrISt7num_putIwSt19ostreambuf_iteratorIwSt11char_traitsIwEEEE6_PsaveE                                              
4030306c  _ZNSt9_FacetptrISt8messagesIcEE6_PsaveE                                                                                         
40303070  _ZNSt9_FacetptrISt8messagesIwEE6_PsaveE                                                                                         
40303074  _ZNSt9_FacetptrISt8numpunctIcEE6_PsaveE                                                                                         
40303078  _ZNSt9_FacetptrISt8numpunctIwEE6_PsaveE                                                                                         
4030307c  _ZNSt9_FacetptrISt8time_getIcSt19istreambuf_iteratorIcSt11char_traitsIcEEEE6_PsaveE                                             
40303080  _ZNSt9_FacetptrISt8time_getIwSt19istreambuf_iteratorIwSt11char_traitsIwEEEE6_PsaveE                                             
40303084  _ZNSt9_FacetptrISt8time_putIcSt19ostreambuf_iteratorIcSt11char_traitsIcEEEE6_PsaveE                                             
40303088  _ZNSt9_FacetptrISt8time_putIwSt19ostreambuf_iteratorIwSt11char_traitsIwEEEE6_PsaveE                                             
4030308c  _ZNSt9_FacetptrISt9money_getIcSt19istreambuf_iteratorIcSt11char_traitsIcEEEE6_PsaveE                                            
40303090  _ZNSt9_FacetptrISt9money_getIwSt19istreambuf_iteratorIwSt11char_traitsIwEEEE6_PsaveE                                            
40303094  _ZNSt9_FacetptrISt9money_putIcSt19ostreambuf_iteratorIcSt11char_traitsIcEEEE6_PsaveE                                            
40303098  _ZNSt9_FacetptrISt9money_putIwSt19ostreambuf_iteratorIwSt11char_traitsIwEEEE6_PsaveE                                            
80023bcc  _ZNSt9bad_allocD0Ev                                                                                                             
80023e0c  _ZNSt9bad_allocD1Ev                                                                                                             
80017ba4  _ZNSt9basic_iosIcSt11char_traitsIcEE4initEPSt15basic_streambufIcS1_Eb                                                           
80022044  _ZNSt9basic_iosIcSt11char_traitsIcEE5clearENSt5_IosbIiE8_IostateEb                                                              
80022084  _ZNSt9basic_iosIcSt11char_traitsIcEE8setstateENSt5_IosbIiE8_IostateEb                                                           
80023890  _ZNSt9basic_iosIcSt11char_traitsIcEED0Ev                                                                                        
80023e10  _ZNSt9basic_iosIcSt11char_traitsIcEED1Ev                                                                                        
80017868  _ZNSt9basic_iosIwSt11char_traitsIwEE4initEPSt15basic_streambufIwS1_Eb                                                           
800238a8  _ZNSt9basic_iosIwSt11char_traitsIwEED0Ev                                                                                        
80023e14  _ZNSt9basic_iosIwSt11char_traitsIwEED1Ev                                                                                        
80023bdc  _ZNSt9exceptionD0Ev                                                                                                             
80023e18  _ZNSt9exceptionD1Ev                                                                                                             
40303350  _ZNSt9money_getIcSt19istreambuf_iteratorIcSt11char_traitsIcEEE2idE                                                              
80023bec  _ZNSt9money_getIcSt19istreambuf_iteratorIcSt11char_traitsIcEEED0Ev                                                              
80023e1c  _ZNSt9money_getIcSt19istreambuf_iteratorIcSt11char_traitsIcEEED1Ev                                                              
40303354  _ZNSt9money_getIwSt19istreambuf_iteratorIwSt11char_traitsIwEEE2idE                                                              
80023bfc  _ZNSt9money_getIwSt19istreambuf_iteratorIwSt11char_traitsIwEEED0Ev                                                              
80023e20  _ZNSt9money_getIwSt19istreambuf_iteratorIwSt11char_traitsIwEEED1Ev                                                              
40303358  _ZNSt9money_putIcSt19ostreambuf_iteratorIcSt11char_traitsIcEEE2idE                                                              
800215b4  _ZNSt9money_putIcSt19ostreambuf_iteratorIcSt11char_traitsIcEEE4_PutES3_St22_String_const_iteratorIcS2_SaIcEEj                   
80021604  _ZNSt9money_putIcSt19ostreambuf_iteratorIcSt11char_traitsIcEEE4_RepES3_cj                                                       
80023c0c  _ZNSt9money_putIcSt19ostreambuf_iteratorIcSt11char_traitsIcEEED0Ev                                                              
80023e24  _ZNSt9money_putIcSt19ostreambuf_iteratorIcSt11char_traitsIcEEED1Ev                                                              
4030335c  _ZNSt9money_putIwSt19ostreambuf_iteratorIwSt11char_traitsIwEEE2idE                                                              
80021654  _ZNSt9money_putIwSt19ostreambuf_iteratorIwSt11char_traitsIwEEE4_PutES3_St22_String_const_iteratorIwS2_SaIwEEj                   
800216a4  _ZNSt9money_putIwSt19ostreambuf_iteratorIwSt11char_traitsIwEEE4_RepES3_wj                                                       
80023c1c  _ZNSt9money_putIwSt19ostreambuf_iteratorIwSt11char_traitsIwEEED0Ev                                                              
80023e28  _ZNSt9money_putIwSt19ostreambuf_iteratorIwSt11char_traitsIwEEED1Ev                                                              
80023c2c  _ZNSt9time_baseD0Ev                                                                                                             
80023e2c  _ZNSt9time_baseD1Ev                                                                                                             
800190a0  _ZNSt9type_infoD0Ev                                                                                                             
8001909c  _ZNSt9type_infoD1Ev                                                                                                             
8001909c  _ZNSt9type_infoD2Ev                                                                                                             
80015300  _ZSt10_GetloctxtIcSt19istreambuf_iteratorIcSt11char_traitsIcEEEiRT0_S5_jPKT_                                                    
80014594  _ZSt10_GetloctxtIwSt19istreambuf_iteratorIwSt11char_traitsIwEEEiRT0_S5_jPKT_                                                    
800235b0  _ZSt10_MaklocchrIcET_cPS0_RKSt7_Cvtvec                                                                                          
80022b40  _ZSt10_MaklocchrIwET_cPS0_RKSt7_Cvtvec                                                                                          
8001f63c  _ZSt10_MaklocstrIcEPT_PKcS1_RKSt7_Cvtvec                                                                                        
8001e41c  _ZSt10_MaklocstrIwEPT_PKcS1_RKSt7_Cvtvec                                                                                        
8001fd2c  _ZSt14_Debug_messagePKcS0_                                                                                                      
403030a8  _ZSt14_Raise_handler                                                                                                            
40303364  _ZSt16__dummy_typeinfo                                                                                                          
8001908c  _ZSt21__gen_dummy_typeinfosv                                                                                                    
4030297c  _ZSt3cin                                                                                                                        
40302f50  _ZSt4_Fpz                                                                                                                       
4030291c  _ZSt4cerr                                                                                                                       
4030294c  _ZSt4clog                                                                                                                       
403028ec  _ZSt4cout                                                                                                                       
8002132c  _ZSt4endlIcSt11char_traitsIcEERSt13basic_ostreamIT_T0_ES6_                                                                      
40302b34  _ZSt4wcin                                                                                                                       
40302ad4  _ZSt5wcerr                                                                                                                      
40302b04  _ZSt5wclog                                                                                                                      
40302aa4  _ZSt5wcout                                                                                                                      
8001fd74  _ZSt6_ThrowRKSt9exception                                                                                                       
403018bc  _ZSt7_BADOFF                                                                                                                    
800235cc  _ZSt8_ToloweriPKSt9_Ctypevec                                                                                                    
800235e8  _ZSt8_ToupperiPKSt9_Ctypevec                                                                                                    
800238c0  _ZSt9_AllocateIcEPT_jS1_                                                                                                        
8001b634  _ZSt9use_facetISt10moneypunctIcLb0EEERKT_RKSt6locale                                                                            
8001b040  _ZSt9use_facetISt10moneypunctIcLb1EEERKT_RKSt6locale                                                                            
8001b730  _ZSt9use_facetISt10moneypunctIwLb0EEERKT_RKSt6locale                                                                            
8001b140  _ZSt9use_facetISt10moneypunctIwLb1EEERKT_RKSt6locale                                                                            
8001db08  _ZSt9use_facetISt5ctypeIcEERKT_RKSt6locale                                                                                      
8001b928  _ZSt9use_facetISt5ctypeIwEERKT_RKSt6locale                                                                                      
8001dbd4  _ZSt9use_facetISt7num_putIcSt19ostreambuf_iteratorIcSt11char_traitsIcEEEERKT_RKSt6locale                                        
8001dca0  _ZSt9use_facetISt8numpunctIcEERKT_RKSt6locale                                                                                   
8001d1bc  _ZSt9use_facetISt8numpunctIwEERKT_RKSt6locale                                                                                   
80023448  _ZStanNSt5_IosbIiE9_FmtflagsES1_                                                                                                
80020a5c  _ZSteqIcSt11char_traitsIcEEbRKSt19istreambuf_iteratorIT_T0_ES7_                                                                 
80020ac0  _ZSteqIwSt11char_traitsIwEEbRKSt19istreambuf_iteratorIT_T0_ES7_                                                                 
80011250  _ZStlsISt11char_traitsIcEERSt13basic_ostreamIcT_ES5_PKc                                                                         
800204b0  _ZStneIcSt11char_traitsIcEEbRKSt19istreambuf_iteratorIT_T0_ES7_                                                                 
80020520  _ZStneIwSt11char_traitsIwEEbRKSt19istreambuf_iteratorIT_T0_ES7_                                                                 
80022b70  _ZStoRRNSt5_IosbIiE8_IostateES1_                                                                                                
403015b0  _ZTIN10__cxxabiv117__class_type_infoE                                                                                           
403015bc  _ZTIN10__cxxabiv117__pbase_type_infoE                                                                                           
403015c8  _ZTIN10__cxxabiv119__pointer_type_infoE                                                                                         
403015d4  _ZTIN10__cxxabiv120__si_class_type_infoE                                                                                        
403015e0  _ZTIN10__cxxabiv121__vmi_class_type_infoE                                                                                       
403015ec  _ZTIN10__cxxabiv123__fundamental_type_infoE                                                                                     
40301858  _ZTINSt6locale5facetE                                                                                                           
403015f8  _ZTINSt6locale7_LocimpE                                                                                                         
40301604  _ZTINSt8ios_base7failureE                                                                                                       
403013c8  _ZTIPKe                                                                                                                         
4030111c  _ZTISi                                                                                                                          
40301134  _ZTISo                                                                                                                          
40301610  _ZTISt10ctype_base                                                                                                              
4030161c  _ZTISt10money_base                                                                                                              
40301628  _ZTISt10moneypunctIcLb0EE                                                                                                       
40301634  _ZTISt10moneypunctIcLb1EE                                                                                                       
40301640  _ZTISt10moneypunctIwLb0EE                                                                                                       
4030164c  _ZTISt10moneypunctIwLb1EE                                                                                                       
40301658  _ZTISt11logic_error                                                                                                             
40301664  _ZTISt12codecvt_base                                                                                                            
40301670  _ZTISt12length_error                                                                                                            
4030167c  _ZTISt12out_of_range                                                                                                            
40301688  _ZTISt13basic_filebufIcSt11char_traitsIcEE                                                                                      
40301694  _ZTISt13basic_filebufIwSt11char_traitsIwEE                                                                                      
4030114c  _ZTISt13basic_istreamIwSt11char_traitsIwEE                                                                                      
40301164  _ZTISt13basic_ostreamIwSt11char_traitsIwEE                                                                                      
403016a0  _ZTISt13messages_base                                                                                                           
403016ac  _ZTISt13runtime_error                                                                                                           
40301860  _ZTISt15basic_streambufIcSt11char_traitsIcEE                                                                                    
40301868  _ZTISt15basic_streambufIwSt11char_traitsIwEE                                                                                    
40301870  _ZTISt5_IosbIiE                                                                                                                 
403016b8  _ZTISt5ctypeIcE                                                                                                                 
403016c4  _ZTISt5ctypeIwE                                                                                                                 
403016d0  _ZTISt7_MpunctIcE                                                                                                               
403016dc  _ZTISt7_MpunctIwE                                                                                                               
403016e8  _ZTISt7codecvtIcciE                                                                                                             
403016f4  _ZTISt7codecvtIwciE                                                                                                             
40301700  _ZTISt7collateIcE                                                                                                               
4030170c  _ZTISt7collateIwE                                                                                                               
40301718  _ZTISt7num_getIcSt19istreambuf_iteratorIcSt11char_traitsIcEEE                                                                   
40301724  _ZTISt7num_getIwSt19istreambuf_iteratorIwSt11char_traitsIwEEE                                                                   
40301730  _ZTISt7num_putIcSt19ostreambuf_iteratorIcSt11char_traitsIcEEE                                                                   
4030173c  _ZTISt7num_putIwSt19ostreambuf_iteratorIwSt11char_traitsIwEEE                                                                   
40301748  _ZTISt8ios_base                                                                                                                 
40301754  _ZTISt8messagesIcE                                                                                                              
40301760  _ZTISt8messagesIwE                                                                                                              
4030176c  _ZTISt8numpunctIcE                                                                                                              
40301778  _ZTISt8numpunctIwE                                                                                                              
40301784  _ZTISt8time_getIcSt19istreambuf_iteratorIcSt11char_traitsIcEEE                                                                  
40301790  _ZTISt8time_getIwSt19istreambuf_iteratorIwSt11char_traitsIwEEE                                                                  
4030179c  _ZTISt8time_putIcSt19ostreambuf_iteratorIcSt11char_traitsIcEEE                                                                  
403017a8  _ZTISt8time_putIwSt19ostreambuf_iteratorIwSt11char_traitsIwEEE                                                                  
403017b4  _ZTISt9bad_alloc                                                                                                                
403017c0  _ZTISt9basic_iosIcSt11char_traitsIcEE                                                                                           
403017cc  _ZTISt9basic_iosIwSt11char_traitsIwEE                                                                                           
40301878  _ZTISt9exception                                                                                                                
403017d8  _ZTISt9money_getIcSt19istreambuf_iteratorIcSt11char_traitsIcEEE                                                                 
403017e4  _ZTISt9money_getIwSt19istreambuf_iteratorIwSt11char_traitsIwEEE                                                                 
403017f0  _ZTISt9money_putIcSt19ostreambuf_iteratorIcSt11char_traitsIcEEE                                                                 
403017fc  _ZTISt9money_putIwSt19ostreambuf_iteratorIwSt11char_traitsIwEEE                                                                 
40301808  _ZTISt9time_base                                                                                                                
40301880  _ZTISt9type_info                                                                                                                
40301888  _ZTIe                                                                                                                           
40300fec  _ZTSN10__cxxabiv117__class_type_infoE                                                                                           
4030100e  _ZTSN10__cxxabiv117__pbase_type_infoE                                                                                           
40300f7f  _ZTSN10__cxxabiv119__pointer_type_infoE                                                                                         
40300f5a  _ZTSN10__cxxabiv120__si_class_type_infoE                                                                                        
40300f34  _ZTSN10__cxxabiv121__vmi_class_type_infoE                                                                                       
40300e1e  _ZTSN10__cxxabiv123__fundamental_type_infoE                                                                                     
4030135c  _ZTSNSt6locale5facetE                                                                                                           
40301320  _ZTSNSt6locale7_LocimpE                                                                                                         
403012b2  _ZTSNSt8ios_base7failureE                                                                                                       
403018b6  _ZTSPKe                                                                                                                         
403018d8  _ZTSSi                                                                                                                          
403018db  _ZTSSo                                                                                                                          
403014e8  _ZTSSt10ctype_base                                                                                                              
403014f7  _ZTSSt10money_base                                                                                                              
403012c8  _ZTSSt10moneypunctIcLb0EE                                                                                                       
403012de  _ZTSSt10moneypunctIcLb1EE                                                                                                       
403012f4  _ZTSSt10moneypunctIwLb0EE                                                                                                       
4030130a  _ZTSSt10moneypunctIwLb1EE                                                                                                       
403013d8  _ZTSSt11logic_error                                                                                                             
40301392  _ZTSSt12codecvt_base                                                                                                            
403013a3  _ZTSSt12length_error                                                                                                            
403013b4  _ZTSSt12out_of_range                                                                                                            
40300e98  _ZTSSt13basic_filebufIcSt11char_traitsIcEE                                                                                      
40300ebf  _ZTSSt13basic_filebufIwSt11char_traitsIwEE                                                                                      
40300ee6  _ZTSSt13basic_istreamIwSt11char_traitsIwEE                                                                                      
40300f0d  _ZTSSt13basic_ostreamIwSt11char_traitsIwEE                                                                                      
4030136e  _ZTSSt13messages_base                                                                                                           
40301380  _ZTSSt13runtime_error                                                                                                           
40300dcc  _ZTSSt15basic_streambufIcSt11char_traitsIcEE                                                                                    
40300df5  _ZTSSt15basic_streambufIwSt11char_traitsIwEE                                                                                    
40301814  _ZTSSt5_IosbIiE                                                                                                                 
40301820  _ZTSSt5ctypeIcE                                                                                                                 
4030182c  _ZTSSt5ctypeIwE                                                                                                                 
40301542  _ZTSSt7_MpunctIcE                                                                                                               
40301550  _ZTSSt7_MpunctIwE                                                                                                               
403013e8  _ZTSSt7codecvtIcciE                                                                                                             
403013f8  _ZTSSt7codecvtIwciE                                                                                                             
4030155e  _ZTSSt7collateIcE                                                                                                               
4030156c  _ZTSSt7collateIwE                                                                                                               
403009d4  _ZTSSt7num_getIcSt19istreambuf_iteratorIcSt11char_traitsIcEEE                                                                   
40300a0e  _ZTSSt7num_getIwSt19istreambuf_iteratorIwSt11char_traitsIwEEE                                                                   
40300a48  _ZTSSt7num_putIcSt19ostreambuf_iteratorIcSt11char_traitsIcEEE                                                                   
40300a82  _ZTSSt7num_putIwSt19ostreambuf_iteratorIwSt11char_traitsIwEEE                                                                   
40301838  _ZTSSt8ios_base                                                                                                                 
40301506  _ZTSSt8messagesIcE                                                                                                              
40301515  _ZTSSt8messagesIwE                                                                                                              
40301524  _ZTSSt8numpunctIcE                                                                                                              
40301533  _ZTSSt8numpunctIwE                                                                                                              
403008e8  _ZTSSt8time_getIcSt19istreambuf_iteratorIcSt11char_traitsIcEEE                                                                  
40300923  _ZTSSt8time_getIwSt19istreambuf_iteratorIwSt11char_traitsIwEEE                                                                  
4030095e  _ZTSSt8time_putIcSt19ostreambuf_iteratorIcSt11char_traitsIcEEE                                                                  
40300999  _ZTSSt8time_putIwSt19ostreambuf_iteratorIwSt11char_traitsIwEEE                                                                  
4030157a  _ZTSSt9bad_alloc                                                                                                                
40301030  _ZTSSt9basic_iosIcSt11char_traitsIcEE                                                                                           
40301052  _ZTSSt9basic_iosIwSt11char_traitsIwEE                                                                                           
40301587  _ZTSSt9exception                                                                                                                
40300780  _ZTSSt9money_getIcSt19istreambuf_iteratorIcSt11char_traitsIcEEE                                                                 
403007bc  _ZTSSt9money_getIwSt19istreambuf_iteratorIwSt11char_traitsIwEEE                                                                 
403007f8  _ZTSSt9money_putIcSt19ostreambuf_iteratorIcSt11char_traitsIcEEE                                                                 
40300834  _ZTSSt9money_putIwSt19ostreambuf_iteratorIwSt11char_traitsIwEEE                                                                 
40301594  _ZTSSt9time_base                                                                                                                
403015a1  _ZTSSt9type_info                                                                                                                
403018e4  _ZTSe                                                                                                                           
40300c1c  _ZTTSi                                                                                                                          
40300c4c  _ZTTSo                                                                                                                          
40300c7c  _ZTTSt13basic_istreamIwSt11char_traitsIwEE                                                                                      
40300cac  _ZTTSt13basic_ostreamIwSt11char_traitsIwEE                                                                                      
40301408  _ZTVN10__cxxabiv117__class_type_infoE                                                                                           
40301418  _ZTVN10__cxxabiv119__pointer_type_infoE                                                                                         
40301428  _ZTVN10__cxxabiv120__si_class_type_infoE                                                                                        
40301438  _ZTVN10__cxxabiv121__vmi_class_type_infoE                                                                                       
40301448  _ZTVN10__cxxabiv123__fundamental_type_infoE                                                                                     
40301458  _ZTVNSt6locale5facetE                                                                                                           
40301468  _ZTVNSt6locale7_LocimpE                                                                                                         
4030117c  _ZTVNSt8ios_base7failureE                                                                                                       
40300bf4  _ZTVSi                                                                                                                          
40300c24  _ZTVSo                                                                                                                          
40301478  _ZTVSt10ctype_base                                                                                                              
40301488  _ZTVSt10money_base                                                                                                              
40300abc  _ZTVSt10moneypunctIcLb0EE                                                                                                       
40300af0  _ZTVSt10moneypunctIcLb1EE                                                                                                       
40300b24  _ZTVSt10moneypunctIwLb0EE                                                                                                       
40300b58  _ZTVSt10moneypunctIwLb1EE                                                                                                       
40301194  _ZTVSt11logic_error                                                                                                             
40301074  _ZTVSt12codecvt_base                                                                                                            
403011ac  _ZTVSt12length_error                                                                                                            
403011c4  _ZTVSt12out_of_range                                                                                                            
403005d8  _ZTVSt13basic_filebufIcSt11char_traitsIcEE                                                                                      
40300620  _ZTVSt13basic_filebufIwSt11char_traitsIwEE                                                                                      
40300c54  _ZTVSt13basic_istreamIwSt11char_traitsIwEE                                                                                      
40300c84  _ZTVSt13basic_ostreamIwSt11char_traitsIwEE                                                                                      
40301498  _ZTVSt13messages_base                                                                                                           
403011dc  _ZTVSt13runtime_error                                                                                                           
40300668  _ZTVSt15basic_streambufIcSt11char_traitsIcEE                                                                                    
403006b0  _ZTVSt15basic_streambufIwSt11char_traitsIwEE                                                                                    
40300cb4  _ZTVSt5ctypeIcE                                                                                                                 
40300740  _ZTVSt5ctypeIwE                                                                                                                 
40300b8c  _ZTVSt7_MpunctIcE                                                                                                               
40300bc0  _ZTVSt7_MpunctIwE                                                                                                               
40300d74  _ZTVSt7codecvtIcciE                                                                                                             
40300da0  _ZTVSt7codecvtIwciE                                                                                                             
40301090  _ZTVSt7collateIcE                                                                                                               
403010ac  _ZTVSt7collateIwE                                                                                                               
40300870  _ZTVSt7num_getIcSt19istreambuf_iteratorIcSt11char_traitsIcEEE                                                                   
403008ac  _ZTVSt7num_getIwSt19istreambuf_iteratorIwSt11char_traitsIwEEE                                                                   
40300ce4  _ZTVSt7num_putIcSt19ostreambuf_iteratorIcSt11char_traitsIcEEE                                                                   
40300d14  _ZTVSt7num_putIwSt19ostreambuf_iteratorIwSt11char_traitsIwEEE                                                                   
403014a8  _ZTVSt8ios_base                                                                                                                 
403010c8  _ZTVSt8messagesIcE                                                                                                              
403010e4  _ZTVSt8messagesIwE                                                                                                              
40300fa4  _ZTVSt8numpunctIcE                                                                                                              
40300fc8  _ZTVSt8numpunctIwE                                                                                                              
40300e48  _ZTVSt8time_getIcSt19istreambuf_iteratorIcSt11char_traitsIcEEE                                                                  
40300e70  _ZTVSt8time_getIwSt19istreambuf_iteratorIwSt11char_traitsIwEEE                                                                  
40301334  _ZTVSt8time_putIcSt19ostreambuf_iteratorIcSt11char_traitsIcEEE                                                                  
40301348  _ZTVSt8time_putIwSt19ostreambuf_iteratorIwSt11char_traitsIwEEE                                                                  
403011f4  _ZTVSt9bad_alloc                                                                                                                
403014b8  _ZTVSt9basic_iosIcSt11char_traitsIcEE                                                                                           
403014c8  _ZTVSt9basic_iosIwSt11char_traitsIwEE                                                                                           
4030120c  _ZTVSt9exception                                                                                                                
40301224  _ZTVSt9money_getIcSt19istreambuf_iteratorIcSt11char_traitsIcEEE                                                                 
4030123c  _ZTVSt9money_getIwSt19istreambuf_iteratorIwSt11char_traitsIwEEE                                                                 
40301254  _ZTVSt9money_putIcSt19ostreambuf_iteratorIcSt11char_traitsIcEEE                                                                 
4030126c  _ZTVSt9money_putIwSt19ostreambuf_iteratorIwSt11char_traitsIwEEE                                                                 
403014d8  _ZTVSt9time_base                                                                                                                
80022f3c  _ZTv0_n12_NSiD0Ev                                                                                                               
80023468  _ZTv0_n12_NSiD1Ev                                                                                                               
80022f64  _ZTv0_n12_NSoD0Ev                                                                                                               
80023488  _ZTv0_n12_NSoD1Ev                                                                                                               
80022f8c  _ZTv0_n12_NSt13basic_istreamIwSt11char_traitsIwEED0Ev                                                                           
800234a8  _ZTv0_n12_NSt13basic_istreamIwSt11char_traitsIwEED1Ev                                                                           
80022fb4  _ZTv0_n12_NSt13basic_ostreamIwSt11char_traitsIwEED0Ev                                                                           
800234c8  _ZTv0_n12_NSt13basic_ostreamIwSt11char_traitsIwEED1Ev                                                                           
40301284  _ZZNKSt7num_getIcSt19istreambuf_iteratorIcSt11char_traitsIcEEE8_GetifldEPcRS3_S6_NSt5_IosbIiE9_FmtflagsERKSt6localeEs           
4030129b  _ZZNKSt7num_getIwSt19istreambuf_iteratorIwSt11char_traitsIwEEE8_GetifldEPcRS3_S6_NSt5_IosbIiE9_FmtflagsERKSt6localeEs           
40300e46  _ZZNKSt7num_putIcSt19ostreambuf_iteratorIcSt11char_traitsIcEEE5_FputES3_RSt8ios_basecPKcjjjjEs                                  
403015ae  _ZZNKSt7num_putIcSt19ostreambuf_iteratorIcSt11char_traitsIcEEE5_FputES3_RSt8ios_basecPKcjjjjEs_0                                
403013c5  _ZZNKSt7num_putIcSt19ostreambuf_iteratorIcSt11char_traitsIcEEE6do_putES3_RSt8ios_basecPKvEs                                     
4030184d  _ZZNKSt7num_putIcSt19ostreambuf_iteratorIcSt11char_traitsIcEEE6do_putES3_RSt8ios_baseclEs                                       
403018c0  _ZZNKSt7num_putIcSt19ostreambuf_iteratorIcSt11char_traitsIcEEE6do_putES3_RSt8ios_basecmEs                                       
403018c3  _ZZNKSt7num_putIcSt19ostreambuf_iteratorIcSt11char_traitsIcEEE6do_putES3_RSt8ios_basecxEs                                       
403018c6  _ZZNKSt7num_putIcSt19ostreambuf_iteratorIcSt11char_traitsIcEEE6do_putES3_RSt8ios_basecyEs                                       
403018ba  _ZZNKSt7num_putIwSt19ostreambuf_iteratorIwSt11char_traitsIwEEE5_FputES3_RSt8ios_basewPKcjjjjEs                                  
403018de  _ZZNKSt7num_putIwSt19ostreambuf_iteratorIwSt11char_traitsIwEEE5_FputES3_RSt8ios_basewPKcjjjjEs_0                                
403018c9  _ZZNKSt7num_putIwSt19ostreambuf_iteratorIwSt11char_traitsIwEEE6do_putES3_RSt8ios_basewPKvEs                                     
403018cc  _ZZNKSt7num_putIwSt19ostreambuf_iteratorIwSt11char_traitsIwEEE6do_putES3_RSt8ios_basewlEs                                       
403018cf  _ZZNKSt7num_putIwSt19ostreambuf_iteratorIwSt11char_traitsIwEEE6do_putES3_RSt8ios_basewmEs                                       
403018d2  _ZZNKSt7num_putIwSt19ostreambuf_iteratorIwSt11char_traitsIwEEE6do_putES3_RSt8ios_basewxEs                                       
403018d5  _ZZNKSt7num_putIwSt19ostreambuf_iteratorIwSt11char_traitsIwEEE6do_putES3_RSt8ios_basewyEs                                       
403003b4  _ZZNKSt8_Locinfo10_GetmonthsEvEs                                                                                                
4030052d  _ZZNKSt8_Locinfo8_GetdaysEvEs                                                                                                   
40300583  _ZZNKSt8_Locinfo8_GettrueEvEs                                                                                                   
40301890  _ZZNKSt8_Locinfo9_GetfalseEvEs                                                                                                  
40301896  _ZZNKSt9money_putIcSt19ostreambuf_iteratorIcSt11char_traitsIcEEE6do_putES3_bRSt8ios_baseceEs                                    
4030189c  _ZZNKSt9money_putIwSt19ostreambuf_iteratorIwSt11char_traitsIwEEE6do_putES3_bRSt8ios_baseweEs                                    
40300303  _ZZNSt7_MpunctIcE5_InitERKSt8_LocinfoEs                                                                                         
403018e0  _ZZNSt7_MpunctIcE5_InitERKSt8_LocinfoEs_0                                                                                       
403018a2  _ZZNSt7_MpunctIcE7_MakpatERNSt10money_base7patternEjjjEs                                                                        
4030043b  _ZZNSt7_MpunctIcE7_MakpatERNSt10money_base7patternEjjjEs_0                                                                      
40300fa3  _ZZNSt7_MpunctIwE5_InitERKSt8_LocinfoEs                                                                                         
403018e2  _ZZNSt7_MpunctIwE5_InitERKSt8_LocinfoEs_0                                                                                       
403018a7  _ZZNSt7_MpunctIwE7_MakpatERNSt10money_base7patternEjjjEs                                                                        
403004b4  _ZZNSt7_MpunctIwE7_MakpatERNSt10money_base7patternEjjjEs_0                                                                      
80023c4c  _ZdaPv                                                                                                                          
80023c4c  _ZdlPv                                                                                                                          
40302f40  _Zero                                                                                                                           
800218bc  _Znaj                                                                                                                           
800218bc  _Znwj                                                                                                                           
80023d80  _ZnwjPv                                                                                                                         
403030b4  __CIOBUF_                                                                                                                       
403020e8  __STACK_END                                                                                                                     
00000800  __STACK_SIZE                                                                                                                    
00000800  __SYSMEM_SIZE                                                                                                                   
403034a8  __TI_CINIT_Base                                                                                                                 
403034b8  __TI_CINIT_Limit                                                                                                                
40303494  __TI_Handler_Table_Base                                                                                                         
403034a0  __TI_Handler_Table_Limit                                                                                                        
8001ec0c  __TI_auto_init                                                                                                                  
8001bb14  __TI_buff_read                                                                                                                  
80013bb4  __TI_cleanup                                                                                                                    
40303024  __TI_cleanup_ptr                                                                                                                
8001b82c  __TI_closefile                                                                                                                  
80023a88  __TI_decompress_none                                                                                                            
80023d78  __TI_decompress_rle24                                                                                                           
80019950  __TI_doflush                                                                                                                    
40303028  __TI_dtors_ptr                                                                                                                  
40302ff0  __TI_ft_end                                                                                                                     
80001574  __TI_printfi                                                                                                                    
8001a1fc  __TI_rd_ok                                                                                                                      
8001eda4  __TI_readmsg                                                                                                                    
40303390  __TI_static_base__                                                                                                              
403031d4  __TI_tmpnams                                                                                                                    
8001fa94  __TI_tvaltostr                                                                                                                  
8001ed54  __TI_writemsg                                                                                                                   
8001a15c  __TI_wrt_ok                                                                                                                     
80023c3c  __TI_zero_init                                                                                                                  
800180fc  __aeabi_atexit                                                                                                                  
8001d29c  __aeabi_cdcmpeq                                                                                                                 
8001d29c  __aeabi_cdcmple                                                                                                                 
8001d37c  __aeabi_cdrcmple                                                                                                                
800211cc  __aeabi_d2f                                                                                                                     
80021170  __aeabi_d2iz                                                                                                                    
80016750  __aeabi_dadd                                                                                                                    
80018390  __aeabi_ddiv                                                                                                                    
80019dfc  __aeabi_dmul                                                                                                                    
80016744  __aeabi_dsub                                                                                                                    
800224fc  __aeabi_i2d                                                                                                                     
8001aa00  __aeabi_idiv                                                                                                                    
80023e30  __aeabi_idiv0                                                                                                                   
8001aa00  __aeabi_idivmod                                                                                                                 
8001e4cc  __aeabi_memclr                                                                                                                  
8001e4cc  __aeabi_memclr4                                                                                                                 
8001e4cc  __aeabi_memclr8                                                                                                                 
80018828  __aeabi_memcpy                                                                                                                  
80018828  __aeabi_memcpy4                                                                                                                 
80018828  __aeabi_memcpy8                                                                                                                 
8001e4d0  __aeabi_memset                                                                                                                  
8001e4d0  __aeabi_memset4                                                                                                                 
8001e4d0  __aeabi_memset8                                                                                                                 
40302ffc  __aeabi_stderr                                                                                                                  
40302ff4  __aeabi_stdin                                                                                                                   
40302ff8  __aeabi_stdout                                                                                                                  
8001bc04  __aeabi_uidiv                                                                                                                   
8001bc04  __aeabi_uidivmod                                                                                                                
80014854  __aeabi_uldivmod                                                                                                                
ffffffff  __binit__                                                                                                                       
ffffffff  __c_args__                                                                                                                      
80018174  __cxa_atexit                                                                                                                    
8001806c  __cxa_finalize                                                                                                                  
800228ec  __cxa_guard_abort                                                                                                               
800228d8  __cxa_guard_acquire                                                                                                             
800228c8  __cxa_guard_release                                                                                                             
800180dc  __cxa_ia64_exit                                                                                                                 
40303368  __dso_handle                                                                                                                    
403018e8  __stack                                                                                                                         
80001a70  __sti___10_locale_cpp_badf69ba                                                                                                  
800099f4  __sti___11_locale0_cpp_36e19383                                                                                                 
8000420c  __sti___11_wlocale_cpp_3b9bd5f7                                                                                                 
800085ac  __sti___11_xlocale_cpp_3609b607                                                                                                 
8000d2dc  __sti___12_iostream_cpp_b004430c                                                                                                
8000bbe0  __sti___12_wiostrea_cpp_9fa80e7a                                                                                                
80014cb0  __sti___14_SimpleClass_cc_main                                                                                                  
800234e8  _args_main                                                                                                                      
80021380  _c_int00                                                                                                                        
40300202  _ctypes_                                                                                                                        
40302c58  _ftable                                                                                                                         
4030301c  _lock                                                                                                                           
403030b0  _new_handler                                                                                                                    
8002323c  _nop                                                                                                                            
80023230  _register_lock                                                                                                                  
80023224  _register_unlock                                                                                                                
403020e8  _sys_memory                                                                                                                     
80023d88  _system_pre_init                                                                                                                
40303000  _tz                                                                                                                             
40303020  _unlock                                                                                                                         
80020204  abort                                                                                                                           
8000f05c  add_device                                                                                                                      
800180e4  atexit                                                                                                                          
8001fc24  atoi                                                                                                                            
ffffffff  binit                                                                                                                           
80016b2c  btowc                                                                                                                           
8000e5c4  calloc                                                                                                                          
8000efcc  close                                                                                                                           
8001fca8  copy_in                                                                                                                         
80020210  exit                                                                                                                            
8001b8d8  fclose                                                                                                                          
80021280  feraiseexcept                                                                                                                   
800199d4  fflush                                                                                                                          
8001d45c  fgetc                                                                                                                           
80022ba0  fgetpos                                                                                                                         
8001d45c  fgetwc                                                                                                                          
80013c4c  fopen                                                                                                                           
8001b240  fputc                                                                                                                           
80017338  fputs                                                                                                                           
80016b18  fputwc                                                                                                                          
8000e198  free                                                                                                                            
80013c00  freopen                                                                                                                         
80022bd0  frexp                                                                                                                           
8001e974  fseek                                                                                                                           
80023c5c  fsetpos                                                                                                                         
8001ecb0  ftell                                                                                                                           
800157f0  fwrite                                                                                                                          
8001d45c  getc                                                                                                                            
8001d528  getchar                                                                                                                         
8002079c  ldexp                                                                                                                           
80021a64  localeconv                                                                                                                      
8000ef88  lseek                                                                                                                           
8001fdb0  ltoa                                                                                                                            
80014b0c  main                                                                                                                            
403030ac  main_func_sp                                                                                                                    
8000e0dc  malloc                                                                                                                          
8001c520  mblen                                                                                                                           
80016af4  mbrtowc                                                                                                                         
8001c4e4  mbstowcs                                                                                                                        
8001c4b0  mbtowc                                                                                                                          
8000e484  memalign                                                                                                                        
80022cb0  memccpy                                                                                                                         
80022cdc  memchr                                                                                                                          
800228fc  memcmp                                                                                                                          
80018828  memcpy                                                                                                                          
80022650  memmove                                                                                                                         
8001e4dc  memset                                                                                                                          
8000dfe0  minit                                                                                                                           
8000ee70  open                                                                                                                            
8001b240  putc                                                                                                                            
8001b32c  putchar                                                                                                                         
800174c8  puts                                                                                                                            
80021908  raise                                                                                                                           
8000ee2c  read                                                                                                                            
8000e2f0  realloc                                                                                                                         
8000ed34  remove                                                                                                                          
8000ede0  remove_device                                                                                                                   
8000ed74  rename                                                                                                                          
80021a2c  setlocale                                                                                                                       
80018f34  setvbuf                                                                                                                         
80020b24  signal                                                                                                                          
8001ea1c  sprintf                                                                                                                         
80022d08  strcat                                                                                                                          
80022fdc  strchr                                                                                                                          
80023004  strcmp                                                                                                                          
800238d8  strcpy                                                                                                                          
80021efc  strcspn                                                                                                                         
8000f184  strftime                                                                                                                        
80023604  strlen                                                                                                                          
80021a74  strncpy                                                                                                                         
80012e54  strtod                                                                                                                          
80016f74  strtol                                                                                                                          
80012e54  strtold                                                                                                                         
80013790  strtoll                                                                                                                         
80017500  strtoul                                                                                                                         
80015a34  strtoull                                                                                                                        
800238f0  tolower                                                                                                                         
80023908  toupper                                                                                                                         
8001dfc4  ungetc                                                                                                                          
80016ac0  ungetwc                                                                                                                         
8000ed34  unlink                                                                                                                          
80016aac  wcrtomb                                                                                                                         
80016a88  wcslen                                                                                                                          
8001c470  wcstombs                                                                                                                        
80016a58  wctob                                                                                                                           
8001c458  wctomb                                                                                                                          
80016a30  wmemchr                                                                                                                         
800169f0  wmemcmp                                                                                                                         
800169d0  wmemcpy                                                                                                                         
80016974  wmemmove                                                                                                                        
80016958  wmemset                                                                                                                         
8000ec3c  write                                                                                                                           


GLOBAL SYMBOLS: SORTED BY Symbol Address 

address   name                                                                                                                            
-------   ----                                                                                                                            
00000800  __STACK_SIZE                                                                                                                    
00000800  __SYSMEM_SIZE                                                                                                                   
40300202  _ctypes_                                                                                                                        
40300303  _ZZNSt7_MpunctIcE5_InitERKSt8_LocinfoEs                                                                                         
403003b4  _ZZNKSt8_Locinfo10_GetmonthsEvEs                                                                                                
4030043b  _ZZNSt7_MpunctIcE7_MakpatERNSt10money_base7patternEjjjEs_0                                                                      
403004b4  _ZZNSt7_MpunctIwE7_MakpatERNSt10money_base7patternEjjjEs_0                                                                      
4030052d  _ZZNKSt8_Locinfo8_GetdaysEvEs                                                                                                   
40300583  _ZZNKSt8_Locinfo8_GettrueEvEs                                                                                                   
403005d8  _ZTVSt13basic_filebufIcSt11char_traitsIcEE                                                                                      
40300620  _ZTVSt13basic_filebufIwSt11char_traitsIwEE                                                                                      
40300668  _ZTVSt15basic_streambufIcSt11char_traitsIcEE                                                                                    
403006b0  _ZTVSt15basic_streambufIwSt11char_traitsIwEE                                                                                    
40300740  _ZTVSt5ctypeIwE                                                                                                                 
40300780  _ZTSSt9money_getIcSt19istreambuf_iteratorIcSt11char_traitsIcEEE                                                                 
403007bc  _ZTSSt9money_getIwSt19istreambuf_iteratorIwSt11char_traitsIwEEE                                                                 
403007f8  _ZTSSt9money_putIcSt19ostreambuf_iteratorIcSt11char_traitsIcEEE                                                                 
40300834  _ZTSSt9money_putIwSt19ostreambuf_iteratorIwSt11char_traitsIwEEE                                                                 
40300870  _ZTVSt7num_getIcSt19istreambuf_iteratorIcSt11char_traitsIcEEE                                                                   
403008ac  _ZTVSt7num_getIwSt19istreambuf_iteratorIwSt11char_traitsIwEEE                                                                   
403008e8  _ZTSSt8time_getIcSt19istreambuf_iteratorIcSt11char_traitsIcEEE                                                                  
40300923  _ZTSSt8time_getIwSt19istreambuf_iteratorIwSt11char_traitsIwEEE                                                                  
4030095e  _ZTSSt8time_putIcSt19ostreambuf_iteratorIcSt11char_traitsIcEEE                                                                  
40300999  _ZTSSt8time_putIwSt19ostreambuf_iteratorIwSt11char_traitsIwEEE                                                                  
403009d4  _ZTSSt7num_getIcSt19istreambuf_iteratorIcSt11char_traitsIcEEE                                                                   
40300a0e  _ZTSSt7num_getIwSt19istreambuf_iteratorIwSt11char_traitsIwEEE                                                                   
40300a48  _ZTSSt7num_putIcSt19ostreambuf_iteratorIcSt11char_traitsIcEEE                                                                   
40300a82  _ZTSSt7num_putIwSt19ostreambuf_iteratorIwSt11char_traitsIwEEE                                                                   
40300abc  _ZTVSt10moneypunctIcLb0EE                                                                                                       
40300af0  _ZTVSt10moneypunctIcLb1EE                                                                                                       
40300b24  _ZTVSt10moneypunctIwLb0EE                                                                                                       
40300b58  _ZTVSt10moneypunctIwLb1EE                                                                                                       
40300b8c  _ZTVSt7_MpunctIcE                                                                                                               
40300bc0  _ZTVSt7_MpunctIwE                                                                                                               
40300bf4  _ZTVSi                                                                                                                          
40300c1c  _ZTTSi                                                                                                                          
40300c24  _ZTVSo                                                                                                                          
40300c4c  _ZTTSo                                                                                                                          
40300c54  _ZTVSt13basic_istreamIwSt11char_traitsIwEE                                                                                      
40300c7c  _ZTTSt13basic_istreamIwSt11char_traitsIwEE                                                                                      
40300c84  _ZTVSt13basic_ostreamIwSt11char_traitsIwEE                                                                                      
40300cac  _ZTTSt13basic_ostreamIwSt11char_traitsIwEE                                                                                      
40300cb4  _ZTVSt5ctypeIcE                                                                                                                 
40300ce4  _ZTVSt7num_putIcSt19ostreambuf_iteratorIcSt11char_traitsIcEEE                                                                   
40300d14  _ZTVSt7num_putIwSt19ostreambuf_iteratorIwSt11char_traitsIwEEE                                                                   
40300d74  _ZTVSt7codecvtIcciE                                                                                                             
40300da0  _ZTVSt7codecvtIwciE                                                                                                             
40300dcc  _ZTSSt15basic_streambufIcSt11char_traitsIcEE                                                                                    
40300df5  _ZTSSt15basic_streambufIwSt11char_traitsIwEE                                                                                    
40300e1e  _ZTSN10__cxxabiv123__fundamental_type_infoE                                                                                     
40300e46  _ZZNKSt7num_putIcSt19ostreambuf_iteratorIcSt11char_traitsIcEEE5_FputES3_RSt8ios_basecPKcjjjjEs                                  
40300e48  _ZTVSt8time_getIcSt19istreambuf_iteratorIcSt11char_traitsIcEEE                                                                  
40300e70  _ZTVSt8time_getIwSt19istreambuf_iteratorIwSt11char_traitsIwEEE                                                                  
40300e98  _ZTSSt13basic_filebufIcSt11char_traitsIcEE                                                                                      
40300ebf  _ZTSSt13basic_filebufIwSt11char_traitsIwEE                                                                                      
40300ee6  _ZTSSt13basic_istreamIwSt11char_traitsIwEE                                                                                      
40300f0d  _ZTSSt13basic_ostreamIwSt11char_traitsIwEE                                                                                      
40300f34  _ZTSN10__cxxabiv121__vmi_class_type_infoE                                                                                       
40300f5a  _ZTSN10__cxxabiv120__si_class_type_infoE                                                                                        
40300f7f  _ZTSN10__cxxabiv119__pointer_type_infoE                                                                                         
40300fa3  _ZZNSt7_MpunctIwE5_InitERKSt8_LocinfoEs                                                                                         
40300fa4  _ZTVSt8numpunctIcE                                                                                                              
40300fc8  _ZTVSt8numpunctIwE                                                                                                              
40300fec  _ZTSN10__cxxabiv117__class_type_infoE                                                                                           
4030100e  _ZTSN10__cxxabiv117__pbase_type_infoE                                                                                           
40301030  _ZTSSt9basic_iosIcSt11char_traitsIcEE                                                                                           
40301052  _ZTSSt9basic_iosIwSt11char_traitsIwEE                                                                                           
40301074  _ZTVSt12codecvt_base                                                                                                            
40301090  _ZTVSt7collateIcE                                                                                                               
403010ac  _ZTVSt7collateIwE                                                                                                               
403010c8  _ZTVSt8messagesIcE                                                                                                              
403010e4  _ZTVSt8messagesIwE                                                                                                              
4030111c  _ZTISi                                                                                                                          
40301134  _ZTISo                                                                                                                          
4030114c  _ZTISt13basic_istreamIwSt11char_traitsIwEE                                                                                      
40301164  _ZTISt13basic_ostreamIwSt11char_traitsIwEE                                                                                      
4030117c  _ZTVNSt8ios_base7failureE                                                                                                       
40301194  _ZTVSt11logic_error                                                                                                             
403011ac  _ZTVSt12length_error                                                                                                            
403011c4  _ZTVSt12out_of_range                                                                                                            
403011dc  _ZTVSt13runtime_error                                                                                                           
403011f4  _ZTVSt9bad_alloc                                                                                                                
4030120c  _ZTVSt9exception                                                                                                                
40301224  _ZTVSt9money_getIcSt19istreambuf_iteratorIcSt11char_traitsIcEEE                                                                 
4030123c  _ZTVSt9money_getIwSt19istreambuf_iteratorIwSt11char_traitsIwEEE                                                                 
40301254  _ZTVSt9money_putIcSt19ostreambuf_iteratorIcSt11char_traitsIcEEE                                                                 
4030126c  _ZTVSt9money_putIwSt19ostreambuf_iteratorIwSt11char_traitsIwEEE                                                                 
40301284  _ZZNKSt7num_getIcSt19istreambuf_iteratorIcSt11char_traitsIcEEE8_GetifldEPcRS3_S6_NSt5_IosbIiE9_FmtflagsERKSt6localeEs           
4030129b  _ZZNKSt7num_getIwSt19istreambuf_iteratorIwSt11char_traitsIwEEE8_GetifldEPcRS3_S6_NSt5_IosbIiE9_FmtflagsERKSt6localeEs           
403012b2  _ZTSNSt8ios_base7failureE                                                                                                       
403012c8  _ZTSSt10moneypunctIcLb0EE                                                                                                       
403012de  _ZTSSt10moneypunctIcLb1EE                                                                                                       
403012f4  _ZTSSt10moneypunctIwLb0EE                                                                                                       
4030130a  _ZTSSt10moneypunctIwLb1EE                                                                                                       
40301320  _ZTSNSt6locale7_LocimpE                                                                                                         
40301334  _ZTVSt8time_putIcSt19ostreambuf_iteratorIcSt11char_traitsIcEEE                                                                  
40301348  _ZTVSt8time_putIwSt19ostreambuf_iteratorIwSt11char_traitsIwEEE                                                                  
4030135c  _ZTSNSt6locale5facetE                                                                                                           
4030136e  _ZTSSt13messages_base                                                                                                           
40301380  _ZTSSt13runtime_error                                                                                                           
40301392  _ZTSSt12codecvt_base                                                                                                            
403013a3  _ZTSSt12length_error                                                                                                            
403013b4  _ZTSSt12out_of_range                                                                                                            
403013c5  _ZZNKSt7num_putIcSt19ostreambuf_iteratorIcSt11char_traitsIcEEE6do_putES3_RSt8ios_basecPKvEs                                     
403013c8  _ZTIPKe                                                                                                                         
403013d8  _ZTSSt11logic_error                                                                                                             
403013e8  _ZTSSt7codecvtIcciE                                                                                                             
403013f8  _ZTSSt7codecvtIwciE                                                                                                             
40301408  _ZTVN10__cxxabiv117__class_type_infoE                                                                                           
40301418  _ZTVN10__cxxabiv119__pointer_type_infoE                                                                                         
40301428  _ZTVN10__cxxabiv120__si_class_type_infoE                                                                                        
40301438  _ZTVN10__cxxabiv121__vmi_class_type_infoE                                                                                       
40301448  _ZTVN10__cxxabiv123__fundamental_type_infoE                                                                                     
40301458  _ZTVNSt6locale5facetE                                                                                                           
40301468  _ZTVNSt6locale7_LocimpE                                                                                                         
40301478  _ZTVSt10ctype_base                                                                                                              
40301488  _ZTVSt10money_base                                                                                                              
40301498  _ZTVSt13messages_base                                                                                                           
403014a8  _ZTVSt8ios_base                                                                                                                 
403014b8  _ZTVSt9basic_iosIcSt11char_traitsIcEE                                                                                           
403014c8  _ZTVSt9basic_iosIwSt11char_traitsIwEE                                                                                           
403014d8  _ZTVSt9time_base                                                                                                                
403014e8  _ZTSSt10ctype_base                                                                                                              
403014f7  _ZTSSt10money_base                                                                                                              
40301506  _ZTSSt8messagesIcE                                                                                                              
40301515  _ZTSSt8messagesIwE                                                                                                              
40301524  _ZTSSt8numpunctIcE                                                                                                              
40301533  _ZTSSt8numpunctIwE                                                                                                              
40301542  _ZTSSt7_MpunctIcE                                                                                                               
40301550  _ZTSSt7_MpunctIwE                                                                                                               
4030155e  _ZTSSt7collateIcE                                                                                                               
4030156c  _ZTSSt7collateIwE                                                                                                               
4030157a  _ZTSSt9bad_alloc                                                                                                                
40301587  _ZTSSt9exception                                                                                                                
40301594  _ZTSSt9time_base                                                                                                                
403015a1  _ZTSSt9type_info                                                                                                                
403015ae  _ZZNKSt7num_putIcSt19ostreambuf_iteratorIcSt11char_traitsIcEEE5_FputES3_RSt8ios_basecPKcjjjjEs_0                                
403015b0  _ZTIN10__cxxabiv117__class_type_infoE                                                                                           
403015bc  _ZTIN10__cxxabiv117__pbase_type_infoE                                                                                           
403015c8  _ZTIN10__cxxabiv119__pointer_type_infoE                                                                                         
403015d4  _ZTIN10__cxxabiv120__si_class_type_infoE                                                                                        
403015e0  _ZTIN10__cxxabiv121__vmi_class_type_infoE                                                                                       
403015ec  _ZTIN10__cxxabiv123__fundamental_type_infoE                                                                                     
403015f8  _ZTINSt6locale7_LocimpE                                                                                                         
40301604  _ZTINSt8ios_base7failureE                                                                                                       
40301610  _ZTISt10ctype_base                                                                                                              
4030161c  _ZTISt10money_base                                                                                                              
40301628  _ZTISt10moneypunctIcLb0EE                                                                                                       
40301634  _ZTISt10moneypunctIcLb1EE                                                                                                       
40301640  _ZTISt10moneypunctIwLb0EE                                                                                                       
4030164c  _ZTISt10moneypunctIwLb1EE                                                                                                       
40301658  _ZTISt11logic_error                                                                                                             
40301664  _ZTISt12codecvt_base                                                                                                            
40301670  _ZTISt12length_error                                                                                                            
4030167c  _ZTISt12out_of_range                                                                                                            
40301688  _ZTISt13basic_filebufIcSt11char_traitsIcEE                                                                                      
40301694  _ZTISt13basic_filebufIwSt11char_traitsIwEE                                                                                      
403016a0  _ZTISt13messages_base                                                                                                           
403016ac  _ZTISt13runtime_error                                                                                                           
403016b8  _ZTISt5ctypeIcE                                                                                                                 
403016c4  _ZTISt5ctypeIwE                                                                                                                 
403016d0  _ZTISt7_MpunctIcE                                                                                                               
403016dc  _ZTISt7_MpunctIwE                                                                                                               
403016e8  _ZTISt7codecvtIcciE                                                                                                             
403016f4  _ZTISt7codecvtIwciE                                                                                                             
40301700  _ZTISt7collateIcE                                                                                                               
4030170c  _ZTISt7collateIwE                                                                                                               
40301718  _ZTISt7num_getIcSt19istreambuf_iteratorIcSt11char_traitsIcEEE                                                                   
40301724  _ZTISt7num_getIwSt19istreambuf_iteratorIwSt11char_traitsIwEEE                                                                   
40301730  _ZTISt7num_putIcSt19ostreambuf_iteratorIcSt11char_traitsIcEEE                                                                   
4030173c  _ZTISt7num_putIwSt19ostreambuf_iteratorIwSt11char_traitsIwEEE                                                                   
40301748  _ZTISt8ios_base                                                                                                                 
40301754  _ZTISt8messagesIcE                                                                                                              
40301760  _ZTISt8messagesIwE                                                                                                              
4030176c  _ZTISt8numpunctIcE                                                                                                              
40301778  _ZTISt8numpunctIwE                                                                                                              
40301784  _ZTISt8time_getIcSt19istreambuf_iteratorIcSt11char_traitsIcEEE                                                                  
40301790  _ZTISt8time_getIwSt19istreambuf_iteratorIwSt11char_traitsIwEEE                                                                  
4030179c  _ZTISt8time_putIcSt19ostreambuf_iteratorIcSt11char_traitsIcEEE                                                                  
403017a8  _ZTISt8time_putIwSt19ostreambuf_iteratorIwSt11char_traitsIwEEE                                                                  
403017b4  _ZTISt9bad_alloc                                                                                                                
403017c0  _ZTISt9basic_iosIcSt11char_traitsIcEE                                                                                           
403017cc  _ZTISt9basic_iosIwSt11char_traitsIwEE                                                                                           
403017d8  _ZTISt9money_getIcSt19istreambuf_iteratorIcSt11char_traitsIcEEE                                                                 
403017e4  _ZTISt9money_getIwSt19istreambuf_iteratorIwSt11char_traitsIwEEE                                                                 
403017f0  _ZTISt9money_putIcSt19ostreambuf_iteratorIcSt11char_traitsIcEEE                                                                 
403017fc  _ZTISt9money_putIwSt19ostreambuf_iteratorIwSt11char_traitsIwEEE                                                                 
40301808  _ZTISt9time_base                                                                                                                
40301814  _ZTSSt5_IosbIiE                                                                                                                 
40301820  _ZTSSt5ctypeIcE                                                                                                                 
4030182c  _ZTSSt5ctypeIwE                                                                                                                 
40301838  _ZTSSt8ios_base                                                                                                                 
4030184d  _ZZNKSt7num_putIcSt19ostreambuf_iteratorIcSt11char_traitsIcEEE6do_putES3_RSt8ios_baseclEs                                       
40301858  _ZTINSt6locale5facetE                                                                                                           
40301860  _ZTISt15basic_streambufIcSt11char_traitsIcEE                                                                                    
40301868  _ZTISt15basic_streambufIwSt11char_traitsIwEE                                                                                    
40301870  _ZTISt5_IosbIiE                                                                                                                 
40301878  _ZTISt9exception                                                                                                                
40301880  _ZTISt9type_info                                                                                                                
40301888  _ZTIe                                                                                                                           
40301890  _ZZNKSt8_Locinfo9_GetfalseEvEs                                                                                                  
40301896  _ZZNKSt9money_putIcSt19ostreambuf_iteratorIcSt11char_traitsIcEEE6do_putES3_bRSt8ios_baseceEs                                    
4030189c  _ZZNKSt9money_putIwSt19ostreambuf_iteratorIwSt11char_traitsIwEEE6do_putES3_bRSt8ios_baseweEs                                    
403018a2  _ZZNSt7_MpunctIcE7_MakpatERNSt10money_base7patternEjjjEs                                                                        
403018a7  _ZZNSt7_MpunctIwE7_MakpatERNSt10money_base7patternEjjjEs                                                                        
403018b6  _ZTSPKe                                                                                                                         
403018ba  _ZZNKSt7num_putIwSt19ostreambuf_iteratorIwSt11char_traitsIwEEE5_FputES3_RSt8ios_basewPKcjjjjEs                                  
403018bc  _ZSt7_BADOFF                                                                                                                    
403018c0  _ZZNKSt7num_putIcSt19ostreambuf_iteratorIcSt11char_traitsIcEEE6do_putES3_RSt8ios_basecmEs                                       
403018c3  _ZZNKSt7num_putIcSt19ostreambuf_iteratorIcSt11char_traitsIcEEE6do_putES3_RSt8ios_basecxEs                                       
403018c6  _ZZNKSt7num_putIcSt19ostreambuf_iteratorIcSt11char_traitsIcEEE6do_putES3_RSt8ios_basecyEs                                       
403018c9  _ZZNKSt7num_putIwSt19ostreambuf_iteratorIwSt11char_traitsIwEEE6do_putES3_RSt8ios_basewPKvEs                                     
403018cc  _ZZNKSt7num_putIwSt19ostreambuf_iteratorIwSt11char_traitsIwEEE6do_putES3_RSt8ios_basewlEs                                       
403018cf  _ZZNKSt7num_putIwSt19ostreambuf_iteratorIwSt11char_traitsIwEEE6do_putES3_RSt8ios_basewmEs                                       
403018d2  _ZZNKSt7num_putIwSt19ostreambuf_iteratorIwSt11char_traitsIwEEE6do_putES3_RSt8ios_basewxEs                                       
403018d5  _ZZNKSt7num_putIwSt19ostreambuf_iteratorIwSt11char_traitsIwEEE6do_putES3_RSt8ios_basewyEs                                       
403018d8  _ZTSSi                                                                                                                          
403018db  _ZTSSo                                                                                                                          
403018de  _ZZNKSt7num_putIwSt19ostreambuf_iteratorIwSt11char_traitsIwEEE5_FputES3_RSt8ios_basewPKcjjjjEs_0                                
403018e0  _ZZNSt7_MpunctIcE5_InitERKSt8_LocinfoEs_0                                                                                       
403018e2  _ZZNSt7_MpunctIwE5_InitERKSt8_LocinfoEs_0                                                                                       
403018e4  _ZTSe                                                                                                                           
403018e8  __stack                                                                                                                         
403020e8  __STACK_END                                                                                                                     
403020e8  _sys_memory                                                                                                                     
403028e8  _ZNSt8ios_base4Init9_Init_cntE                                                                                                  
403028ec  _ZSt4cout                                                                                                                       
4030291c  _ZSt4cerr                                                                                                                       
4030294c  _ZSt4clog                                                                                                                       
4030297c  _ZSt3cin                                                                                                                        
40302aa0  _ZNSt6_Winit9_Init_cntE                                                                                                         
40302aa4  _ZSt5wcout                                                                                                                      
40302ad4  _ZSt5wcerr                                                                                                                      
40302b04  _ZSt5wclog                                                                                                                      
40302b34  _ZSt4wcin                                                                                                                       
40302c58  _ftable                                                                                                                         
40302ec8  _Denorm                                                                                                                         
40302ed8  _Eps                                                                                                                            
40302ee8  _Hugeval                                                                                                                        
40302ef8  _Inf                                                                                                                            
40302f08  _Nan                                                                                                                            
40302f18  _Snan                                                                                                                           
40302f28  _Rteps                                                                                                                          
40302f38  _Xbig                                                                                                                           
40302f40  _Zero                                                                                                                           
40302f48  _ZNSt8ios_base6_IndexE                                                                                                          
40302f4c  _ZNSt8ios_base5_SyncE                                                                                                           
40302f50  _ZSt4_Fpz                                                                                                                       
40302fd0  _ZNSt6locale2id7_Id_cntE                                                                                                        
40302fd8  _ZNSt6locale7_Locimp8_ClocptrE                                                                                                  
40302fdc  _ZNSt7codecvtIwciE2idE                                                                                                          
40302fe0  _ZNSt5ctypeIcE2idE                                                                                                              
40302ff0  __TI_ft_end                                                                                                                     
40302ff4  __aeabi_stdin                                                                                                                   
40302ff8  __aeabi_stdout                                                                                                                  
40302ffc  __aeabi_stderr                                                                                                                  
40303000  _tz                                                                                                                             
4030301c  _lock                                                                                                                           
40303020  _unlock                                                                                                                         
40303024  __TI_cleanup_ptr                                                                                                                
40303028  __TI_dtors_ptr                                                                                                                  
4030302c  _Fenv                                                                                                                           
40303030  _Tls_setup__Fenv                                                                                                                
40303034  _ZNSt9_FacetptrISt10moneypunctIcLb0EEE6_PsaveE                                                                                  
40303038  _ZNSt9_FacetptrISt10moneypunctIcLb1EEE6_PsaveE                                                                                  
4030303c  _ZNSt9_FacetptrISt10moneypunctIwLb0EEE6_PsaveE                                                                                  
40303040  _ZNSt9_FacetptrISt10moneypunctIwLb1EEE6_PsaveE                                                                                  
40303044  _ZNSt9_FacetptrISt5ctypeIcEE6_PsaveE                                                                                            
40303048  _ZNSt9_FacetptrISt5ctypeIwEE6_PsaveE                                                                                            
4030304c  _ZNSt9_FacetptrISt7codecvtIcciEE6_PsaveE                                                                                        
40303050  _ZNSt9_FacetptrISt7codecvtIwciEE6_PsaveE                                                                                        
40303054  _ZNSt9_FacetptrISt7collateIcEE6_PsaveE                                                                                          
40303058  _ZNSt9_FacetptrISt7collateIwEE6_PsaveE                                                                                          
4030305c  _ZNSt9_FacetptrISt7num_getIcSt19istreambuf_iteratorIcSt11char_traitsIcEEEE6_PsaveE                                              
40303060  _ZNSt9_FacetptrISt7num_getIwSt19istreambuf_iteratorIwSt11char_traitsIwEEEE6_PsaveE                                              
40303064  _ZNSt9_FacetptrISt7num_putIcSt19ostreambuf_iteratorIcSt11char_traitsIcEEEE6_PsaveE                                              
40303068  _ZNSt9_FacetptrISt7num_putIwSt19ostreambuf_iteratorIwSt11char_traitsIwEEEE6_PsaveE                                              
4030306c  _ZNSt9_FacetptrISt8messagesIcEE6_PsaveE                                                                                         
40303070  _ZNSt9_FacetptrISt8messagesIwEE6_PsaveE                                                                                         
40303074  _ZNSt9_FacetptrISt8numpunctIcEE6_PsaveE                                                                                         
40303078  _ZNSt9_FacetptrISt8numpunctIwEE6_PsaveE                                                                                         
4030307c  _ZNSt9_FacetptrISt8time_getIcSt19istreambuf_iteratorIcSt11char_traitsIcEEEE6_PsaveE                                             
40303080  _ZNSt9_FacetptrISt8time_getIwSt19istreambuf_iteratorIwSt11char_traitsIwEEEE6_PsaveE                                             
40303084  _ZNSt9_FacetptrISt8time_putIcSt19ostreambuf_iteratorIcSt11char_traitsIcEEEE6_PsaveE                                             
40303088  _ZNSt9_FacetptrISt8time_putIwSt19ostreambuf_iteratorIwSt11char_traitsIwEEEE6_PsaveE                                             
4030308c  _ZNSt9_FacetptrISt9money_getIcSt19istreambuf_iteratorIcSt11char_traitsIcEEEE6_PsaveE                                            
40303090  _ZNSt9_FacetptrISt9money_getIwSt19istreambuf_iteratorIwSt11char_traitsIwEEEE6_PsaveE                                            
40303094  _ZNSt9_FacetptrISt9money_putIcSt19ostreambuf_iteratorIcSt11char_traitsIcEEEE6_PsaveE                                            
40303098  _ZNSt9_FacetptrISt9money_putIwSt19ostreambuf_iteratorIwSt11char_traitsIwEEEE6_PsaveE                                            
403030a0  _Errno                                                                                                                          
403030a8  _ZSt14_Raise_handler                                                                                                            
403030ac  main_func_sp                                                                                                                    
403030b0  _new_handler                                                                                                                    
403030b4  __CIOBUF_                                                                                                                       
403031d4  __TI_tmpnams                                                                                                                    
403032a0  _ZGVNSt10moneypunctIcLb0EE2idE                                                                                                  
403032a4  _ZGVNSt10moneypunctIcLb1EE2idE                                                                                                  
403032a8  _ZGVNSt10moneypunctIwLb0EE2idE                                                                                                  
403032ac  _ZGVNSt10moneypunctIwLb1EE2idE                                                                                                  
403032b0  _ZGVNSt7codecvtIcciE2idE                                                                                                        
403032b4  _ZGVNSt7collateIcE2idE                                                                                                          
403032b8  _ZGVNSt7collateIwE2idE                                                                                                          
403032bc  _ZGVNSt7num_getIcSt19istreambuf_iteratorIcSt11char_traitsIcEEE2idE                                                              
403032c0  _ZGVNSt7num_getIwSt19istreambuf_iteratorIwSt11char_traitsIwEEE2idE                                                              
403032c4  _ZGVNSt7num_putIcSt19ostreambuf_iteratorIcSt11char_traitsIcEEE2idE                                                              
403032c8  _ZGVNSt7num_putIwSt19ostreambuf_iteratorIwSt11char_traitsIwEEE2idE                                                              
403032cc  _ZGVNSt8messagesIcE2idE                                                                                                         
403032d0  _ZGVNSt8messagesIwE2idE                                                                                                         
403032d4  _ZGVNSt8numpunctIcE2idE                                                                                                         
403032d8  _ZGVNSt8numpunctIwE2idE                                                                                                         
403032dc  _ZGVNSt8time_getIcSt19istreambuf_iteratorIcSt11char_traitsIcEEE2idE                                                             
403032e0  _ZGVNSt8time_getIwSt19istreambuf_iteratorIwSt11char_traitsIwEEE2idE                                                             
403032e4  _ZGVNSt8time_putIcSt19ostreambuf_iteratorIcSt11char_traitsIcEEE2idE                                                             
403032e8  _ZGVNSt9money_getIcSt19istreambuf_iteratorIcSt11char_traitsIcEEE2idE                                                            
403032ec  _ZGVNSt9money_getIwSt19istreambuf_iteratorIwSt11char_traitsIwEEE2idE                                                            
403032f0  _ZGVNSt9money_putIcSt19ostreambuf_iteratorIcSt11char_traitsIcEEE2idE                                                            
403032f4  _ZGVNSt9money_putIwSt19ostreambuf_iteratorIwSt11char_traitsIwEEE2idE                                                            
403032f8  _ZNSt10moneypunctIcLb0EE2idE                                                                                                    
403032fc  _ZNSt10moneypunctIcLb1EE2idE                                                                                                    
40303300  _ZNSt10moneypunctIwLb0EE2idE                                                                                                    
40303304  _ZNSt10moneypunctIwLb1EE2idE                                                                                                    
40303308  _ZNSt13basic_filebufIcSt11char_traitsIcEE7_StinitE                                                                              
4030330c  _ZNSt13basic_filebufIwSt11char_traitsIwEE7_StinitE                                                                              
40303310  _ZNSt4fposIiE4_StzE                                                                                                             
40303314  _ZNSt7codecvtIcciE2idE                                                                                                          
40303318  _ZNSt7collateIcE2idE                                                                                                            
4030331c  _ZNSt7collateIwE2idE                                                                                                            
40303320  _ZNSt7num_getIcSt19istreambuf_iteratorIcSt11char_traitsIcEEE2idE                                                                
40303324  _ZNSt7num_getIwSt19istreambuf_iteratorIwSt11char_traitsIwEEE2idE                                                                
40303328  _ZNSt7num_putIcSt19ostreambuf_iteratorIcSt11char_traitsIcEEE2idE                                                                
4030332c  _ZNSt7num_putIwSt19ostreambuf_iteratorIwSt11char_traitsIwEEE2idE                                                                
40303330  _ZNSt8messagesIcE2idE                                                                                                           
40303334  _ZNSt8messagesIwE2idE                                                                                                           
40303338  _ZNSt8numpunctIcE2idE                                                                                                           
4030333c  _ZNSt8numpunctIwE2idE                                                                                                           
40303340  _ZNSt8time_getIcSt19istreambuf_iteratorIcSt11char_traitsIcEEE2idE                                                               
40303344  _ZNSt8time_getIwSt19istreambuf_iteratorIwSt11char_traitsIwEEE2idE                                                               
40303348  _ZNSt8time_putIcSt19ostreambuf_iteratorIcSt11char_traitsIcEEE2idE                                                               
4030334c  _ZNSt8time_putIwSt19ostreambuf_iteratorIwSt11char_traitsIwEEE2idE                                                               
40303350  _ZNSt9money_getIcSt19istreambuf_iteratorIcSt11char_traitsIcEEE2idE                                                              
40303354  _ZNSt9money_getIwSt19istreambuf_iteratorIwSt11char_traitsIwEEE2idE                                                              
40303358  _ZNSt9money_putIcSt19ostreambuf_iteratorIcSt11char_traitsIcEEE2idE                                                              
4030335c  _ZNSt9money_putIwSt19ostreambuf_iteratorIwSt11char_traitsIwEEE2idE                                                              
40303360  _ZNSt5ctypeIwE2idE                                                                                                              
40303364  _ZSt16__dummy_typeinfo                                                                                                          
40303368  __dso_handle                                                                                                                    
40303370  SHT$$INIT_ARRAY$$Base                                                                                                           
4030338c  SHT$$INIT_ARRAY$$Limit                                                                                                          
40303390  __TI_static_base__                                                                                                              
40303494  __TI_Handler_Table_Base                                                                                                         
403034a0  __TI_Handler_Table_Limit                                                                                                        
403034a8  __TI_CINIT_Base                                                                                                                 
403034b8  __TI_CINIT_Limit                                                                                                                
80001574  __TI_printfi                                                                                                                    
80001a70  __sti___10_locale_cpp_badf69ba                                                                                                  
80001b48  _ZNSt8_Locinfo8_AddcatsEiPKc                                                                                                    
80001dec  _ZNSt8_LocinfoC1EiPKc                                                                                                           
80001dec  _ZNSt8_LocinfoC2EiPKc                                                                                                           
80001f70  _ZNSt6locale7_Locimp7_AddfacEPNS_5facetEj                                                                                       
800020b0  _ZNSt6locale7_Locimp8_MakelocERKSt8_LocinfoiPS0_PKS_                                                                            
800026e8  _ZNSt6locale7_LocimpC1ERKS0_                                                                                                    
800026e8  _ZNSt6locale7_LocimpC2ERKS0_                                                                                                    
80002860  _ZNSt6localeC1ERKS_S1_i                                                                                                         
80002860  _ZNSt6localeC2ERKS_S1_i                                                                                                         
8000292c  _ZNSt6localeC1ERKS_PKci                                                                                                         
8000292c  _ZNSt6localeC2ERKS_PKci                                                                                                         
80002cc0  _ZNSt6localeC1EPKci                                                                                                             
80002cc0  _ZNSt6localeC2EPKci                                                                                                             
80002f84  _ZNSt6locale7_AddfacEPNS_5facetEjj                                                                                              
800030cc  _ZNSt6locale6globalERKS_                                                                                                        
8000322c  _ZNKSt9money_getIcSt19istreambuf_iteratorIcSt11char_traitsIcEEE8_GetmfldERS3_S5_bRSt8ios_base                                   
8000420c  __sti___11_wlocale_cpp_3b9bd5f7                                                                                                 
8000440c  _ZNSt6locale7_Locimp9_MakewlocERKSt8_LocinfoiPS0_PKS_                                                                           
800051e0  _ZNKSt9money_getIwSt19istreambuf_iteratorIwSt11char_traitsIwEEE8_GetmfldERS3_S5_bRSt8ios_base                                   
80006188  _ZNKSt7num_getIcSt19istreambuf_iteratorIcSt11char_traitsIcEEE8_GetffldEPcRS3_S6_RKSt6locale                                     
80006e40  _ZNKSt9money_putIwSt19ostreambuf_iteratorIwSt11char_traitsIwEEE8_PutmfldES3_bRSt8ios_basewbSbIwS2_SaIwEE                        
80007a44  _ZNKSt9money_putIcSt19ostreambuf_iteratorIcSt11char_traitsIcEEE8_PutmfldES3_bRSt8ios_basecbSs                                   
800085ac  __sti___11_xlocale_cpp_3609b607                                                                                                 
80008758  _ZNSt6locale7_Locimp9_MakexlocERKSt8_LocinfoiPS0_PKS_                                                                           
80009038  _ZNKSt7num_getIwSt19istreambuf_iteratorIwSt11char_traitsIwEEE8_GetffldEPcRS3_S6_RKSt6locale                                     
800099f4  __sti___11_locale0_cpp_36e19383                                                                                                 
80009a1c  _ZNSt6locale7_LocimpD1Ev                                                                                                        
80009a1c  _ZNSt6locale7_LocimpD2Ev                                                                                                        
80009ad4  _ZNSt6locale7_LocimpD0Ev                                                                                                        
80009aec  _Fac_tidy                                                                                                                       
80009b44  _Deletegloballocale                                                                                                             
80009b78  _ZNSt8_LocinfoD1Ev                                                                                                              
80009b78  _ZNSt8_LocinfoD2Ev                                                                                                              
80009c04  _ZNSt8_LocinfoC1EPKc                                                                                                            
80009c04  _ZNSt8_LocinfoC2EPKc                                                                                                            
80009df4  _Getgloballocale                                                                                                                
80009e00  _ZNSt6locale7_LocimpC1Eb                                                                                                        
80009e00  _ZNSt6locale7_LocimpC2Eb                                                                                                        
80009ef8  _Setgloballocale                                                                                                                
80009f28  _ZNSt6locale5_InitEv                                                                                                            
8000a054  _ZNSt6localeC1Ev                                                                                                                
8000a054  _ZNSt6localeC2Ev                                                                                                                
8000a088  _ZNSt6locale7classicEv                                                                                                          
8000a098  _ZNSt6locale5facet9_RegisterEv                                                                                                  
8000a0dc  _ZNSt6locale5emptyEv                                                                                                            
8000a114  _ZNKSt6localeeqERKS_                                                                                                            
8000a2f8  _ZNKSt6locale9_GetfacetEj                                                                                                       
8000a378  _ZNKSt7num_putIwSt19ostreambuf_iteratorIwSt11char_traitsIwEEE5_FputES3_RSt8ios_basewPKcjjjj                                     
8000ac80  _ZNSt8ios_baseD0Ev                                                                                                              
8000ac98  _ZNSt8ios_base8_CallfnsENS_5eventE                                                                                              
8000acd0  _ZNSt8ios_base5_TidyEv                                                                                                          
8000ad28  _ZNSt8ios_baseD1Ev                                                                                                              
8000ad28  _ZNSt8ios_baseD2Ev                                                                                                              
8000ad88  _ZNSt8ios_base5clearENSt5_IosbIiE8_IostateEb                                                                                    
8000b1a8  _ZNSt8ios_base8_FindarrEi                                                                                                       
8000b29c  _ZNSt8ios_base17register_callbackEPFvNS_5eventERS_iEi                                                                           
8000b2ec  _ZNSt8ios_base7copyfmtERKS_                                                                                                     
8000b438  _ZNSt8ios_base7_AddstdEv                                                                                                        
8000b480  _ZNSt8ios_base5imbueERKSt6locale                                                                                                
8000b4e8  _ZNSt8ios_base5_InitEv                                                                                                          
8000b558  _ZNSt6_WinitD1Ev                                                                                                                
8000b558  _ZNSt6_WinitD2Ev                                                                                                                
8000b6b8  _ZNSt6_WinitC1Ev                                                                                                                
8000b6b8  _ZNSt6_WinitC2Ev                                                                                                                
8000bbe0  __sti___12_wiostrea_cpp_9fa80e7a                                                                                                
8000bda8  _ZNKSt7num_getIcSt19istreambuf_iteratorIcSt11char_traitsIcEEE8_GetifldEPcRS3_S6_NSt5_IosbIiE9_FmtflagsERKSt6locale              
8000c4c8  _ZNKSt7num_putIcSt19ostreambuf_iteratorIcSt11char_traitsIcEEE5_FputES3_RSt8ios_basecPKcjjjj                                     
8000cbd4  _ZNKSt8time_getIwSt19istreambuf_iteratorIwSt11char_traitsIwEEE11do_get_dateES3_S3_RSt8ios_baseRNSt5_IosbIiE8_IostateEPSt2tm     
8000d2dc  __sti___12_iostream_cpp_b004430c                                                                                                
8000d474  _ZNSt8ios_base4InitD1Ev                                                                                                         
8000d474  _ZNSt8ios_base4InitD2Ev                                                                                                         
8000d56c  _ZNSt8ios_base4InitC1Ev                                                                                                         
8000d56c  _ZNSt8ios_base4InitC2Ev                                                                                                         
8000d964  _ZNKSt8time_getIcSt19istreambuf_iteratorIcSt11char_traitsIcEEE11do_get_dateES3_S3_RSt8ios_baseRNSt5_IosbIiE8_IostateEPSt2tm     
8000dfe0  minit                                                                                                                           
8000e0dc  malloc                                                                                                                          
8000e198  free                                                                                                                            
8000e2f0  realloc                                                                                                                         
8000e484  memalign                                                                                                                        
8000e5c4  calloc                                                                                                                          
8000e61c  _ZNKSt7num_getIwSt19istreambuf_iteratorIwSt11char_traitsIwEEE8_GetifldEPcRS3_S6_NSt5_IosbIiE9_FmtflagsERKSt6locale              
8000ec3c  write                                                                                                                           
8000ed34  remove                                                                                                                          
8000ed34  unlink                                                                                                                          
8000ed74  rename                                                                                                                          
8000ede0  remove_device                                                                                                                   
8000ee2c  read                                                                                                                            
8000ee70  open                                                                                                                            
8000ef88  lseek                                                                                                                           
8000efcc  close                                                                                                                           
8000f05c  add_device                                                                                                                      
8000f184  strftime                                                                                                                        
8000f69c  HOSTwrite                                                                                                                       
8000f720  HOSTunlink                                                                                                                      
8000f784  HOSTtime                                                                                                                        
8000f7e4  HOSTrename                                                                                                                      
8000f87c  HOSTread                                                                                                                        
8000f900  HOSTopen                                                                                                                        
8000f98c  HOSTlseek                                                                                                                       
8000fa2c  HOSTgetenv                                                                                                                      
8000fa94  HOSTclose                                                                                                                       
8000fafc  HOSTclock                                                                                                                       
8000fb68  _ZNKSt7num_getIwSt19istreambuf_iteratorIwSt11char_traitsIwEEE6do_getES3_S3_RSt8ios_baseRNSt5_IosbIiE8_IostateERb                
8000ffbc  _ZNKSt8time_getIwSt19istreambuf_iteratorIwSt11char_traitsIwEEE7_GetintERS3_S5_iiRi                                              
800103a0  _ZNKSt9money_putIwSt19ostreambuf_iteratorIwSt11char_traitsIwEEE6do_putES3_bRSt8ios_basewe                                       
80010768  _ZNKSt9money_getIwSt19istreambuf_iteratorIwSt11char_traitsIwEEE6do_getES3_S3_bRSt8ios_baseRNSt5_IosbIiE8_IostateERe             
80010b0c  _ZNSt13basic_filebufIwSt11char_traitsIwEE8overflowEi                                                                            
80010eb0  _ZNKSt9money_putIwSt19ostreambuf_iteratorIwSt11char_traitsIwEEE6do_putES3_bRSt8ios_basewRKSbIwS2_SaIwEE                         
80011250  _ZStlsISt11char_traitsIcEERSt13basic_ostreamIcT_ES5_PKc                                                                         
800115f0  _ZNSt13basic_filebufIcSt11char_traitsIcEE8overflowEi                                                                            
80011988  _ZNKSt7num_putIwSt19ostreambuf_iteratorIwSt11char_traitsIwEEE6do_putES3_RSt8ios_basewb                                          
80011d14  _ZNKSt7num_putIcSt19ostreambuf_iteratorIcSt11char_traitsIcEEE5_IputES3_RSt8ios_basecPcj                                         
8001209c  _ZNSt13basic_filebufIcSt11char_traitsIcEE5uflowEv                                                                               
80012414  _ZNSt13basic_filebufIwSt11char_traitsIwEE5uflowEv                                                                               
8001278c  _ZNKSt9money_putIcSt19ostreambuf_iteratorIcSt11char_traitsIcEEE6do_putES3_bRSt8ios_basece                                       
80012af4  _ZNKSt8time_getIcSt19istreambuf_iteratorIcSt11char_traitsIcEEE7_GetintERS3_S5_iiRi                                              
80012e54  strtod                                                                                                                          
80012e54  strtold                                                                                                                         
80013198  _ZNSt13basic_filebufIcSt11char_traitsIcEE9_EndwriteEv                                                                           
80013494  _ZNSt13basic_filebufIwSt11char_traitsIwEE9_EndwriteEv                                                                           
80013790  strtoll                                                                                                                         
80013bb4  __TI_cleanup                                                                                                                    
80013c00  freopen                                                                                                                         
80013c4c  fopen                                                                                                                           
80013d48  _ZNKSt7num_getIcSt19istreambuf_iteratorIcSt11char_traitsIcEEE6do_getES3_S3_RSt8ios_baseRNSt5_IosbIiE8_IostateERb                
80014010  _ZNKSt8time_putIwSt19ostreambuf_iteratorIwSt11char_traitsIwEEE6do_putES3_RSt8ios_basewPKSt2tmcc                                 
800142d4  _ZNKSt7num_putIwSt19ostreambuf_iteratorIwSt11char_traitsIwEEE5_IputES3_RSt8ios_basewPcj                                         
80014594  _ZSt10_GetloctxtIwSt19istreambuf_iteratorIwSt11char_traitsIwEEEiRT0_S5_jPKT_                                                    
80014854  __aeabi_uldivmod                                                                                                                
80014b0c  main                                                                                                                            
80014b68  _ZN4DateC1Eiii                                                                                                                  
80014b68  _ZN4DateC2Eiii                                                                                                                  
80014be8  _ZN4Date3setEiii                                                                                                                
80014c64  _ZN4Date5printEv                                                                                                                
80014cb0  __sti___14_SimpleClass_cc_main                                                                                                  
80014dc0  _ZNKSt7num_putIcSt19ostreambuf_iteratorIcSt11char_traitsIcEEE6do_putES3_RSt8ios_basecd                                          
80015060  _ZNKSt7num_putIcSt19ostreambuf_iteratorIcSt11char_traitsIcEEE6do_putES3_RSt8ios_basece                                          
80015300  _ZSt10_GetloctxtIcSt19istreambuf_iteratorIcSt11char_traitsIcEEEiRT0_S5_jPKT_                                                    
80015598  _ZNKSt9money_putIcSt19ostreambuf_iteratorIcSt11char_traitsIcEEE6do_putES3_bRSt8ios_basecRKSs                                    
800157f0  fwrite                                                                                                                          
80015a34  strtoull                                                                                                                        
80015c78  _ZNKSt7num_putIcSt19ostreambuf_iteratorIcSt11char_traitsIcEEE6do_putES3_RSt8ios_basecb                                          
80015eb4  _ZNKSt9money_getIcSt19istreambuf_iteratorIcSt11char_traitsIcEEE6do_getES3_S3_bRSt8ios_baseRNSt5_IosbIiE8_IostateERe             
800160e8  _ZNKSt7num_putIwSt19ostreambuf_iteratorIwSt11char_traitsIwEEE6do_putES3_RSt8ios_basewd                                          
80016308  _ZNKSt7num_putIwSt19ostreambuf_iteratorIwSt11char_traitsIwEEE6do_putES3_RSt8ios_basewe                                          
80016528  _ZNKSt8time_putIcSt19ostreambuf_iteratorIcSt11char_traitsIcEEE6do_putES3_RSt8ios_basecPKSt2tmcc                                 
80016744  __aeabi_dsub                                                                                                                    
80016750  __aeabi_dadd                                                                                                                    
80016958  wmemset                                                                                                                         
80016974  wmemmove                                                                                                                        
800169d0  wmemcpy                                                                                                                         
800169f0  wmemcmp                                                                                                                         
80016a30  wmemchr                                                                                                                         
80016a58  wctob                                                                                                                           
80016a88  wcslen                                                                                                                          
80016aac  wcrtomb                                                                                                                         
80016ac0  ungetwc                                                                                                                         
80016af4  mbrtowc                                                                                                                         
80016b18  fputwc                                                                                                                          
80016b2c  btowc                                                                                                                           
80016b68  _ZNKSt7collateIcE12do_transformEPKcS2_                                                                                          
80016d70  _ZNKSt7collateIwE12do_transformEPKwS2_                                                                                          
80016f74  strtol                                                                                                                          
8001716c  _ZNKSt12_String_base5_XlenEv                                                                                                    
800171f0  _ZNKSt12_String_base5_XranEv                                                                                                    
80017338  fputs                                                                                                                           
800174c8  puts                                                                                                                            
80017500  strtoul                                                                                                                         
800176c0  _Dscale                                                                                                                         
80017868  _ZNSt9basic_iosIwSt11char_traitsIwEE4initEPSt15basic_streambufIwS1_Eb                                                           
80017a08  _ZNKSt9money_getIwSt19istreambuf_iteratorIwSt11char_traitsIwEEE6do_getES3_S3_bRSt8ios_baseRNSt5_IosbIiE8_IostateERSbIwS2_SaIwEE 
80017ba4  _ZNSt9basic_iosIcSt11char_traitsIcEE4initEPSt15basic_streambufIcS1_Eb                                                           
80017d40  _ZNKSt9money_getIcSt19istreambuf_iteratorIcSt11char_traitsIcEEE6do_getES3_S3_bRSt8ios_baseRNSt5_IosbIiE8_IostateERSs            
80017ed8  _ZNSolsEi                                                                                                                       
8001806c  __cxa_finalize                                                                                                                  
800180dc  __cxa_ia64_exit                                                                                                                 
800180e4  atexit                                                                                                                          
800180fc  __aeabi_atexit                                                                                                                  
80018174  __cxa_atexit                                                                                                                    
80018200  _ZNSt7_MpunctIwE5_InitERKSt8_Locinfo                                                                                            
80018390  __aeabi_ddiv                                                                                                                    
80018520  _ZNKSt7_MpunctIwE11do_groupingEv                                                                                                
800186a4  _ZNKSt8numpunctIwE11do_groupingEv                                                                                               
80018828  __aeabi_memcpy                                                                                                                  
80018828  __aeabi_memcpy4                                                                                                                 
80018828  __aeabi_memcpy8                                                                                                                 
80018828  memcpy                                                                                                                          
800189a8  _ZNKSt8time_getIwSt19istreambuf_iteratorIwSt11char_traitsIwEEE11do_get_timeES3_S3_RSt8ios_baseRNSt5_IosbIiE8_IostateEPSt2tm     
80018b18  _ZNSt7_MpunctIcE5_InitERKSt8_Locinfo                                                                                            
80018c78  _Dnorm                                                                                                                          
80018dd8  _ZNKSt7num_putIcSt19ostreambuf_iteratorIcSt11char_traitsIcEEE5_IfmtEPcPKcNSt5_IosbIiE9_FmtflagsE                                
80018f34  setvbuf                                                                                                                         
8001908c  _ZSt21__gen_dummy_typeinfosv                                                                                                    
8001909c  _ZNSt9type_infoD1Ev                                                                                                             
8001909c  _ZNSt9type_infoD2Ev                                                                                                             
800190a0  _ZNSt9type_infoD0Ev                                                                                                             
800190b0  _ZNKSt9type_info4nameEv                                                                                                         
800190b8  _ZNKSt9type_infoneERKS_                                                                                                         
800190d8  _ZNKSt9type_infoeqERKS_                                                                                                         
800190f8  _ZNKSt9type_info6beforeERKS_                                                                                                    
80019110  _ZN10__cxxabiv129__pointer_to_member_type_infoD1Ev                                                                              
80019110  _ZN10__cxxabiv129__pointer_to_member_type_infoD2Ev                                                                              
80019114  _ZN10__cxxabiv129__pointer_to_member_type_infoD0Ev                                                                              
80019124  _ZN10__cxxabiv123__fundamental_type_infoD1Ev                                                                                    
80019124  _ZN10__cxxabiv123__fundamental_type_infoD2Ev                                                                                    
80019128  _ZN10__cxxabiv123__fundamental_type_infoD0Ev                                                                                    
80019138  _ZN10__cxxabiv121__vmi_class_type_infoD1Ev                                                                                      
80019138  _ZN10__cxxabiv121__vmi_class_type_infoD2Ev                                                                                      
8001913c  _ZN10__cxxabiv121__vmi_class_type_infoD0Ev                                                                                      
8001914c  _ZN10__cxxabiv120__si_class_type_infoD1Ev                                                                                       
8001914c  _ZN10__cxxabiv120__si_class_type_infoD2Ev                                                                                       
80019150  _ZN10__cxxabiv120__si_class_type_infoD0Ev                                                                                       
80019160  _ZN10__cxxabiv120__function_type_infoD1Ev                                                                                       
80019160  _ZN10__cxxabiv120__function_type_infoD2Ev                                                                                       
80019164  _ZN10__cxxabiv120__function_type_infoD0Ev                                                                                       
80019174  _ZN10__cxxabiv119__pointer_type_infoD1Ev                                                                                        
80019174  _ZN10__cxxabiv119__pointer_type_infoD2Ev                                                                                        
80019178  _ZN10__cxxabiv119__pointer_type_infoD0Ev                                                                                        
80019188  _ZN10__cxxabiv117__pbase_type_infoD1Ev                                                                                          
80019188  _ZN10__cxxabiv117__pbase_type_infoD2Ev                                                                                          
8001918c  _ZN10__cxxabiv117__pbase_type_infoD0Ev                                                                                          
8001919c  _ZN10__cxxabiv117__class_type_infoD1Ev                                                                                          
8001919c  _ZN10__cxxabiv117__class_type_infoD2Ev                                                                                          
800191a0  _ZN10__cxxabiv117__class_type_infoD0Ev                                                                                          
800191b0  _ZN10__cxxabiv117__array_type_infoD1Ev                                                                                          
800191b0  _ZN10__cxxabiv117__array_type_infoD2Ev                                                                                          
800191b4  _ZN10__cxxabiv117__array_type_infoD0Ev                                                                                          
800191c4  _ZN10__cxxabiv116__enum_type_infoD1Ev                                                                                           
800191c4  _ZN10__cxxabiv116__enum_type_infoD2Ev                                                                                           
800191c8  _ZN10__cxxabiv116__enum_type_infoD0Ev                                                                                           
800191e0  _ZNSt13basic_filebufIwSt11char_traitsIwEE5imbueERKSt6locale                                                                     
8001932c  _ZNSt13basic_filebufIcSt11char_traitsIcEE5imbueERKSt6locale                                                                     
80019474  _ZNKSt8time_getIcSt19istreambuf_iteratorIcSt11char_traitsIcEEE11do_get_timeES3_S3_RSt8ios_baseRNSt5_IosbIiE8_IostateEPSt2tm     
800195b8  _ZNSt13basic_filebufIcSt11char_traitsIcEE7seekoffElNSt5_IosbIiE8_SeekdirENS4_9_OpenmodeE                                        
800196ec  _ZNSt13basic_filebufIwSt11char_traitsIwEE7seekoffElNSt5_IosbIiE8_SeekdirENS4_9_OpenmodeE                                        
80019820  _ZNKSt7num_putIcSt19ostreambuf_iteratorIcSt11char_traitsIcEEE5_FfmtEPccNSt5_IosbIiE9_FmtflagsE                                  
80019950  __TI_doflush                                                                                                                    
800199d4  fflush                                                                                                                          
80019a80  _ZNSt8numpunctIcE5_InitERKSt8_Locinfo                                                                                           
80019bac  _ZNSt13basic_filebufIcSt11char_traitsIcEE7seekposESt4fposIiENSt5_IosbIiE9_OpenmodeE                                             
80019cd4  _ZNSt13basic_filebufIwSt11char_traitsIwEE7seekposESt4fposIiENSt5_IosbIiE9_OpenmodeE                                             
80019dfc  __aeabi_dmul                                                                                                                    
80019f24  _ZNKSt7num_putIcSt19ostreambuf_iteratorIcSt11char_traitsIcEEE11_PutgroupedES3_PKcjc                                             
8001a040  _ZNSbIwSt11char_traitsIwESaIwEE6insertEjjw                                                                                      
8001a15c  __TI_wrt_ok                                                                                                                     
8001a1fc  __TI_rd_ok                                                                                                                      
8001a274  _ZNKSt7_MpunctIwE14do_curr_symbolEv                                                                                             
8001a388  _ZNKSt7_MpunctIwE16do_negative_signEv                                                                                           
8001a49c  _ZNKSt7_MpunctIwE16do_positive_signEv                                                                                           
8001a5b0  _ZNKSt7num_getIcSt19istreambuf_iteratorIcSt11char_traitsIcEEE6do_getES3_S3_RSt8ios_baseRNSt5_IosbIiE8_IostateERt                
8001a6c4  _ZNKSt7num_getIwSt19istreambuf_iteratorIwSt11char_traitsIwEEE6do_getES3_S3_RSt8ios_baseRNSt5_IosbIiE8_IostateERt                
8001a7d8  _ZNKSt8numpunctIwE11do_truenameEv                                                                                               
8001a8ec  _ZNKSt8numpunctIwE12do_falsenameEv                                                                                              
8001aa00  __aeabi_idiv                                                                                                                    
8001aa00  __aeabi_idivmod                                                                                                                 
8001ab14  _ZNSs5_CopyEjj                                                                                                                  
8001ac24  _ZNSbIwSt11char_traitsIwESaIwEE6assignERKS2_jj                                                                                  
8001ad30  _ZNKSt7num_getIcSt19istreambuf_iteratorIcSt11char_traitsIcEEE6do_getES3_S3_RSt8ios_baseRNSt5_IosbIiE8_IostateERj                
8001ae38  _ZNKSt7num_getIwSt19istreambuf_iteratorIwSt11char_traitsIwEEE6do_getES3_S3_RSt8ios_baseRNSt5_IosbIiE8_IostateERj                
8001af40  _ZNSs6appendERKSsjj                                                                                                             
8001b040  _ZSt9use_facetISt10moneypunctIcLb1EEERKT_RKSt6locale                                                                            
8001b140  _ZSt9use_facetISt10moneypunctIwLb1EEERKT_RKSt6locale                                                                            
8001b240  fputc                                                                                                                           
8001b240  putc                                                                                                                            
8001b32c  putchar                                                                                                                         
8001b340  _ZNKSt7num_putIwSt19ostreambuf_iteratorIwSt11char_traitsIwEEE11_PutgroupedES3_PKcjw                                             
8001b43c  _ZNSs6insertEjjc                                                                                                                
8001b538  _ZNSt8numpunctIwE5_InitERKSt8_Locinfo                                                                                           
8001b634  _ZSt9use_facetISt10moneypunctIcLb0EEERKT_RKSt6locale                                                                            
8001b730  _ZSt9use_facetISt10moneypunctIwLb0EEERKT_RKSt6locale                                                                            
8001b82c  __TI_closefile                                                                                                                  
8001b8d8  fclose                                                                                                                          
8001b928  _ZSt9use_facetISt5ctypeIwEERKT_RKSt6locale                                                                                      
8001ba20  _ZNSs6assignERKSsjj                                                                                                             
8001bb14  __TI_buff_read                                                                                                                  
8001bc04  __aeabi_uidiv                                                                                                                   
8001bc04  __aeabi_uidivmod                                                                                                                
8001bcf4  _Getctyptab                                                                                                                     
8001bde4  _ZNKSt7num_getIcSt19istreambuf_iteratorIcSt11char_traitsIcEEE6do_getES3_S3_RSt8ios_baseRNSt5_IosbIiE8_IostateERPv               
8001bed0  _ZNKSt7num_getIcSt19istreambuf_iteratorIcSt11char_traitsIcEEE6do_getES3_S3_RSt8ios_baseRNSt5_IosbIiE8_IostateERx                
8001bfbc  _ZNKSt7num_getIcSt19istreambuf_iteratorIcSt11char_traitsIcEEE6do_getES3_S3_RSt8ios_baseRNSt5_IosbIiE8_IostateERy                
8001c0a8  _ZNKSt7num_getIwSt19istreambuf_iteratorIwSt11char_traitsIwEEE6do_getES3_S3_RSt8ios_baseRNSt5_IosbIiE8_IostateERPv               
8001c194  _ZNKSt7num_getIwSt19istreambuf_iteratorIwSt11char_traitsIwEEE6do_getES3_S3_RSt8ios_baseRNSt5_IosbIiE8_IostateERx                
8001c280  _ZNKSt7num_getIwSt19istreambuf_iteratorIwSt11char_traitsIwEEE6do_getES3_S3_RSt8ios_baseRNSt5_IosbIiE8_IostateERy                
8001c36c  _ZNSo6sentryC1ERSo                                                                                                              
8001c458  wctomb                                                                                                                          
8001c470  wcstombs                                                                                                                        
8001c4b0  mbtowc                                                                                                                          
8001c4e4  mbstowcs                                                                                                                        
8001c520  mblen                                                                                                                           
8001c544  _ZNKSt7num_getIcSt19istreambuf_iteratorIcSt11char_traitsIcEEE6do_getES3_S3_RSt8ios_baseRNSt5_IosbIiE8_IostateERl                
8001c62c  _ZNKSt7num_getIcSt19istreambuf_iteratorIcSt11char_traitsIcEEE6do_getES3_S3_RSt8ios_baseRNSt5_IosbIiE8_IostateERm                
8001c714  _ZNKSt7num_getIwSt19istreambuf_iteratorIwSt11char_traitsIwEEE6do_getES3_S3_RSt8ios_baseRNSt5_IosbIiE8_IostateERl                
8001c7fc  _ZNKSt7num_getIwSt19istreambuf_iteratorIwSt11char_traitsIwEEE6do_getES3_S3_RSt8ios_baseRNSt5_IosbIiE8_IostateERm                
8001c8e4  _ZNKSt7num_getIcSt19istreambuf_iteratorIcSt11char_traitsIcEEE6do_getES3_S3_RSt8ios_baseRNSt5_IosbIiE8_IostateERd                
8001c9c8  _ZNKSt7num_getIcSt19istreambuf_iteratorIcSt11char_traitsIcEEE6do_getES3_S3_RSt8ios_baseRNSt5_IosbIiE8_IostateERe                
8001caac  _ZNKSt7num_getIwSt19istreambuf_iteratorIwSt11char_traitsIwEEE6do_getES3_S3_RSt8ios_baseRNSt5_IosbIiE8_IostateERd                
8001cb90  _ZNKSt7num_getIwSt19istreambuf_iteratorIwSt11char_traitsIwEEE6do_getES3_S3_RSt8ios_baseRNSt5_IosbIiE8_IostateERe                
8001cc74  _ZNKSt8messagesIwE6do_getEiiiRKSbIwSt11char_traitsIwESaIwEE                                                                     
8001cd58  _ZNSs5eraseEjj                                                                                                                  
8001ce3c  _ZNKSt7num_getIcSt19istreambuf_iteratorIcSt11char_traitsIcEEE6do_getES3_S3_RSt8ios_baseRNSt5_IosbIiE8_IostateERf                
8001cf1c  _ZNKSt7num_getIwSt19istreambuf_iteratorIwSt11char_traitsIwEEE6do_getES3_S3_RSt8ios_baseRNSt5_IosbIiE8_IostateERf                
8001cffc  _ZNKSt8messagesIcE6do_getEiiiRKSs                                                                                               
8001d0dc  _ZNSt13basic_filebufIwSt11char_traitsIwEED0Ev                                                                                   
8001d1bc  _ZSt9use_facetISt8numpunctIwEERKT_RKSt6locale                                                                                   
8001d29c  __aeabi_cdcmpeq                                                                                                                 
8001d29c  __aeabi_cdcmple                                                                                                                 
8001d37c  __aeabi_cdrcmple                                                                                                                
8001d45c  fgetc                                                                                                                           
8001d45c  fgetwc                                                                                                                          
8001d45c  getc                                                                                                                            
8001d528  getchar                                                                                                                         
8001d53c  _ZNSs6appendEPKcj                                                                                                               
8001d618  _ZNKSt7codecvtIwciE6do_outERiPKwS3_RS3_PcS5_RS5_                                                                                
8001d6f0  _ZNSt13basic_filebufIwSt11char_traitsIwEED1Ev                                                                                   
8001d7c8  _ZNSs5_GrowEjb                                                                                                                  
8001d89c  _ZNSbIwSt11char_traitsIwESaIwEE6appendEjw                                                                                       
8001d96c  _ZNSt13basic_filebufIwSt11char_traitsIwEE6setbufEPwi                                                                            
8001da3c  _ZNSo3putEc                                                                                                                     
8001db08  _ZSt9use_facetISt5ctypeIcEERKT_RKSt6locale                                                                                      
8001dbd4  _ZSt9use_facetISt7num_putIcSt19ostreambuf_iteratorIcSt11char_traitsIcEEEERKT_RKSt6locale                                        
8001dca0  _ZSt9use_facetISt8numpunctIcEERKT_RKSt6locale                                                                                   
8001dd6c  _ZNSbIwSt11char_traitsIwESaIwEE5_CopyEjj                                                                                        
8001de34  _ZNSt13basic_filebufIcSt11char_traitsIcEE9pbackfailEi                                                                           
8001defc  _ZNSt13basic_filebufIwSt11char_traitsIwEE9pbackfailEi                                                                           
8001dfc4  ungetc                                                                                                                          
8001e08c  _ZNKSt7codecvtIwciE5do_inERiPKcS3_RS3_PwS5_RS5_                                                                                 
8001e14c  _Stoulx                                                                                                                         
8001e150  _Stoullx                                                                                                                        
8001e154  _Stolx                                                                                                                          
8001e158  _Stollx                                                                                                                         
8001e15c  _Stoldx                                                                                                                         
8001e1a4  _Stodx                                                                                                                          
8001e1ec  _Stofx                                                                                                                          
8001e204  _Dunscale                                                                                                                       
8001e2bc  _ZNKSt7num_putIcSt19ostreambuf_iteratorIcSt11char_traitsIcEEE6do_putES3_RSt8ios_basecPKv                                        
8001e36c  _ZNSt15basic_streambufIwSt11char_traitsIwEE6xsputnEPKwi                                                                         
8001e41c  _ZSt10_MaklocstrIwEPT_PKcS1_RKSt7_Cvtvec                                                                                        
8001e4cc  __aeabi_memclr                                                                                                                  
8001e4cc  __aeabi_memclr4                                                                                                                 
8001e4cc  __aeabi_memclr8                                                                                                                 
8001e4d0  __aeabi_memset                                                                                                                  
8001e4d0  __aeabi_memset4                                                                                                                 
8001e4d0  __aeabi_memset8                                                                                                                 
8001e4dc  memset                                                                                                                          
8001e57c  _ZNSo12_Sentry_baseC1ERSo                                                                                                       
8001e628  _ZNSt15basic_streambufIwSt11char_traitsIwEE6xsgetnEPwi                                                                          
8001e6d4  _ZNKSt8time_getIcSt19istreambuf_iteratorIcSt11char_traitsIcEEE11do_get_yearES3_S3_RSt8ios_baseRNSt5_IosbIiE8_IostateEPSt2tm     
8001e77c  _ZNKSt8time_getIwSt19istreambuf_iteratorIwSt11char_traitsIwEEE11do_get_yearES3_S3_RSt8ios_baseRNSt5_IosbIiE8_IostateEPSt2tm     
8001e824  _ZNSt13basic_filebufIcSt11char_traitsIcEE6setbufEPci                                                                            
8001e8cc  _ZNSt15basic_streambufIcSt11char_traitsIcEE6xsputnEPKci                                                                         
8001e974  fseek                                                                                                                           
8001ea1c  sprintf                                                                                                                         
8001eac4  _ZNSt15basic_streambufIcSt11char_traitsIcEE6xsgetnEPci                                                                          
8001eb68  _ZNSt5ctypeIcEC1EPKsbj                                                                                                          
8001ec0c  __TI_auto_init                                                                                                                  
8001ecb0  ftell                                                                                                                           
8001ed54  __TI_writemsg                                                                                                                   
8001ed9c  C$$IO$$                                                                                                                         
8001eda4  __TI_readmsg                                                                                                                    
8001ee98  _ZNSbIwSt11char_traitsIwESaIwEE5eraseEjj                                                                                        
8001ef34  _ZNSo12_Sentry_baseD1Ev                                                                                                         
8001efd0  _ZNSs6appendEjc                                                                                                                 
8001f06c  _ZNSt8time_getIcSt19istreambuf_iteratorIcSt11char_traitsIcEEE5_InitERKSt8_Locinfo                                               
8001f108  _ZNKSt7num_putIcSt19ostreambuf_iteratorIcSt11char_traitsIcEEE5_PutcES3_PKcj                                                     
8001f1a0  _ZNKSt7num_putIcSt19ostreambuf_iteratorIcSt11char_traitsIcEEE6do_putES3_RSt8ios_basecx                                          
8001f238  _ZNKSt7num_putIcSt19ostreambuf_iteratorIcSt11char_traitsIcEEE6do_putES3_RSt8ios_basecy                                          
8001f2d0  _ZNKSt7num_putIcSt19ostreambuf_iteratorIcSt11char_traitsIcEEE6do_putES3_RSt8ios_basecl                                          
8001f364  _ZNKSt7num_putIcSt19ostreambuf_iteratorIcSt11char_traitsIcEEE6do_putES3_RSt8ios_basecm                                          
8001f3f8  _ZNSs5_TidyEbj                                                                                                                  
8001f48c  _ZNKSt7num_putIwSt19ostreambuf_iteratorIwSt11char_traitsIwEEE6do_putES3_RSt8ios_basewPKv                                        
8001f51c  _ZNKSt7num_putIwSt19ostreambuf_iteratorIwSt11char_traitsIwEEE6do_putES3_RSt8ios_basewx                                          
8001f5ac  _ZNKSt7num_putIwSt19ostreambuf_iteratorIwSt11char_traitsIwEEE6do_putES3_RSt8ios_basewy                                          
8001f63c  _ZSt10_MaklocstrIcEPT_PKcS1_RKSt7_Cvtvec                                                                                        
8001f6cc  _ZNKSs7compareEjjPKcj                                                                                                           
8001f758  _ZNKSt7num_putIwSt19ostreambuf_iteratorIwSt11char_traitsIwEEE6do_putES3_RSt8ios_basewl                                          
8001f7e4  _ZNKSt7num_putIwSt19ostreambuf_iteratorIwSt11char_traitsIwEEE6do_putES3_RSt8ios_basewm                                          
8001f870  _ZNSt13basic_filebufIcSt11char_traitsIcEED0Ev                                                                                   
8001f8fc  _ZNKSt7codecvtIwciE10do_unshiftERiPcS2_RS2_                                                                                     
8001f984  _ZNSo5flushEv                                                                                                                   
8001fa0c  _ZNSs6assignEPKcj                                                                                                               
8001fa94  __TI_tvaltostr                                                                                                                  
8001fb1c  _ZNKSt7codecvtIwciE9do_lengthERKiPKcS4_j                                                                                        
8001fba0  _ZNSt13basic_filebufIcSt11char_traitsIcEED1Ev                                                                                   
8001fc24  atoi                                                                                                                            
8001fca8  copy_in                                                                                                                         
8001fd2c  _ZSt14_Debug_messagePKcS0_                                                                                                      
8001fd74  _ZSt6_ThrowRKSt9exception                                                                                                       
8001fdb0  ltoa                                                                                                                            
8001fe30  _ZNKSt7num_putIcSt19ostreambuf_iteratorIcSt11char_traitsIcEEE4_PutES3_PKcj                                                      
8001feac  _ZNSt19istreambuf_iteratorIcSt11char_traitsIcEEppEv                                                                             
8001ff28  _ZNSt19istreambuf_iteratorIwSt11char_traitsIwEEppEv                                                                             
8001ffa4  _ZNKSt5ctypeIwE10do_toupperEPwPKw                                                                                               
8002001c  _ZNKSt7num_putIwSt19ostreambuf_iteratorIwSt11char_traitsIwEEE5_IfmtEPcPKcNSt5_IosbIiE9_FmtflagsE                                
80020094  _ZNKSt7num_putIwSt19ostreambuf_iteratorIwSt11char_traitsIwEEE5_PutcES3_PKcj                                                     
8002010c  _ZNSt19istreambuf_iteratorIcSt11char_traitsIcEE5_PeekEv                                                                         
80020184  _ZNSt19istreambuf_iteratorIwSt11char_traitsIwEE5_PeekEv                                                                         
800201fc  C$$EXIT                                                                                                                         
80020204  abort                                                                                                                           
80020210  exit                                                                                                                            
80020274  _ZNSt12out_of_rangeC1ERKSs                                                                                                      
800202e8  _ZNSt19ostreambuf_iteratorIwSt11char_traitsIwEEaSEw                                                                             
8002035c  _ZNSt6locale5facet7_DecrefEv                                                                                                    
800203d0  _ZNKSt7num_putIwSt19ostreambuf_iteratorIwSt11char_traitsIwEEE5_FfmtEPccNSt5_IosbIiE9_FmtflagsE                                  
80020440  _ZNSt19ostreambuf_iteratorIcSt11char_traitsIcEEaSEc                                                                             
800204b0  _ZStneIcSt11char_traitsIcEEbRKSt19istreambuf_iteratorIT_T0_ES7_                                                                 
80020520  _ZStneIwSt11char_traitsIwEEbRKSt19istreambuf_iteratorIT_T0_ES7_                                                                 
80020590  _ZNKSt7num_putIcSt19ostreambuf_iteratorIcSt11char_traitsIcEEE4_RepES3_cj                                                        
800205fc  _ZNKSt5ctypeIwE10do_tolowerEPwPKw                                                                                               
80020664  _ZNSt11logic_errorC2ERKSs                                                                                                       
800206cc  _ZNSt13basic_filebufIcSt11char_traitsIcEE9underflowEv                                                                           
80020734  _ZNSt13basic_filebufIwSt11char_traitsIwEE9underflowEv                                                                           
8002079c  ldexp                                                                                                                           
80020804  _ZNKSt7collateIcE10do_compareEPKcS2_S2_S2_                                                                                      
80020868  _ZNKSt7collateIwE10do_compareEPKwS2_S2_S2_                                                                                      
800208cc  _ZNKSt7num_putIcSt19ostreambuf_iteratorIcSt11char_traitsIcEEE3putES3_RSt8ios_basecl                                             
80020930  _ZNSs9_ChassignEjjc                                                                                                             
80020994  _ZNSt5ctypeIcE7_GetcatEPPKNSt6locale5facetE                                                                                     
800209f8  _ZNSt6locale2idcvjEv                                                                                                            
80020a5c  _ZSteqIcSt11char_traitsIcEEbRKSt19istreambuf_iteratorIT_T0_ES7_                                                                 
80020ac0  _ZSteqIwSt11char_traitsIwEEbRKSt19istreambuf_iteratorIT_T0_ES7_                                                                 
80020b24  signal                                                                                                                          
80020b88  _ZNKSt5ctypeIcE10do_tolowerEPcPKc                                                                                               
80020be8  _ZNKSt5ctypeIcE10do_toupperEPcPKc                                                                                               
80020c48  _ZNKSt8time_getIcSt19istreambuf_iteratorIcSt11char_traitsIcEEE14do_get_weekdayES3_S3_RSt8ios_baseRNSt5_IosbIiE8_IostateEPSt2tm  
80020ca8  _ZNKSt8time_getIcSt19istreambuf_iteratorIcSt11char_traitsIcEEE16do_get_monthnameES3_S3_RSt8ios_baseRNSt5_IosbIiE8_IostateEPSt2tm
80020d08  _ZNKSt8time_getIwSt19istreambuf_iteratorIwSt11char_traitsIwEEE14do_get_weekdayES3_S3_RSt8ios_baseRNSt5_IosbIiE8_IostateEPSt2tm  
80020d68  _ZNKSt8time_getIwSt19istreambuf_iteratorIwSt11char_traitsIwEEE16do_get_monthnameES3_S3_RSt8ios_baseRNSt5_IosbIiE8_IostateEPSt2tm
80020dc8  _ZNSt15basic_streambufIcSt11char_traitsIcEE5_InitEv                                                                             
80020e28  _ZNSt15basic_streambufIcSt11char_traitsIcEE5sputcEc                                                                             
80020e88  _ZNSt7_MpunctIcE7_MakpatERNSt10money_base7patternEjjj                                                                           
80020ee8  _ZNSt7_MpunctIwE7_MakpatERNSt10money_base7patternEjjj                                                                           
80020f48  _ZNKSt5ctypeIwE8do_widenEPKcS2_Pw                                                                                               
80020fa4  _ZNKSt5ctypeIwE9do_narrowEPKwS2_cPc                                                                                             
80021000  _ZNSt7num_putIcSt19ostreambuf_iteratorIcSt11char_traitsIcEEE7_GetcatEPPKNSt6locale5facetE                                       
8002105c  _ZNSt7num_putIcSt19ostreambuf_iteratorIcSt11char_traitsIcEEEC1Ej                                                                
800210b8  _ZNSt8numpunctIcE7_GetcatEPPKNSt6locale5facetE                                                                                  
80021114  _ZNSt8numpunctIcEC1Ej                                                                                                           
80021170  __aeabi_d2iz                                                                                                                    
800211cc  __aeabi_d2f                                                                                                                     
80021228  _ZNSt8time_getIwSt19istreambuf_iteratorIwSt11char_traitsIwEEE5_InitERKSt8_Locinfo                                               
80021280  feraiseexcept                                                                                                                   
800212d8  _ZNSt6localeaSERKS_                                                                                                             
8002132c  _ZSt4endlIcSt11char_traitsIcEERSt13basic_ostreamIT_T0_ES6_                                                                      
80021380  _c_int00                                                                                                                        
800213d4  _ZNKSt5ctypeIwE5do_isEPKwS2_Ps                                                                                                  
80021424  _ZNKSt7num_putIwSt19ostreambuf_iteratorIwSt11char_traitsIwEEE4_RepES3_wj                                                        
80021474  _ZNKSt9basic_iosIcSt11char_traitsIcEE5widenEc                                                                                   
800214c4  _ZNSs7_InsideEPKc                                                                                                               
80021514  _ZNSt13runtime_errorD0Ev                                                                                                        
80021564  _ZNSt8ios_base7failureD0Ev                                                                                                      
800215b4  _ZNSt9money_putIcSt19ostreambuf_iteratorIcSt11char_traitsIcEEE4_PutES3_St22_String_const_iteratorIcS2_SaIcEEj                   
80021604  _ZNSt9money_putIcSt19ostreambuf_iteratorIcSt11char_traitsIcEEE4_RepES3_cj                                                       
80021654  _ZNSt9money_putIwSt19ostreambuf_iteratorIwSt11char_traitsIwEEE4_PutES3_St22_String_const_iteratorIwS2_SaIwEEj                   
800216a4  _ZNSt9money_putIwSt19ostreambuf_iteratorIwSt11char_traitsIwEEE4_RepES3_wj                                                       
800216f4  _ZNKSt5ctypeIwE11do_scan_notEsPKwS2_                                                                                            
80021740  _ZNSt13basic_filebufIcSt11char_traitsIcEE4syncEv                                                                                
8002178c  _ZNSt13basic_filebufIwSt11char_traitsIwEE4syncEv                                                                                
800217d8  _ZNSt15basic_streambufIcSt11char_traitsIcEE7seekposESt4fposIiENSt5_IosbIiE9_OpenmodeE                                           
80021824  _ZNSt15basic_streambufIwSt11char_traitsIwEE7seekposESt4fposIiENSt5_IosbIiE9_OpenmodeE                                           
80021870  _ZNSt6localeD1Ev                                                                                                                
800218bc  _Znaj                                                                                                                           
800218bc  _Znwj                                                                                                                           
80021908  raise                                                                                                                           
80021954  _ZNKSt15basic_streambufIcSt11char_traitsIcEE8_PnavailEv                                                                         
8002199c  _ZNKSt5ctypeIwE10do_toupperEw                                                                                                   
800219e4  _ZNSt5ctypeIcE5_TidyEv                                                                                                          
80021a2c  setlocale                                                                                                                       
80021a64  localeconv                                                                                                                      
80021a74  strncpy                                                                                                                         
80021abc  _ZNKSt5ctypeIwE10do_scan_isEsPKwS2_                                                                                             
80021b00  _ZNKSt8_Locinfo9_GetctypeEv                                                                                                     
80021b44  _ZNSsC1EPKc                                                                                                                     
80021b88  _ZNSt10moneypunctIcLb0EED0Ev                                                                                                    
80021bcc  _ZNSt10moneypunctIcLb1EED0Ev                                                                                                    
80021c10  _ZNSt10moneypunctIwLb0EED0Ev                                                                                                    
80021c54  _ZNSt10moneypunctIwLb1EED0Ev                                                                                                    
80021c98  _ZNSt11logic_errorD0Ev                                                                                                          
80021cdc  _ZNSt12length_errorD0Ev                                                                                                         
80021d20  _ZNSt12out_of_rangeD0Ev                                                                                                         
80021d64  _ZNSt13runtime_errorD1Ev                                                                                                        
80021da8  _ZNSt15basic_streambufIcSt11char_traitsIcEE7seekoffElNSt5_IosbIiE8_SeekdirENS4_9_OpenmodeE                                      
80021dec  _ZNSt15basic_streambufIwSt11char_traitsIwEE7seekoffElNSt5_IosbIiE8_SeekdirENS4_9_OpenmodeE                                      
80021e30  _ZNSt7_MpunctIcED0Ev                                                                                                            
80021e74  _ZNSt7_MpunctIwED0Ev                                                                                                            
80021eb8  _ZNSt8ios_base7failureD1Ev                                                                                                      
80021efc  strcspn                                                                                                                         
80021f40  _Feraise                                                                                                                        
80021f84  _ZNKSt5ctypeIwE10do_tolowerEw                                                                                                   
80021fc4  _ZNSbIwSt11char_traitsIwESaIwEE9_ChassignEjjw                                                                                   
80022004  _ZNSt6locale5facet7_IncrefEv                                                                                                    
80022044  _ZNSt9basic_iosIcSt11char_traitsIcEE5clearENSt5_IosbIiE8_IostateEb                                                              
80022084  _ZNSt9basic_iosIcSt11char_traitsIcEE8setstateENSt5_IosbIiE8_IostateEb                                                           
800220c4  _ZNKSt5ctypeIcE8do_widenEPKcS2_Pc                                                                                               
80022100  _ZNKSt5ctypeIcE9do_narrowEPKcS2_cPc                                                                                             
8002213c  _ZNKSt7_MpunctIcE11do_groupingEv                                                                                                
80022178  _ZNKSt7_MpunctIcE14do_curr_symbolEv                                                                                             
800221b4  _ZNKSt7_MpunctIcE16do_negative_signEv                                                                                           
800221f0  _ZNKSt7_MpunctIcE16do_positive_signEv                                                                                           
8002222c  _ZNKSt9exception6_RaiseEv                                                                                                       
80022268  _ZNSo5_OsfxEv                                                                                                                   
800222a4  _ZNSt10moneypunctIcLb0EED1Ev                                                                                                    
800222e0  _ZNSt10moneypunctIcLb1EED1Ev                                                                                                    
8002231c  _ZNSt10moneypunctIwLb0EED1Ev                                                                                                    
80022358  _ZNSt10moneypunctIwLb1EED1Ev                                                                                                    
80022394  _ZNSt11logic_errorD1Ev                                                                                                          
800223d0  _ZNSt12length_errorD1Ev                                                                                                         
8002240c  _ZNSt12out_of_rangeD1Ev                                                                                                         
80022448  _ZNSt7_MpunctIcED1Ev                                                                                                            
80022484  _ZNSt7_MpunctIwED1Ev                                                                                                            
800224c0  _ZNSt8numpunctIwED0Ev                                                                                                           
800224fc  __aeabi_i2d                                                                                                                     
80022538  _ZNKSt5ctypeIwE5do_isEsw                                                                                                        
80022570  _ZNSs4_EosEj                                                                                                                    
800225a8  _ZNSt15basic_streambufIcSt11char_traitsIcEE5uflowEv                                                                             
800225e0  _ZNSt15basic_streambufIwSt11char_traitsIwEE5uflowEv                                                                             
80022618  _ZNSt5ctypeIwED0Ev                                                                                                              
80022650  memmove                                                                                                                         
80022688  _Dclass                                                                                                                         
800226c0  _ZNKSs6_MyptrEv                                                                                                                 
800226f4  _ZNKSs8max_sizeEv                                                                                                               
80022728  _ZNKSt5ctypeIwE8do_widenEc                                                                                                      
8002275c  _ZNSs6_MyptrEv                                                                                                                  
80022790  _ZNSsC1Ev                                                                                                                       
800227c4  _ZNSt11char_traitsIcE11eq_int_typeERKiS2_                                                                                       
800227f8  _ZNSt6locale5facetC1Ej                                                                                                          
8002282c  _ZNSt8numpunctIwED1Ev                                                                                                           
80022860  _ZNSt8time_getIcSt19istreambuf_iteratorIcSt11char_traitsIcEEED0Ev                                                               
80022894  _ZNSt8time_getIwSt19istreambuf_iteratorIwSt11char_traitsIwEEED0Ev                                                               
800228c8  __cxa_guard_release                                                                                                             
800228d8  __cxa_guard_acquire                                                                                                             
800228ec  __cxa_guard_abort                                                                                                               
800228fc  memcmp                                                                                                                          
80022930  _ZNKSaIcE8max_sizeEv                                                                                                            
80022960  _ZNKSt5ctypeIwE9do_narrowEwc                                                                                                    
80022990  _ZNSt10ctype_baseC1Ej                                                                                                           
800229c0  _ZNSt15basic_streambufIcSt11char_traitsIcEE5sputnEPKci                                                                          
800229f0  _ZNSt19ostreambuf_iteratorIcSt11char_traitsIcEEC1EPSt15basic_streambufIcS1_E                                                    
80022a20  _ZNSt5ctypeIcED1Ev                                                                                                              
80022a50  _ZNSt5ctypeIwED1Ev                                                                                                              
80022a80  _ZNSt6localeC1ERKS_                                                                                                             
80022ab0  _ZNSt8ios_base5widthEi                                                                                                          
80022ae0  _ZNSt8numpunctIcE5_TidyEv                                                                                                       
80022b10  _ZNSt8numpunctIcED1Ev                                                                                                           
80022b40  _ZSt10_MaklocchrIwET_cPS0_RKSt7_Cvtvec                                                                                          
80022b70  _ZStoRRNSt5_IosbIiE8_IostateES1_                                                                                                
80022ba0  fgetpos                                                                                                                         
80022bd0  frexp                                                                                                                           
80022c00  _ZNSt15basic_streambufIcSt11char_traitsIcEED0Ev                                                                                 
80022c2c  _ZNSt15basic_streambufIwSt11char_traitsIwEED0Ev                                                                                 
80022c58  _ZNSt8time_getIcSt19istreambuf_iteratorIcSt11char_traitsIcEEED1Ev                                                               
80022c84  _ZNSt8time_getIwSt19istreambuf_iteratorIwSt11char_traitsIwEEED1Ev                                                               
80022cb0  memccpy                                                                                                                         
80022cdc  memchr                                                                                                                          
80022d08  strcat                                                                                                                          
80022d34  _ZNKSt5ctypeIcE5widenEc                                                                                                         
80022d5c  _ZNKSt7collateIwE7do_hashEPKwS2_                                                                                                
80022d84  _ZNKSt8ios_base4failEv                                                                                                          
80022dac  _ZNKSt8ios_base4goodEv                                                                                                          
80022dd4  _ZNKSt8numpunctIcE8groupingEv                                                                                                   
80022dfc  _ZNKSt8numpunctIcE8truenameEv                                                                                                   
80022e24  _ZNKSt8numpunctIcE9falsenameEv                                                                                                  
80022e4c  _ZNSs6assignEPKc                                                                                                                
80022e74  _ZNSt10ctype_baseD0Ev                                                                                                           
80022e9c  _ZNSt5ctypeIcED0Ev                                                                                                              
80022ec4  _ZNSt6locale5facetD0Ev                                                                                                          
80022eec  _ZNSt7num_putIcSt19ostreambuf_iteratorIcSt11char_traitsIcEEED0Ev                                                                
80022f14  _ZNSt8numpunctIcED0Ev                                                                                                           
80022f3c  _ZTv0_n12_NSiD0Ev                                                                                                               
80022f64  _ZTv0_n12_NSoD0Ev                                                                                                               
80022f8c  _ZTv0_n12_NSt13basic_istreamIwSt11char_traitsIwEED0Ev                                                                           
80022fb4  _ZTv0_n12_NSt13basic_ostreamIwSt11char_traitsIwEED0Ev                                                                           
80022fdc  strchr                                                                                                                          
80023004  strcmp                                                                                                                          
8002302c  _ZNKSt5ctypeIcE10do_tolowerEc                                                                                                   
80023050  _ZNKSt5ctypeIcE10do_toupperEc                                                                                                   
80023074  _ZNKSt7collateIcE7do_hashEPKcS2_                                                                                                
80023098  _ZNKSt8_Locinfo7_GetcvtEv                                                                                                       
800230bc  _ZNSo6sentryD1Ev                                                                                                                
800230e0  _ZNSs6assignERKSs                                                                                                               
80023104  _ZNSt11char_traitsIcE4copyEPcPKcj                                                                                               
80023128  _ZNSt11char_traitsIcE4moveEPcPKcj                                                                                               
8002314c  _ZNSt11char_traitsIcE6assignEPcjc                                                                                               
80023170  _ZNSt11char_traitsIcE6assignERcRKc                                                                                              
80023194  _ZNSt15basic_streambufIcSt11char_traitsIcEE6_PnincEv                                                                            
800231b8  _ZNSt15basic_streambufIcSt11char_traitsIcEED1Ev                                                                                 
800231dc  _ZNSt15basic_streambufIwSt11char_traitsIwEED1Ev                                                                                 
80023200  _ZNSt6locale2idC1Ej                                                                                                             
80023224  _register_unlock                                                                                                                
80023230  _register_lock                                                                                                                  
8002323c  _nop                                                                                                                            
80023248  _ZNKSt8ios_base6getlocEv                                                                                                        
80023268  _ZNKSt8numpunctIcE11do_groupingEv                                                                                               
80023288  _ZNKSt8numpunctIcE11do_truenameEv                                                                                               
800232a8  _ZNKSt8numpunctIcE12do_falsenameEv                                                                                              
800232c8  _ZNKSt8numpunctIcE13decimal_pointEv                                                                                             
800232e8  _ZNKSt8numpunctIcE13thousands_sepEv                                                                                             
80023308  _ZNSiD0Ev                                                                                                                       
80023328  _ZNSoD0Ev                                                                                                                       
80023348  _ZNSsD1Ev                                                                                                                       
80023368  _ZNSsixEj                                                                                                                       
80023388  _ZNSt11_String_valIcSaIcEEC1ES0_                                                                                                
800233a8  _ZNSt13basic_istreamIwSt11char_traitsIwEED0Ev                                                                                   
800233c8  _ZNSt13basic_ostreamIwSt11char_traitsIwEED0Ev                                                                                   
800233e8  _ZNSt15basic_streambufIcSt11char_traitsIcEE7pubsyncEv                                                                           
80023408  _ZNSt5ctypeIcE5_InitERKSt8_Locinfo                                                                                              
80023428  _ZNSt7num_putIcSt19ostreambuf_iteratorIcSt11char_traitsIcEEE5_InitERKSt8_Locinfo                                                
80023448  _ZStanNSt5_IosbIiE9_FmtflagsES1_                                                                                                
80023468  _ZTv0_n12_NSiD1Ev                                                                                                               
80023488  _ZTv0_n12_NSoD1Ev                                                                                                               
800234a8  _ZTv0_n12_NSt13basic_istreamIwSt11char_traitsIwEED1Ev                                                                           
800234c8  _ZTv0_n12_NSt13basic_ostreamIwSt11char_traitsIwEED1Ev                                                                           
800234e8  _args_main                                                                                                                      
80023508  _ZNKSt5ctypeIcE9do_narrowEcc                                                                                                    
80023524  _ZNKSt7codecvtIcciE5do_inERiPKcS3_RS3_PcS5_RS5_                                                                                 
80023540  _ZNKSt7codecvtIcciE6do_outERiPKcS3_RS3_PcS5_RS5_                                                                                
8002355c  _ZNSaIcE10deallocateEPcj                                                                                                        
80023578  _ZNSaIcE8allocateEj                                                                                                             
80023594  _ZNSolsEPFRSoS_E                                                                                                                
800235b0  _ZSt10_MaklocchrIcET_cPS0_RKSt7_Cvtvec                                                                                          
800235cc  _ZSt8_ToloweriPKSt9_Ctypevec                                                                                                    
800235e8  _ZSt8_ToupperiPKSt9_Ctypevec                                                                                                    
80023604  strlen                                                                                                                          
80023620  _ZNKSo6sentrycvbEv                                                                                                              
80023638  _ZNKSs4sizeEv                                                                                                                   
80023650  _ZNKSt11logic_error4whatEv                                                                                                      
80023668  _ZNKSt13runtime_error4whatEv                                                                                                    
80023680  _ZNKSt19ostreambuf_iteratorIcSt11char_traitsIcEE6failedEv                                                                       
80023698  _ZNKSt5ctypeIcE8do_widenEc                                                                                                      
800236b0  _ZNKSt8_Locinfo8_GettrueEv                                                                                                      
800236c8  _ZNKSt8_Locinfo9_GetfalseEv                                                                                                     
800236e0  _ZNKSt8ios_base5flagsEv                                                                                                         
800236f8  _ZNKSt8ios_base5widthEv                                                                                                         
80023710  _ZNKSt8ios_base7rdstateEv                                                                                                       
80023728  _ZNKSt8ios_base9precisionEv                                                                                                     
80023740  _ZNKSt8numpunctIcE16do_decimal_pointEv                                                                                          
80023758  _ZNKSt8numpunctIcE16do_thousands_sepEv                                                                                          
80023770  _ZNKSt9basic_iosIcSt11char_traitsIcEE3tieEv                                                                                     
80023788  _ZNKSt9basic_iosIcSt11char_traitsIcEE4fillEv                                                                                    
800237a0  _ZNKSt9basic_iosIcSt11char_traitsIcEE5rdbufEv                                                                                   
800237b8  _ZNSaIcEC1ERKS_                                                                                                                 
800237d0  _ZNSiD1Ev                                                                                                                       
800237e8  _ZNSoD1Ev                                                                                                                       
80023800  _ZNSt10ctype_baseD1Ev                                                                                                           
80023818  _ZNSt11char_traitsIcE11to_int_typeERKc                                                                                          
80023830  _ZNSt13basic_istreamIwSt11char_traitsIwEED1Ev                                                                                   
80023848  _ZNSt13basic_ostreamIwSt11char_traitsIwEED1Ev                                                                                   
80023860  _ZNSt7_LockitC1Ei                                                                                                               
80023878  _ZNSt7num_putIcSt19ostreambuf_iteratorIcSt11char_traitsIcEEED1Ev                                                                
80023890  _ZNSt9basic_iosIcSt11char_traitsIcEED0Ev                                                                                        
800238a8  _ZNSt9basic_iosIwSt11char_traitsIwEED0Ev                                                                                        
800238c0  _ZSt9_AllocateIcEPT_jS1_                                                                                                        
800238d8  strcpy                                                                                                                          
800238f0  tolower                                                                                                                         
80023908  toupper                                                                                                                         
80023920  _ZNKSs5c_strEv                                                                                                                  
80023934  _ZNKSt5ctypeIwE2isEsw                                                                                                           
80023948  _ZNKSt5ctypeIwE5widenEc                                                                                                         
8002395c  _ZNKSt5ctypeIwE6narrowEwc                                                                                                       
80023970  _ZNKSt7codecvtIcciE9do_lengthERKiPKcS4_j                                                                                        
80023984  _ZNKSt8numpunctIwE13thousands_sepEv                                                                                             
80023998  _ZNKSt8numpunctIwE8groupingEv                                                                                                   
800239ac  _ZNKSt8numpunctIwE9falsenameEv                                                                                                  
800239c0  _ZNSaIcEC1Ev                                                                                                                    
800239d4  _ZNSo12_Sentry_baseC2ERSo                                                                                                       
800239e8  _ZNSt10ctype_baseC2Ej                                                                                                           
800239fc  _ZNSt11_String_valIcSaIcEEC2ES0_                                                                                                
80023a10  _ZNSt11char_traitsIcE6lengthEPKc                                                                                                
80023a24  _ZNSt19ostreambuf_iteratorIcSt11char_traitsIcEEdeEv                                                                             
80023a38  _ZNSt19ostreambuf_iteratorIcSt11char_traitsIcEEppEv                                                                             
80023a4c  _ZNSt6locale5facetC2Ej                                                                                                          
80023a60  _ZNSt6locale5facetD1Ev                                                                                                          
80023a74  _ZNSt7_LockitD1Ev                                                                                                               
80023a88  __TI_decompress_none                                                                                                            
80023a9c  _ZNKSt7codecvtIcciE10do_unshiftERiPcS2_RS2_                                                                                     
80023aac  _ZNKSt8_Locinfo9_GetlconvEv                                                                                                     
80023abc  _ZNSo12_Sentry_baseD2Ev                                                                                                         
80023acc  _ZNSt10ctype_baseD2Ev                                                                                                           
80023adc  _ZNSt10money_baseD0Ev                                                                                                           
80023aec  _ZNSt12codecvt_baseD0Ev                                                                                                         
80023afc  _ZNSt13messages_baseD0Ev                                                                                                        
80023b0c  _ZNSt6locale5facetD2Ev                                                                                                          
80023b1c  _ZNSt7codecvtIcciED0Ev                                                                                                          
80023b2c  _ZNSt7codecvtIwciED0Ev                                                                                                          
80023b3c  _ZNSt7collateIcED0Ev                                                                                                            
80023b4c  _ZNSt7collateIwED0Ev                                                                                                            
80023b5c  _ZNSt7num_getIcSt19istreambuf_iteratorIcSt11char_traitsIcEEED0Ev                                                                
80023b6c  _ZNSt7num_getIwSt19istreambuf_iteratorIwSt11char_traitsIwEEED0Ev                                                                
80023b7c  _ZNSt7num_putIwSt19ostreambuf_iteratorIwSt11char_traitsIwEEED0Ev                                                                
80023b8c  _ZNSt8messagesIcED0Ev                                                                                                           
80023b9c  _ZNSt8messagesIwED0Ev                                                                                                           
80023bac  _ZNSt8time_putIcSt19ostreambuf_iteratorIcSt11char_traitsIcEEED0Ev                                                               
80023bbc  _ZNSt8time_putIwSt19ostreambuf_iteratorIwSt11char_traitsIwEEED0Ev                                                               
80023bcc  _ZNSt9bad_allocD0Ev                                                                                                             
80023bdc  _ZNSt9exceptionD0Ev                                                                                                             
80023bec  _ZNSt9money_getIcSt19istreambuf_iteratorIcSt11char_traitsIcEEED0Ev                                                              
80023bfc  _ZNSt9money_getIwSt19istreambuf_iteratorIwSt11char_traitsIwEEED0Ev                                                              
80023c0c  _ZNSt9money_putIcSt19ostreambuf_iteratorIcSt11char_traitsIcEEED0Ev                                                              
80023c1c  _ZNSt9money_putIwSt19ostreambuf_iteratorIwSt11char_traitsIwEEED0Ev                                                              
80023c2c  _ZNSt9time_baseD0Ev                                                                                                             
80023c3c  __TI_zero_init                                                                                                                  
80023c4c  _ZdaPv                                                                                                                          
80023c4c  _ZdlPv                                                                                                                          
80023c5c  fsetpos                                                                                                                         
80023c68  _ZNKSt12codecvt_base11do_encodingEv                                                                                             
80023c70  _ZNKSt12codecvt_base13do_max_lengthEv                                                                                           
80023c78  _ZNKSt12codecvt_base16do_always_noconvEv                                                                                        
80023c80  _ZNKSt7_MpunctIcE13do_neg_formatEv                                                                                              
80023c88  _ZNKSt7_MpunctIcE13do_pos_formatEv                                                                                              
80023c90  _ZNKSt7_MpunctIcE14do_frac_digitsEv                                                                                             
80023c98  _ZNKSt7_MpunctIcE16do_decimal_pointEv                                                                                           
80023ca0  _ZNKSt7_MpunctIcE16do_thousands_sepEv                                                                                           
80023ca8  _ZNKSt7_MpunctIwE13do_neg_formatEv                                                                                              
80023cb0  _ZNKSt7_MpunctIwE13do_pos_formatEv                                                                                              
80023cb8  _ZNKSt7_MpunctIwE14do_frac_digitsEv                                                                                             
80023cc0  _ZNKSt7_MpunctIwE16do_decimal_pointEv                                                                                           
80023cc8  _ZNKSt7_MpunctIwE16do_thousands_sepEv                                                                                           
80023cd0  _ZNKSt7codecvtIwciE11do_encodingEv                                                                                              
80023cd8  _ZNKSt7codecvtIwciE13do_max_lengthEv                                                                                            
80023ce0  _ZNKSt7codecvtIwciE16do_always_noconvEv                                                                                         
80023ce8  _ZNKSt8messagesIcE7do_openERKSsRKSt6locale                                                                                      
80023cf0  _ZNKSt8messagesIwE7do_openERKSsRKSt6locale                                                                                      
80023cf8  _ZNKSt8numpunctIwE16do_decimal_pointEv                                                                                          
80023d00  _ZNKSt8numpunctIwE16do_thousands_sepEv                                                                                          
80023d08  _ZNKSt8time_getIcSt19istreambuf_iteratorIcSt11char_traitsIcEEE13do_date_orderEv                                                 
80023d10  _ZNKSt8time_getIwSt19istreambuf_iteratorIwSt11char_traitsIwEEE13do_date_orderEv                                                 
80023d18  _ZNKSt9exception4whatEv                                                                                                         
80023d20  _ZNSt11char_traitsIcE3eofEv                                                                                                     
80023d28  _ZNSt15basic_streambufIcSt11char_traitsIcEE4syncEv                                                                              
80023d30  _ZNSt15basic_streambufIcSt11char_traitsIcEE8overflowEi                                                                          
80023d38  _ZNSt15basic_streambufIcSt11char_traitsIcEE9pbackfailEi                                                                         
80023d40  _ZNSt15basic_streambufIcSt11char_traitsIcEE9showmanycEv                                                                         
80023d48  _ZNSt15basic_streambufIcSt11char_traitsIcEE9underflowEv                                                                         
80023d50  _ZNSt15basic_streambufIwSt11char_traitsIwEE4syncEv                                                                              
80023d58  _ZNSt15basic_streambufIwSt11char_traitsIwEE8overflowEi                                                                          
80023d60  _ZNSt15basic_streambufIwSt11char_traitsIwEE9pbackfailEi                                                                         
80023d68  _ZNSt15basic_streambufIwSt11char_traitsIwEE9showmanycEv                                                                         
80023d70  _ZNSt15basic_streambufIwSt11char_traitsIwEE9underflowEv                                                                         
80023d78  __TI_decompress_rle24                                                                                                           
80023d80  _ZnwjPv                                                                                                                         
80023d88  _system_pre_init                                                                                                                
80023d90  _ZNKSt11logic_error8_DoraiseEv                                                                                                  
80023d94  _ZNKSt12length_error8_DoraiseEv                                                                                                 
80023d98  _ZNKSt12out_of_range8_DoraiseEv                                                                                                 
80023d9c  _ZNKSt13runtime_error8_DoraiseEv                                                                                                
80023da0  _ZNKSt8ios_base7failure8_DoraiseEv                                                                                              
80023da4  _ZNKSt8messagesIcE8do_closeEi                                                                                                   
80023da8  _ZNKSt8messagesIwE8do_closeEi                                                                                                   
80023dac  _ZNKSt9bad_alloc8_DoraiseEv                                                                                                     
80023db0  _ZNKSt9exception8_DoraiseEv                                                                                                     
80023db4  _ZNSt10money_baseD1Ev                                                                                                           
80023db8  _ZNSt12codecvt_baseD1Ev                                                                                                         
80023dbc  _ZNSt13messages_baseD1Ev                                                                                                        
80023dc0  _ZNSt15basic_streambufIcSt11char_traitsIcEE5_LockEv                                                                             
80023dc4  _ZNSt15basic_streambufIcSt11char_traitsIcEE5imbueERKSt6locale                                                                   
80023dc8  _ZNSt15basic_streambufIcSt11char_traitsIcEE6setbufEPci                                                                          
80023dcc  _ZNSt15basic_streambufIcSt11char_traitsIcEE7_UnlockEv                                                                           
80023dd0  _ZNSt15basic_streambufIwSt11char_traitsIwEE5_LockEv                                                                             
80023dd4  _ZNSt15basic_streambufIwSt11char_traitsIwEE5imbueERKSt6locale                                                                   
80023dd8  _ZNSt15basic_streambufIwSt11char_traitsIwEE6setbufEPwi                                                                          
80023ddc  _ZNSt15basic_streambufIwSt11char_traitsIwEE7_UnlockEv                                                                           
80023de0  _ZNSt7codecvtIcciED1Ev                                                                                                          
80023de4  _ZNSt7codecvtIwciED1Ev                                                                                                          
80023de8  _ZNSt7collateIcED1Ev                                                                                                            
80023dec  _ZNSt7collateIwED1Ev                                                                                                            
80023df0  _ZNSt7num_getIcSt19istreambuf_iteratorIcSt11char_traitsIcEEED1Ev                                                                
80023df4  _ZNSt7num_getIwSt19istreambuf_iteratorIwSt11char_traitsIwEEED1Ev                                                                
80023df8  _ZNSt7num_putIwSt19ostreambuf_iteratorIwSt11char_traitsIwEEED1Ev                                                                
80023dfc  _ZNSt8messagesIcED1Ev                                                                                                           
80023e00  _ZNSt8messagesIwED1Ev                                                                                                           
80023e04  _ZNSt8time_putIcSt19ostreambuf_iteratorIcSt11char_traitsIcEEED1Ev                                                               
80023e08  _ZNSt8time_putIwSt19ostreambuf_iteratorIwSt11char_traitsIwEEED1Ev                                                               
80023e0c  _ZNSt9bad_allocD1Ev                                                                                                             
80023e10  _ZNSt9basic_iosIcSt11char_traitsIcEED1Ev                                                                                        
80023e14  _ZNSt9basic_iosIwSt11char_traitsIwEED1Ev                                                                                        
80023e18  _ZNSt9exceptionD1Ev                                                                                                             
80023e1c  _ZNSt9money_getIcSt19istreambuf_iteratorIcSt11char_traitsIcEEED1Ev                                                              
80023e20  _ZNSt9money_getIwSt19istreambuf_iteratorIwSt11char_traitsIwEEED1Ev                                                              
80023e24  _ZNSt9money_putIcSt19ostreambuf_iteratorIcSt11char_traitsIcEEED1Ev                                                              
80023e28  _ZNSt9money_putIwSt19ostreambuf_iteratorIwSt11char_traitsIwEEED1Ev                                                              
80023e2c  _ZNSt9time_baseD1Ev                                                                                                             
80023e30  __aeabi_idiv0                                                                                                                   
80023e34  _Z21__default_new_handlerv                                                                                                      
80023e38  _Atexit                                                                                                                         
ffffffff  __binit__                                                                                                                       
ffffffff  __c_args__                                                                                                                      
ffffffff  binit                                                                                                                           

[1142 symbols]
